:020000040800F2
:104000000050002075C30008719F0008759F0008CC
:10401000799F00087D9F0008819F00080000000034
:10402000000000000000000000000000899F000860
:10403000859F0008000000008D9F0008A1E1000896
:10404000919F0008959F0008999F00089D9F000878
:10405000A19F0008A59F0008A99F0008AD9F000828
:1040600031790008B19F0008B59F000800000000EA
:104070000000000000000000000000000000000040
:104080000000000000000000D59F0008D99F000834
:10409000E99F0008F99F000815A00008A179000811
:1040A00025A0000829850008B18100080000000053
:1040B0004D7E0008E5780008B17D000829A00008C1
:1040C0002DA0000831A0000835A0000839A0000884
:1040D0003DA0000841A0000845A0000899A00008E4
:1040E00049A000084DA0000851A0000800000000F1
:1040F00000000000000000000000000000000000C0
:0C41000000000000000000005FF800005C
:1041100030BF704720BF704740BF7047BFF36F8FFD
:104120007047BFF34F8F7047BFF35F8F704701DF5A
:104130007047EFF31480704780F31488BFF36F8FDC
:104140007047EFF30980704780F309887047EFF3F9
:104150000880704780F30888704772B6704762B66F
:10416000704771B6704761B6704780F31188704729
:10417000EFF31280704740BA704700BA70470000F2
:1041800038B506F0C9FD424B00254FF480301D7054
:1041900006F0E2FD06F046FF0128044627D1102074
:1041A00006F0CCFA022006F0B1FA284606F024FE0A
:1041B000284606F035FE4FF4806006F027FE4FF4E7
:1041C00080304FF4E01106F0F3FD204606F0FCFDD0
:1041D000392006F011FF0028FAD0022006F0FAFD7F
:1041E00006F002FE0828FBD1294B01221A7001209B
:1041F000014606F0B7FE4FF480414FF0006006F034
:10420000ADFC4FF4407006F00BFC2249224A234BD0
:104210001160234A234C136001222270224A234D4D
:104220001360234A13600BF071F80BF09BF800F059
:10423000ADF80AF0AFFF0BF053FA09F0F5FF0BF001
:104240003BF8287809F060FDE87809F0D5FC237880
:104250000BB105F071FE04F03BFB01F03BFA0BF0F3
:10426000BBFA40F2127009F01FFF40F2167009F01D
:104270008BFF104809F018FE02F030FE04F0D8FB66
:1042800003F0DCFE0BF0AAFA09F0ECFEF4E700BF45
:1042900068090020B99D0008740900200573000812
:1042A0006009002050090020540900200800002067
:1042B0005C0900204C00002070B5314B86B01B78A3
:1042C000044683420D46164633D02E48002106F0A0
:1042D00017FF4FF00003ADF804304FF48273ADF8D0
:1042E00006304FF00003ADF808304FF00203ADF890
:1042F0000A304FF00103ADF80C304FF40073ADF805
:104300000E304FF00003ADF81230ADF8143014B990
:104310004FF0100301E04FF018031A4801A9ADF85F
:10432000103006F0B1FE1748012106F0E9FE144BEB
:104330001C7014B1032C20D102E0134B10225A61DF
:104340001048022106F070FF0028F9D029460D48D8
:1043500006F00EFF0B48012106F066FF0028F9D099
:1043600036B114B1032C08D102E0074B10221A61B8
:10437000044806F0FFFEC0B200E0002006B070BDA9
:10438000640200200030014000080140F0B54FF405
:10439000805087B0012106F0E5FD264F012001463F
:1043A00005AE06F0DFFD18244FF0A00203253146CC
:1043B0003846ADF814208DF816508DF8174006F0E9
:1043C000C9F94FF0400331463846ADF814308DF846
:1043D00016508DF8174006F0BDF90120002106F0B7
:1043E00049FA154E4FF48272ADF802204FF00202E6
:1043F0000023012530466946ADF806204FF40072CF
:10440000ADF81030ADF80030ADF80430ADF80A204A
:10441000ADF80E30ADF80C40ADF8085006F034FEA3
:104420003046294606F06CFE044B4FF0FF321A70FE
:1044300007B0F0BD000801400030014064020020D8
:1044400008B5A64A9378002B40F03F845378A32BFD
:1044500000F07A8200F28380822B00F09D813CD8AC
:10446000092B00F0488119D8042B00F00C8109D8E1
:10447000012B00F0FE80002B00F0F680022B40F0B4
:104480002084FBE0062B00F01681C0F00081072B92
:1044900000F01E81082B40F0148427E1192B00F056
:1044A00043810BD80B2B00F02F81C0F028810C2BFF
:1044B00000F02F810E2B40F004842FE11C2B00F024
:1044C0004E8103D81A2B40F0FC833AE11D2B00F0FB
:1044D00053811E2B40F0F58351E18F2B00F0A48116
:1044E0001ED8872B00F080810BD8842B00F05D81D3
:1044F000C0F05681852B00F05D81862B40F0E18372
:1045000065E18C2B00F0818103D8882B40F0D983A2
:104510006EE18D2B00F07E818E2B40F0D2837EE108
:104520009E2B00F0B1810ED8952B00F08E8103D820
:10453000922B40F0C6837BE19A2B00F09B819B2B52
:1045400040F0BF839BE1A02B00F0B681C0F09F81BB
:10455000A12B00F0BC81A22B40F0B383DAE1EA2B5F
:1045600000F0B2823ED8AD2B00F06C821BD8A82B95
:1045700000F050820BD8A52B00F01482C0F0FD8112
:10458000A62B00F01D82A72B40F09B832DE2AA2BC7
:1045900000F04982C0F04282AB2B00F04982AC2B84
:1045A00040F08F8349E2E12B00F071820BD8AF2BF2
:1045B00000F05382C0F04B82B02B00F05482B12B3C
:1045C00040F07F8355E2E72B00F06C8203D8E62BA6
:1045D00040F0778360E2E82B00F06A82E92B40F03C
:1045E00070836BE2F42B00F0E1821BD8EF2B00F01C
:1045F0008F820BD8EC2B00F07282C0F06A82ED2B18
:1046000000F07382EE2B40F05C8374E2F12B00F03B
:10461000A382C0F08A82F22B00F0AC82F32B40F030
:104620005083B5E2FA2B00F009830ED8F72B00F087
:10463000DB8203D8F52B40F04483C4E2F82B00F072
:10464000E182F92B40F03D83EAE2FD2B00F0148378
:1046500003D8FB2B40F03583FDE2FE2B00F01A83DC
:10466000FF2B40F02E8326E31C4B586802F084FF9A
:104670002EE31A4B586803F055FE29E3174B586890
:1046800003F018F824E35268154B1A6020E3154B29
:104690001B68012B0BD1114B5B68B3F5616F02DC1A
:1046A0000F4A536014E3104B04221A7010E30E4BB0
:1046B00008221A700CE30B4B1B68012B04D1074B2B
:1046C0005A68074B9A6003E3074B08221A70FFE20F
:1046D000024B5A68024BDA60FAE200BFD0080020B1
:1046E0004C0000200000002044090020854B5A683F
:1046F000854B1A61ECE25268834B9A61E8E2814B88
:104700005A68814B5A61E3E27E4B5A687E4BDA610C
:10471000DEE27C4B5A687C4B1A62D9E2794B5A68CC
:10472000794BC3F8DC20D3E2784B1B68012B04D112
:104730005268754BC3F8D420CAE2754B08221A7030
:10474000C6E2724B1B68012B05D16E4B5A686E4B4B
:10475000C3F8D020BCE26E4B08221A70B8E26B4B53
:104760001B68012B04D1674B586809F0FBFCAFE2D2
:10477000674B08221A70ABE203F0C8F8A8E2634B5B
:104780001B68012B04D15F4B586809F053FC9FE272
:104790005F4B08221A709BE252685B4B5A6297E2A9
:1047A000584B5A68584B9A6292E2564B5A68564B8D
:1047B000DA628DE2554B1B68012B04D1514B5A68CC
:1047C000514B5A6384E2524B08221A7080E24F4BDD
:1047D0001B68012B04D14B4B5A684B4B9A6377E211
:1047E0004B4B08221A7073E25268474B1A636FE210
:1047F000464B1B68012B04D1424B5A68424BDA638B
:1048000066E2434B08221A7062E23E4B5A683E4B06
:104810001A645DE23B4B5A683B4B5A6458E2394B91
:104820005A68394B9A6453E25268374BDA644FE264
:10483000344B5A68012A04D81A79334B83F8502034
:1048400046E2334B04221A7042E2304B1B68012BC4
:104850000CD12C4B5A68022A04D81A792A4B83F8B7
:10486000562035E22A4B04221A7031E2284B0822E6
:104870001A702DE2234B586802F052FE28E2214BB9
:10488000586802F063FE23E203F04CF820E21F4B6D
:104890001B68012B0CD11B4B5A68062A04D81A79C5
:1048A000194B83F8512013E2194B04221A700FE2BE
:1048B000174B08221A700BE2144B1B68012B02D114
:1048C00002F088FF04E2124B08221A7000E20F4B3C
:1048D0001B68012B11D10B4A0B4B526832B193F874
:1048E000CD2042F0010283F8CD20F1E193F8CD20F4
:1048F00022F0010283F8CD20EAE1054B08221A706C
:10490000E6E100BFD00800204C000020000000209D
:10491000440900208A4B1B68012B11D1894A8A4B1C
:10492000526832B193F8CD2042F0020283F8CD20D4
:10493000CEE193F8CD2022F0020283F8CD20C7E12A
:10494000824B08221A70C3E17D4B1B68012B10D1EA
:1049500052687D4B32B193F8CD2042F0040283F8C7
:10496000CD20B5E193F8CD2022F0040283F8CD20CC
:10497000AEE1764B08221A70AAE1714B1B68012B3D
:104980000CD1704B5A68032A04D81A796E4B83F8FD
:1049900052209DE16D4B04221A7099E16B4B082265
:1049A0001A7095E1664B1B68012B05D1654B5A685F
:1049B000654BC3F898208BE1644B08221A7087E19D
:1049C0005F4B1B68012B0CD15E4B5A68032A04D83D
:1049D0001A795D4B83F853207AE15C4B04221A70FC
:1049E00076E15A4B08221A7072E1554B1B68012B75
:1049F0000CD1544B5A68022A04D81A79524B83F8C6
:104A0000692065E1514B04221A7061E14F4B082285
:104A10001A705DE152684C4BDA6659E1494B5A68AD
:104A2000494B1A6754E1474B5A68474B5A674FE165
:104A3000444B5A68444B9A674AE1424B5A68424B8E
:104A4000DA6745E15268404BC3F8802040E13D4BB6
:104A50005A683D4BC3F884203AE13A4B5A683A4BC6
:104A6000C3F8882034E1374B5A68374BC3F88C20A1
:104A70002EE1334B1B68012B05D1324B5A68324B68
:104A8000C3F8902024E1314B08221A7020E15268CB
:104A90002D4B83F8CC201BE12A4B5A682A4BC3F8D4
:104AA000A82015E1274B5A68274BC3F8AC200FE12B
:104AB000244B5A68244BC3F8B02009E1214B5A68B3
:104AC000214BC3F8B42003E152681F4BC3F8B82050
:104AD000FEE01C4B5A681C4BC3F8BC20F8E0194B95
:104AE0005A68194BC3F8C020F2E0164B5A68164BAF
:104AF000C3F8C420ECE0124B1B68012B04D1114B0E
:104B00005A68114B1A66E3E0104B08221A70DFE076
:104B10000B4B1B68012B04D152680B4BC3F8A02030
:104B2000D6E00A4B08221A70D2E0054B1B68012B15
:104B30000ED1044B5A68044BC3F8A420C8E000BF50
:104B400000000020D00800204C0000204409002074
:104B5000604B08221A70BBE05F4B1B68012B05D12C
:104B60005E4A5F4B9288A3F85820B1E0594B082267
:104B70001A70ADE0584B1B68012B05D1574A584BB2
:104B80009288A3F85C20A3E0524B08221A709FE0A1
:104B9000514B1B68012B05D1504A514B9288A3F809
:104BA0005A2095E04B4B08221A7091E04A4B1B6843
:104BB000012B04D14A4B9288A3F85E2088E0454B34
:104BC00008221A7084E0444B1B68012B08D1434B28
:104BD0005A68434B003A18BF012283F8672077E0F8
:104BE0003C4B08221A7073E03B4B1B68012B05D12C
:104BF0003A4B5A683A4BC3F8C82069E0354B082253
:104C00001A7065E0344B354A5968526835488A4213
:104C1000026002D101221A605AE000221A6057E0B5
:104C20002D4B1B68012B05D12C4B5A682C4B83F85C
:104C300066204DE0274B08221A7049E0264B1B687E
:104C4000012B04D15268264BC3F8942040E0214B3D
:104C500008221A703CE0204B1B68012B08D11F4B27
:104C60005A681F4B003A18BF012283F868202FE0D2
:104C7000184B08221A702BE0174B1B68012B05D12B
:104C8000164B5A68164B83F8552021E0114B082229
:104C90001A701DE0104B1B68012B08D10F4B5A688E
:104CA0000F4B003A18BF012283F8542010E0094B43
:104CB00008221A700CE0094A094B9288A3F8642074
:104CC00006E0044B03221A7002E0024B04221A7021
:104CD00008BD00BF4409002000000020D0080020CB
:104CE0004C0000206802002008B5A14B9A78002AE9
:104CF00040F0ED815A78A72A00F0318163D8842AE8
:104D000000F0FC8033D80B2A00F0DA8012D8072A92
:104D100000F0CA8008D8052A00F0C08000F2C180E7
:104D2000042A40F0D281B6E0092A00F0C38000F2E4
:104D3000C480BCE01A2A00F0D18009D80E2A00F005
:104D4000C580192A00F0C6800C2A40F0BE81BAE066
:104D50001E2A00F0CA8003D81C2A40F0B681C1E0A8
:104D6000822A00F0C580832A40F0AF81C3E08F2AF9
:104D700000F0DC8012D8882A00F0CC8005D8862A82
:104D800000F0C28000F2C380BBE08D2A00F0C88032
:104D900000F2C9808C2A40F09881BEE0A32A0CD88A
:104DA000A12A80F0CF80952A00F0C6809F2A00F0CB
:104DB000C680922A40F08981BBE0A52A00F0C98014
:104DC00000F2CA80C2E0EB2A00F041812CD8AF2A61
:104DD00000F021810FD8AB2A00F0118105D8A92A53
:104DE00000F0C38000F20881BCE0AD2A00F00D8124
:104DF00000F20E8106E1E62A00F01A8108D8B12AF5
:104E000000F00F81C0F00A81E12A40F05E810BE1E1
:104E1000E82A00F01381C0F00E81E92A00F0118128
:104E2000EA2A40F052810FE1F42A00F02D8115D8D2
:104E3000EF2A00F01A8105D8ED2A00F00F8100F268
:104E4000118107E1F12A00F01681C0F01181F22AE8
:104E500000F01481F32A40F0388112E1FA2A00F0C0
:104E6000208109D8F72A00F01581F92A00F016816F
:104E7000F52A40F02A810AE1FD2A00F0198103D8C1
:104E8000FB2A40F0228110E1FE2A00F01481FF2A63
:104E900040F01B8113E14020364913E1442036499C
:104EA00001E148203549FEE04C203549FBE0502027
:104EB0003449F8E058203449F5E054203349F2E011
:104EC0005C203349EFE060203249ECE04FF48E7013
:104ED0003149E8E04FF48A703049E4E04FF48870DB
:104EE0002F49E0E009F044F9F4E009F0A9F8F1E015
:104EF00064202C49D7E068202B49D4E06C202B4952
:104F0000D1E074202A49CEE078202A49CBE07020F5
:104F10002949C8E07C202949C5E080202849C2E011
:104F200084202849BFE088202749BCE08C202749FD
:104F3000B9E090202649C0E096202649BDE09120A6
:104F40002549BAE040F20D102449B6E092202449E8
:104F5000B3E0D8202349A6E093202349ADE0A9205F
:104F60002249AAE0AC2022499DE0B02021499AE0E4
:104F7000D00800204C0000205000002054000020E9
:104F8000580000205C000020640000206000002029
:104F9000680000206C000020280100202001002073
:104FA0001C01002070000020740000207800002008
:104FB00080000020840000207C0000208800002069
:104FC0008C00002090000020940000209800002019
:104FD0009C000020A20000209D000020190100205C
:104FE0009E000020E40000209F000020B50000206B
:104FF000B8000020BC000020B420374953E0B8209E
:10500000364950E0BC2036494DE0C02035494AE0E1
:10501000C420354947E0C820344944E0CC20344915
:1050200041E0D02033493EE04FF48670324944E0FD
:10503000E820324937E0EC20314934E0F0203149B2
:1050400031E0F42030492EE0F82030492BE0FC20FC
:105050002F4928E04FF480702E4924E04FF48270ED
:105060002D4920E0A0202D491DE0E0202C491AE028
:10507000E4202C4917E098202B4922E09C202B4962
:105080001FE09A202A491CE09E202A4919E0A72007
:10509000294912E04FF48470284904E0A6202849E9
:1050A0000BE02849D42004220CE0A820264904E083
:1050B0009520264901E026499420012202E0254955
:1050C000A42002220AF07AF904E0032200E004227C
:1050D000214B1A7008BD00BFC0000020C400002092
:1050E000C8000020CC000020D0000020D400002008
:1050F000D8000020DC00002018010020F40000206F
:10510000F8000020FC000020000100200401002025
:10511000080100200C01002010010020AC0000203C
:10512000EC000020F0000020A4000020A8000020D7
:10513000A6000020AA000020B300002014010020D7
:10514000B2000020E0000020B4000020A1000020F8
:10515000A0000020B00000204409002008B5A34BA7
:105160009A78002A40F059825A78A82A00F0A7813C
:1051700063D8852A00F013812DD80B2A00F0EA802D
:1051800012D8072A00F0D08008D8052A00F0BC8089
:1051900000F2C280042A40F03E82B2E0092A00F008
:1051A000CE8000F2CF80C7E01A2A00F0E68009D84E
:1051B0000E2A00F0D580192A00F0D6800C2A40F083
:1051C0002A82CAE0832A00F0E48000F2E580822A85
:1051D00040F02182DAE0922A00F03A8115D88C2A38
:1051E00000F0F88008D8872A00F0E980C0F0DF805E
:1051F000882A40F01082E5E08E2A00F0F180C0F0AD
:10520000EC808F2A40F00782EDE0A32A09D8A12A7A
:1052100080F02C81952A00F01E819F2A40F0FB81AE
:105220001CE1A52A00F03381C0F02981A62A00F0F4
:105230003681A72A40F0EF8139E1EC2A00F079812C
:105240002DD8B02A00F053810FD8AC2A00F043814A
:1052500005D8AA2A00F0398100F23A8132E1AE2A5B
:1052600000F03F8100F2408138E1E72A00F05281EE
:1052700009D8E12A00F04681E62A00F04881B12AE7
:1052800040F0C98136E1E92A00F04A81C0F0458149
:10529000EA2A00F04881EB2A40F0BD8146E1F42A79
:1052A00000F0778110D8F02A00F0598105D8EE2A55
:1052B00000F0478100F24C813FE1F22A00F05C816E
:1052C0004B4B00F2608151E1FA2A00F07F8109D84E
:1052D000F72A00F06C81F92A00F07181F52A40F07C
:1052E0009A815DE1FD2A00F0808103D8FB2A40F01D
:1052F000928173E1FE2A00F07F81FF2A40F08B81CA
:1053000083E140203B4983E1394B1B68012B40F08E
:105310007A81442038495FE1354B1B68012B40F00E
:1053200072814820354957E1314B1B68012B40F011
:105330006A814C2032494FE1502032494CE15820DB
:10534000314949E12A4B1B68012B40F05C81542014
:105350002E4941E15C202E493EE160202D493BE190
:105360004FF48E702C4937E1214B1B68012B40F024
:105370004A814FF48A7029492EE11D4B1B68012B8D
:1053800040F041814FF48870254925E1642025498A
:1053900022E1682024491FE16C2024491CE1144BC0
:1053A0001B68012B40F02F817420214914E1104B20
:1053B0001B68012B40F0278178201E490CE17020EA
:1053C0001D4909E10A4B1B68012B40F01C817C2020
:1053D0001A4901E180201A49FEE084201949FBE0C6
:1053E00088201949F8E08C201849F5E0D008002001
:1053F000000000204C00002050000020540000203D
:10540000580000205C0000206400002060000020A4
:10541000680000206C0000202801002020010020EE
:105420001C01002070000020740000207800002083
:1054300080000020840000207C00002088000020E4
:105440008C00002090000020940000209800002094
:105450009020744959E09620734956E0734B1A68BE
:10546000012A40F0D08091207149D1E06F4B1B6838
:10547000012B40F0C88040F20D106E4945E06B4BA7
:105480001A68012A40F0BF8092206B49C0E0674B48
:105490001B68012B40F0B780D82068499CE0634B23
:1054A0001A68012A40F0AF8093206549B0E05F4B55
:1054B0001A68012A40F0A780A9206249A8E0AC2020
:1054C000614989E0B020614986E0B420604983E009
:1054D000B820604980E0BC205F497DE0C0205F4982
:1054E0007AE0C4205E4977E0C8205E4974E0CC20B1
:1054F0005D4971E04D4B1B68012B40F08480D0204A
:105500005A4969E05A494FF48670012280E0E82048
:10551000584961E0EC2058495EE0F02057495BE0D3
:10552000F420574958E0F820564955E0FC205649E8
:1055300052E04FF4807055494EE04FF48270544968
:105540004AE03A4B1B68012B5DD1A020514943E052
:10555000364B1B68012B56D1E0204F493CE0334BC2
:105560001B68012B4FD1E4204C4935E01B68012B0F
:1055700049D198204A494AE02C4B1B68012B42D163
:105580009C20484943E01B68012B3CD19A204649A6
:105590003DE0264B1B68012B35D19E20434936E068
:1055A000224B1A68012A2ED1A720414930E01F4B17
:1055B0001B68012B27D14FF484703E490CE01B4B34
:1055C0001A68012A1FD1A6203B4921E0174B1B680E
:1055D000012B18D13949D420042219E0134B1A6841
:1055E000012A10D1A820364912E0104B1A68012A6E
:1055F00009D1952033490BE00C4B1A68012A02D1DE
:105600009420314904E0082208E03049A420022215
:1056100009F0B0FE04E0032200E004222C4B1A70D3
:1056200008BD00BF9C000020A20000200000002058
:105630009D000020190100209E000020E4000020B1
:105640009F000020B5000020B8000020BC00002012
:10565000C0000020C4000020C8000020CC000020B2
:10566000D0000020D4000020D8000020DC00002062
:1056700018010020F4000020F8000020FC000020A9
:105680000001002004010020080100200C0100207E
:1056900010010020AC000020EC000020F0000020F1
:1056A000A4000020A8000020A6000020AA000020DE
:1056B000B300002014010020B2000020E000002010
:1056C000B4000020A1000020A0000020B0000020B5
:1056D000440900201C4900230B601C491C4A0B6034
:1056E0001C4910B50B60137253601B4A002199507E
:1056F0000433B3F5806FF8D1184B1B68012B0CD025
:1057000040F21A74164920460919042209F032FEA3
:10571000043440F25A739C42F4D1124B1B7E63B99D
:1057200040F21A740E4920460919042209F022FE9B
:10573000043440F2FA739C42F4D10A4A044B527D7D
:1057400002B101225A7210BD300900204C0900201C
:1057500068020020D8080020D004002000000020AB
:10576000B6FDFF1F0800002010B57C4B987818B1DB
:10577000022840F0EE80DAE05A784C2A00F0878068
:105780001ED8442A55D00CD8412A3FD003D8402AED
:1057900040F0DD8036E0422A3FD0432A40F0D780F7
:1057A00041E0472A57D005D8452A48D0462A40F03C
:1057B000CE804AE0492A54D04B2A40F0C8805BE0B2
:1057C000532A00F08E800CD8502A6CD003D84D2A72
:1057D00040F0BD8061E0512A6BD0522A40F0B78082
:1057E00079E0832A00F0968005D8552A7FD05A2A7E
:1057F00040F0AD8085E0842A00F09180FF2A40F0DF
:10580000A68091E0197940F2FF7003E01B79544AB9
:105810001946137009F068FE9EE01B79504A19463C
:1058200001205370F6E71B794D4A19460420137185
:10583000F0E75B684A491C2041F81C3F66E01B7991
:10584000474A194605205371E4E75B6844490C2038
:1058500041F80C3F5AE05B684149082041F8083F95
:1058600054E01A793E4B12B13E4901224A60DA7582
:105870003B4B1720D97DCDE71B79394C03201946C6
:10588000E37009F031FEE07808F0B6F964E01B79C6
:10589000334A194602209370BCE71B79304A1946F7
:1058A00015205375B6E71B792D4A194616209375B6
:1058B000B0E72B4A127D12F0010F05D01B7913F0CF
:1058C000010F01D109F0C8FE244B254A1B79142091
:1058D000194613759EE75B682149202041F8203F57
:1058E00014E05B681E49102041F8103F0EE05A6832
:1058F000012A2ED81B791A49182001F8183F0122D5
:1059000005E05B681649242041F8243F042209F091
:1059100055FD21E0134B5A68134BDA601CE0114B24
:105920005A68124B1A6017E01A79114B13E05A7833
:105930000F2A05D80F490968012903D0082209E078
:10594000372A04D859680C4B43F8221004E003228C
:1059500000E00422034B1A7010BD00BFD0080020E5
:1059600008000020440900206802002040090020AF
:105970003D09002000000020D00400202DE9FF4157
:105980007D4C7E4D237862686421212B29706B70D9
:105990006A6000F0A8875DD80E2B00F054852BD8E4
:1059A000062B00F0EF8011D8032B00F0C08006D842
:1059B000012B00F0B080022B41F00282B0E0042BFA
:1059C00000F0BA80052B41F0FB81D1E0092B00F0FB
:1059D000188407D8072B00F00C84082B41F0F081C5
:1059E00000F00BBC0B2B00F0E084C0F00E840C2BFD
:1059F00041F0E68100F0F5BC172B00F0B88613D813
:105A0000142B00F0E38507D80F2B00F04085132BF3
:105A100041F0D68100F08ABD152B00F0FE85162BD3
:105A200041F0CE8100F09EBE1C2B00F00A8707D803
:105A3000182B00F0A9861B2B41F0C28100F0B0BEEC
:105A40001F2B00F0158700F23A871E2B41F0B8811A
:105A500000F0FBBE802B01F012802DD8412B00F00E
:105A6000F98713D8242B00F0B18707D8222B00F038
:105A7000A087232B41F0A48100F0A1BF272B00F0C9
:105A8000D287402B41F09C8100F0E1BF442B00F015
:105A9000EA8707D8422B00F0E087432B41F0908142
:105AA00000F0DEBF462B00F0E487C0F0DF87472B15
:105AB00041F0868100F0E0BF872B01F0728013D89F
:105AC000832B00F0F08707D8812B00F0DC87822B36
:105AD00041F0768100F0E3BF852B01F00080284B78
:105AE00001F2018000F0ECBF8C2B01F0BD8007D8E3
:105AF000882B01F03580892B41F0628101F094B848
:105B0000F22B01F01F81FF2B01F04F818D2B41F013
:105B1000578101F0CEB8104601F0CCFD01F053B929
:105B2000154B5868404201F0C5FD01F04CB900200A
:105B300001F0C0FD01F047B9A378A3B90E4B5A7824
:105B400012B1012A0AD104E0586801F015FD01F0F4
:105B50003AB9586801F044FD01F035B9074B03220A
:105B60001A7001F030B9054B04221A7001F02BB9FC
:105B7000FEF766FC01F027B9D00800204409002098
:105B800008000020A378002B40F01A836378FF2BD5
:105B900000F21383DFE813F00001040108010C0197
:105BA0001001140118011C012001240128012C01FD
:105BB00030013401380111031103110311031103E2
:105BC0003D01590176017B011103800185018A01A4
:105BD0008E0111039201110311031103110311032B
:105BE0001103110311031103110311031103110315
:105BF0001103110311031103110311031103110305
:105C000011031103110311031103110311031103F4
:105C100011031103110311031103110311031103E4
:105C200011031103110311031103110311031103D4
:105C300011031103110311031103110311031103C4
:105C400011031103110311031103110311031103B4
:105C500011031103110311031103110311031103A4
:105C60001103110311031103110311031103110394
:105C70001103110311031103110311031103110384
:105C80001103110311031103110311031103110374
:105C900011031103110311031103110396019A015A
:105CA0009E01A201A601AA01AE0111031103110375
:105CB000B201B601BA01BE0111031103C201110301
:105CC0001103CA01CF01D301D801DD01E101E501D2
:105CD000E90111031103ED01F201F601FD010402D6
:105CE0000B02100215021A021F02230227023002C1
:105CF000340238023D02420247024C0211031103F2
:105D000011031103110311031103110311031103F3
:105D1000110311035102550259025D02610265022D
:105D200069026D021103110371027502110311035F
:105D3000110311031103110311037902110311035C
:105D400011031103110311031103110311031103B3
:105D5000110311031103110311037D028202860254
:105D60008A028E02920297029C02A102A602AB0254
:105D7000B002B502BA02BE02C302C802CD02D2020C
:105D8000D702DC021103E402E902ED02F202F7029B
:105D90001103FF0204030C0301F00CFB686011E225
:105DA00001F01CFB68600DE201F01EFB686009E277
:105DB00001F020FB686005E28D4B1B686B6001E21F
:105DC0008B4B5B686B60FDE1894B9B686B60F9E115
:105DD000874BDB686B60F5E1854B1B696B60F1E11C
:105DE000834B9B696B60EDE1814B5B696B60E9E123
:105DF0007F4BDB696B60E5E17D4B1B6A6B60E1E12A
:105E000001F0E4FA6860DDE1794BD3F8DC306B60D7
:105E1000D8E1774B93F8530010F0010002D109F05C
:105E200095FA50B1724B93F8533013F0010F08D02C
:105E3000002009F08BFA012803D16E4B01225A6031
:105E4000C0E16C4B00225A60BCE1694B93F85330BF
:105E500013F0020F03D1012009F078FA50B1644B1E
:105E600093F8533013F0020F08D0012009F06EFAB6
:105E7000012803D15F4B01225A60A3E15D4B002250
:105E80005A609FE1002008F011F868609AE1012053
:105E900008F00CF8686095E1554BD3F8D4306B608E
:105EA00090E1534BD3F8D0306B608BE108F04EF9A2
:105EB000686087E108F050F9686083E108F0B4F8A1
:105EC00068607FE14A4B5B6A6B607BE1484B9B6A91
:105ED0006B6077E1464BDB6A6B6073E1444B5B6B55
:105EE0006B606FE1424B9B6B6B606BE1404B1B6BDC
:105EF0006B6067E13E4BDB6B6B6063E13C4B1B6CA3
:105F00006B605FE13A4B5B6C6B605BE1384B9B6CA9
:105F10006B6057E1364BDB6C6B6053E1344B93F8AD
:105F20005030003B18BF01236B604BE1304B93F8BE
:105F300056306B6046E101F063FA686042E103208D
:105F400009F030F868603DE1042009F02BF8686042
:105F500038E101F05BFA686034E101F031FA686021
:105F600030E101F021FA68602CE101F08FFB6860FC
:105F700028E11F4B93F851306B6023E101F03CFCAA
:105F800068601FE11A4B93F8CD3003F001036B609A
:105F900018E1174B93F8CD30C3F340036B6011E168
:105FA000134B93F8CD30C3F380036B600AE1104BC1
:105FB00093F852306B6005E10D4BD3F898306B606D
:105FC00000E10B4B93F853306B60FBE0084B93F808
:105FD00069306B60F6E0064BDB6E6B60F2E0044B01
:105FE0001B6F6B60EEE0024B5B6F6B60EAE000BF23
:105FF0004C00002044090020934B9B6F6B60E1E054
:10600000914BDB6F6B60DDE08F4BD3F880306B60C2
:10601000D8E08D4BD3F884306B60D3E08A4BD3F853
:1060200088306B60CEE0884BD3F88C306B60C9E071
:10603000854BD3F890306B60C4E009F0E1FB6860F9
:10604000C0E009F0E3FB6860BCE009F0E5FB6860D4
:10605000B8E009F0E7FB6860B4E009F0E9FB6860CC
:10606000B0E009F0EBFB6860ACE009F0EDFB6860C4
:10607000A8E009F0EFFB6860A4E001F089FB68602C
:10608000A0E001F08BFB68609CE001F063FB6860BE
:1060900098E06D4B93F8CC306B6093E001F060FBBF
:1060A00068608FE001F062FB68608BE001F064FBE8
:1060B000686087E001F066FB686083E0624BD3F8BC
:1060C000A8306B607EE0604BD3F8AC306B6079E059
:1060D0005D4BD3F8B0306B6074E05B4BD3F8B430F9
:1060E0006B606FE0584BD3F8B8306B606AE0564B8A
:1060F000D3F8BC306B6065E0534BD3F8C0306B60B5
:1061000060E0514BD3F8C4306B605BE04E4B1B6ECC
:106110006B6057E04C4BD3F8A0306B6052E04A4BB9
:10612000D3F8A4306B604DE0474BB3F958306B6047
:1061300048E0454BB3F95C306B6043E0424BB3F948
:106140005A306B603EE0404BB3F95E306B6039E033
:106150003D4B93F86730003B18BF01236B6031E083
:10616000394BD3F8C8306B602CE0384B1B686B6040
:1061700028E0354B93F866306B6023E0324BD3F860
:1061800094306B601EE0304B93F86830003B18BFD2
:1061900001236B6016E02C4B93F855306B6011E0D7
:1061A000294B93F85430003B18BF01236B6009E082
:1061B000254BB3F864306B6004E003232B7001E0DF
:1061C00004232B70224B1B78002B00F0FC85214B05
:1061D00021495A68214B0A602AB91A6842F008021C
:1061E0001A6000F0F0BD1A6822F008021A6000F090
:1061F000EABDFEF779FD00F0E6BDFEF7AFFF00F067
:10620000E2BDFFF7B1FA00F0DEBD154B9A7822B17E
:10621000022A104D40F0B080A8E05B78512B76D078
:106220002FD8452B5FD01DD8422B51D005D8402BFD
:1062300045D0412B40F0968048E0432B4DD0442B75
:1062400040F090804CE000BF4C000020680200202D
:106250003E0900204409002030090020D808002011
:10626000D0080020492B46D004D8462B3ED0472BDF
:1062700078D13DE04D2B44D0502B45D04C2B71D1E3
:106280003CE0812B55D00CD8552B49D004D8522B4B
:1062900040D0532B66D140E05A2B44D0802B61D1A3
:1062A00044E0842B52D004D8822B49D0832B59D17F
:1062B00049E0FE2B4DD04FD8F02B53D149E040F2AE
:1062C000FF7009F0F9F88A4B586057E0894B41E0BC
:1062D000884B5A78864B5A6050E0864B1A79F9E71A
:1062E000844BDA69F6E7834B5A79F3E7814B2BE06D
:1062F000804B9A68EEE77F4BDA7D2FE07D4B9A78F2
:10630000E8E77C4B5A7DE5E77A4B9A7DE2E7794BEB
:106310001A7DDFE7774B1A6ADCE7764B1A69D9E713
:10632000744B1A7ED6E7734B5A6AD3E7724B5A7A8C
:10633000D0E7714B5A7A042A14BF00220122C9E720
:106340006D4B5A68C6E76C4BDA68C3E76B4B1A684B
:10635000C0E76B4B1A78BDE76A4B1A78003A18BF52
:106360000122B7E7624B03221A7007E05A78664BA6
:1063700053F822306B6001E004232B70634B1B78D1
:10638000002B00F020855A4B61495A68614B0A6026
:106390002AB91A6842F008021A6000F014BD1A689F
:1063A00022F008021A6000F00EBDA378022B13D170
:1063B000594B5B78372B0AD89B00534903F5E260B1
:1063C000C9180A30042208F0F9FF00F0FCBC484B61
:1063D00003221A7000F0F7BC454B04221A7000F03B
:1063E000F2BC4D4B9A78022A28D159780F2913D83C
:1063F0004A4B1B68012B0AD18900434B01F5E2602F
:106400000A305918023208F0B5FF00F0DCBC384BF6
:1064100008221A7000F0D7BC37290AD889003A4BF5
:1064200001F5E2600A305918042208F0A3FF00F0D9
:10643000CABC2F4B03221A7000F0C5BC2C4B04229F
:106440001A7000F0C0BCA378012B02D0022B1AD125
:106450000FE0607848B922B9104608F063FF00F0F9
:10646000B2BC08F057FF00F0AEBC03232B7000F065
:10647000AABC60781AB908F071FF00F0A4BC08F05B
:1064800069FF00F0A0BC04232B7000F09CBCA37833
:10649000012B0BD01BB1022B154D16D10FE01E4B5B
:1064A000587808F053FF124B586010E01A4B104D0B
:1064B000587810B907F0FAFC05E0032306E0164B04
:1064C000587808F03FFF686001E004232B700F4B01
:1064D0001B78002B00F07784054B0D495A680D4B53
:1064E0000A60EAB91A6842F008021A6000F06BBC50
:1064F0004409002008000020680200204009002014
:10650000680900203D090020D00400203E09002039
:1065100030090020D8080020D0080020000000200A
:106520001A6822F008021A6000F04DBC894A8A4BB2
:106530005278092A3BD8DFE802F0050A0F141A2224
:10654000282E343783491A6849688A182EE0814A10
:10655000196852688A1A29E07E4A196852684A43C3
:1065600024E07C4A1968526891FBF2F21EE0794AF5
:106570001968526891FBF2F002FB101216E075499F
:106580001A68496801EA020210E072491A6849680B
:1065900041EA02020AE06F491A68496881EA020288
:1065A00004E01A68D24301E06A4A52681A606A4AF3
:1065B0006A4B12682AB91A6842F008021A6000F0A1
:1065C00002BC1A6822F008021A60FCE3624B1B68E6
:1065D000934206DD614B1A6842F0040222F0030286
:1065E0000CE05E4B05D11A6822F0060242F001026F
:1065F00004E01A6822F0070242F002021A60564ACA
:10660000564B126822B91A6842F008021A60DAE39F
:106610001A6822F008021A60D5E363780C2B00F2A6
:10662000D283DFE803F007121D28333E49545F6A26
:1066300075808B00494B1B6813F0080F00F0C38373
:10664000444B5A68464B5A60BDE3444B1B6813F0F9
:10665000080F40F0B8833F4B5A68414B5A60B2E391
:106660003E4B1B6813F0010F00F0AD83394B5A68A5
:106670003B4B5A60A7E3394B1B6813F0010F40F006
:10668000A283344B5A68364B5A609CE3334B1B68E9
:1066900013F0040F00F097832E4B5A68304B5A606A
:1066A00091E32E4B1B6813F0050F00F08C83294BF0
:1066B0005A682B4B5A6086E3284B1B6813F0020F75
:1066C00000F08183234B5A68254B5A607BE3234BB0
:1066D0001B6813F0030F00F076831E4B5A68204BA3
:1066E0005A6070E31D4B1B6813F0100F00F06B83B2
:1066F000184B5A681A4B5A6065E3184B1B6813F025
:10670000200F00F06083134B5A68154B5A605AE310
:10671000124B1B6813F0400F00F055830D4B5A6865
:106720000F4B5A604FE30D4B1B6813F0800F00F0C6
:106730004A83084B5A680A4B5A6044E3074B1B686C
:1067400013F4807F00F03F83024B5A68044B5A6079
:1067500039E300BFD008002030090020D80800200D
:1067600068020020814B5A68814B5A602BE3804BB2
:106770001969072900F227835C68481C03EB810133
:106780004C615A6018611EE3794B1A69002A00F0C7
:106790001A83013A03EB820149691A61596012E3D5
:1067A000734B1A7A7AB9714A5268B2F1FF3F04BF4B
:1067B000704A12680A214A435A6307F02FFD6C4B56
:1067C00001221A729863694B5C781CB1012C40F06D
:1067D000FA8210E007F022FD654B996B5A6B411A63
:1067E0000029B8BF4942914201D91C72EBE25A68B4
:1067F000013A5A60E7E200F049FF10F480455C4C32
:1068000007D05D4B00211A68217222F010021A6035
:10681000D9E2636B83B107F001FDA26B636B821A4F
:10682000002AB8BF52429A4206D9534B25721A68C1
:1068300042F010021A60C6E24D4B5A68013A5A60A3
:10684000C1E24B4B00225A72BDE2484B9A785AB9CA
:106850005A78142A04D85968484B43F82210B2E2F7
:10686000474B03221A70AEE2454B04221A70AAE28B
:10687000A37863B93D4B424D5B78142B04D83F4A53
:1068800052F823306B6005E003232B7002E03C4B91
:1068900004221A703B4B1B78002B00F09482384B7B
:1068A00034495A68344B0A6022B91A6842F0080227
:1068B0001A6088E21A6822F008021A6083E22B4B01
:1068C0009A7862B95C78142C05D800F087FD2B4BC0
:1068D00043F8240077E22A4B03221A7073E2284B14
:1068E00004221A706FE26278224B0A2A53D8DFE83A
:1068F00002F0060B11161C242A30363A4D002249AC
:106900001A6809688A1803E01F4A196812688A1A07
:106910001A6040E01C4A196812684A43F8E71A4AAC
:106920001968126891FBF2F2F2E7174A19681268C7
:1069300091FBF2F002FB1012EAE713491A680968AA
:1069400001EA0202E4E710491A68096841EA020212
:10695000DEE70D491A68096881EA0202D8E70A4BA6
:106960001A68D243D4E71A68074BD1E7D008002051
:106970006802002030090020D8080020DC08002030
:10698000440900203E0900204C090020894A18686B
:10699000116810601960884A884B126822B91A6819
:1069A00042F008021A600EE21A6822F008021A6029
:1069B00009E2814B1B686360FDF742FD03E27E4BF9
:1069C0001A687F4B5A60FEF7CFFEFCE16378052B17
:1069D00000F2F981DFE803F003090F151B21774B63
:1069E0001A6802F00F021A60EDE1744B1A6822F087
:1069F00010021A60E7E1714B1A6822F020021A6057
:106A0000E1E16E4B1A6822F040021A60DBE16B4B49
:106A10001A6822F080021A60D5E1684B1A6822F4E5
:106A200080721A60CFE1A3786BB9654B5B78142B49
:106A300005D8614A1168634A42F82310C3E1624BEA
:106A400003221A70BFE1604B04221A70BBE108F008
:106A5000C7FEB8E108F0C6FEB5E108F0C5FEB2E138
:106A600008F0C4FEAFE108F0C3FEACE108F0C2FEDE
:106A7000A9E108F0C1FEA6E108F0C0FEA3E1534B76
:106A800000225A729FE163780121504A8B42517271
:106A900040F099814A4B5A684C4B5A6093E14B4BFA
:106AA00002225A728FE1454900230B604249474A4E
:106AB0000B60404913720B6053725360136182E1A3
:106AC0001B7D13F0020F06D13D4A404B5268DA633A
:106AD00004225A7277E13C4B08221A7073E13B4B57
:106AE00000225A726FE1364A9B785068384C394A16
:106AF0000125B0F5006F1570237027DC364B1E7D25
:106B00002E4023D101A908F025FE9DF804809DF8B0
:106B100005709DF806C09DF80B009DF80A109DF8C1
:106B200009209DF80830267284F80180A77084F847
:106B300003C020716171A271E371254BE95C1A7A7F
:106B400001358A18082D1A72F7D13CE10123204A39
:106B5000002199540133082BF9D11378137232E1D3
:106B6000627892B91C4B01219A781C4B1868194B1A
:106B70001970174B1A7000230133C21812F8011C48
:106B8000134A082B9954F7D11DE1012A40F01B81CB
:106B90000D4B2F2119710221D971593199715A71F7
:106BA00011E16378032B00F20E81DFE803F0192670
:106BB000333800BF4C09002030090020D8080020DD
:106BC000D0080020DC0800204409002068020020D2
:106BD00034090020CC0400200800002060020020BE
:106BE0007A4A7B4BD16B92F809C0107A0A0A197164
:106BF00083F807C098715A71E5E0744A744B516884
:106C000092F809C0107A0A0A197183F807C09871BE
:106C10005A71D8E06F4B1A686D4B5A60D3E06E4BD7
:106C20001A686B4B5A60CEE06C4B1C68012C17D174
:106C30006B4B6C491A6802EA0101002940F0C380DD
:106C40005A6840F2D2439A4240F0BD8040F2FF7051
:106C500008F04AFC08F000FD204608F06BFBB2E0AB
:106C60005B4B08221A70AEE0667816B1012E1DD17A
:106C70000EE0042240F2FB7003A908F07BFB62687F
:106C8000039B9A4202D101236B609CE06E609AE004
:106C9000A3782A2B06D140F2FB705349042208F056
:106CA0008DFB90E04A4B03221A708CE003232B707B
:106CB00089E04B4B5B78032B40D8DFE803F00802F8
:106CC000313B424B196C464B5C68002324E03F4B40
:106CD0001A6C092A07D84248511C406803EB82020B
:106CE000506419646FE03A4B09221A706BE052F855
:106CF0002350581CA5420ED102EB8002013904E05A
:106D000052F8040C013342F8080C04328B42F7D3DA
:106D10002E4B196457E003468B42344AE7D352E0C6
:106D20002A4A00231364314A0021D1500433282B0E
:106D3000F9D148E0264B0A225A6044E0244B032252
:106D40001A7040E02268274B02EA0303284A934264
:106D500039D1234B5A68274B9A4234D1264B4FF4F2
:106D600000525A6103F098F807F058FA044607F009
:106D700055FA001B0028B8BF4042B0F57A7FF6DB19
:106D800008F0C6FA03F01AFE002004F047FB0021C9
:106D90001A4803F0F1FB194803F04EFB184803F0C2
:106DA00021FB002008F0C6FA0DE00D4B5A6840F2B6
:106DB000D2439A4207D1054B012283F86C2002E0AE
:106DC000034B02221A70BDE8FF8100BF6802002059
:106DD00044090020300900204C0900200000002058
:106DE000D008002000FFFF00D4080020AC020020E3
:106DF00000819200D6C5B4A30010014008000240F3
:106E00000024014073B5204B024640781F4D187096
:106E1000907800265870D078EC46987010790C461F
:106E2000D8715079987192F806E095E8030083F8DC
:106E300005E0D2798CE803001A71154B1E70FEF73D
:106E40009DFD144B1B7873B9637023702B78A3706E
:106E50006B78E370EB792371AB7963716B79A37114
:106E60002B79E37108E0012B06D10B4B9B195B7862
:106E7000A3550136082EF8D1044B6A4692E8030068
:106E800083E803007CBD00BFD00800204409002037
:106E90003E090020CC0400203409002073B50C4EBC
:106EA0000C4C73600C4B4FF0000C6D4683F800C027
:106EB00030707170B27094E8030085E80300FEF74B
:106EC0005DFD95E80300636884E8030018467CBD17
:106ED000D0080020440900203E09002070B5994BDD
:106EE00086B01B786BB1984B1B78062B09D00A2B08
:106EF00007D00F2B05D01F2B03D0944B002283F813
:106F00006D20924B93F86D30032B21D1904B1B7861
:106F100093B9904D904CA8786E7822786378861952
:106F2000B618E279F618A379B6186279F6182379BB
:106F3000B618F618F6B21AE0012B40F09280002441
:106F4000864BE05C013406F067FE092CF8D188E03E
:106F5000042B27D17F4D804CAB786E7818469E1954
:106F600001360023012222706360F6B2637006F0DE
:106F700053FE687806F050FE207806F04DFE6078EB
:106F800006F04AFEE07906F047FEA07906F044FEDE
:106F9000607906F041FE207906F03EFE304606F0AC
:106FA0003BFE5EE0072B35D1694B1B782BBB694A52
:106FB000694B5478957893F800E093F801C066190E
:106FC000D8797644997966445A7986191B798E194D
:106FD00096199E198DF808608DF800508DF80140C3
:106FE0008DF802E08DF803C08DF804008DF80510CF
:106FF0008DF806208DF8073009E0012B07D1013B01
:10700000564A995C0DF803100133092BF8D16846F4
:10701000092124E0082B24D14E4A4F4B92F801C09D
:1070200092F802E001240EEB0C05002201356846BF
:1070300009215A608DF802408DF8032016468DF81C
:1070400004208DF805208DF806208DF807208DF896
:1070500008505A701C708DF800E08DF801C002F0E5
:1070600009FE3A4B3A4893F86C100022027083F8FC
:107070006D2011B1012008F05DF90DF1170006F047
:10708000A5FD044600286FD006F0BCFD18B12F4BBB
:10709000002283F86E202D4A9DF8170092F86E109A
:1070A0004B1CDBB28918092B81F8700082F86E3016
:1070B00040F0B980274B92F870005978002388423D
:1070C00082F86E3040F0AF801A46204C04F1700117
:1070D000C95C01335218082BD2B2F6D194F878303B
:1070E00093422CD1184B94F8751094F8762094F8AC
:1070F000775094F8716094F872E094F873C094F843
:1071000074001D7199715A711E7083F801E083F843
:1071100002C0D87107F082F8114D637A2860591EB9
:1071200010480022C9B202700320012984F86D00C2
:1071300084F86E205AD9052B58D0013257E0042329
:1071400058E000BF3D090020D00800206802002060
:10715000CC0400200800002044090020340900204D
:107160006C0900207009002003A802F06DFD0028C2
:1071700043D05D4B9DF80C205B789A4253D1234657
:10718000224603A9C95C01335218082BD2B2F8D1A8
:107190009DF81410554C91422CD1554B9DF811106F
:1071A0009DF812209DF80D609DF80EE09DF80FC02F
:1071B0009DF810009DF8135099715A711E701D7141
:1071C00083F801E083F802C0D87107F027F8494935
:1071D000637A08605A1E48490020D2B2087007211D
:1071E000012A84F86D1001D9052B19D10022434BD7
:1071F0001A7018E084F86D3015E03C4C637A013B5E
:10720000DBB2012B0FD86368B3F5006F0AD81846BC
:1072100001336360364908F09DFA092384F86D3024
:107220000122E4E76072314C637A042B04D1304EC2
:10723000327812F0800F2FD02C4B93F86D303BB189
:10724000042B05D0082B03D0062B01D0FEF796FBAC
:10725000264B93F86D20092A04D1597A022901D1CD
:1072600003315972214B196C00293AD0092A38D1BF
:107270005A7A012A35D15868002307E054F8234090
:107280000133A04202D1052353722AE0174A8B42F0
:1072900002F14404F2D324E094F86D300BB3042BD4
:1072A0001FD0082B1DD0062B1BD0E06B144D73682C
:1072B000B0F5006F6A706B600FD8314608F04CF97A
:1072C0003146E06B08F070F920B1E36B0133E36302
:1072D000652300E007232B7003E007232B700023B6
:1072E000637206B070BD00BF080000206802002075
:1072F000D00800206C090020700900203E09002001
:1073000044090020704700BF234A244B30B5D3F80E
:10731000943014684FEA530C041B6445106001DD7F
:10732000E41A04E0CCF1000C6445B8BFE4181C4D2D
:107330001A4A2D7815B9D2F8C82002E0D2F8C82030
:10734000524208180419A41848BFE418B4FBF3F219
:1073500003FB1244114AA40292F85510104A49083E
:107360001278B3FBF1F3B4FBF3F312B903F58073B6
:1073700001E0A3F58073002B0A48B8BF03F58063D2
:1073800003EA0000002805DA01386FEA80506FEA4E
:107390009050013030BD00BFE40200204C000020BE
:1073A000E4090020FF030080014B1868704700BF0C
:1073B000D4090020014B5868704700BFE402002048
:1073C000014B1868704700BFF009002008B5024B58
:1073D000186808F051FF08BD100A0020014B18681A
:1073E000704700BFD0090020014B1868704700BFEC
:1073F000200A0020014B1868704700BFE8090020F0
:10740000014B1868704700BFF8090020064A074B77
:10741000127822B918680028B8BF404203E0186803
:107420000028C8BF40427047E4090020D809002066
:10743000024B9A6840EA02029A607047E402002018
:1074400008B50A4B93F851300BB1022B0CD1084B05
:107450009A6812F0070F04D09B6803F00703072B0C
:1074600002D12020FFF7E4FF08BD00BF4C00002040
:1074700000080140024B9A6822EA00029A607047B5
:10748000E4020020B0F5007F10B5044610D003DC04
:10749000B0F5807F34D121E0B0F5806F03D0B0F536
:1074A000006F2DD10DE0FFF7C3FF4FF4007003E034
:1074B000FFF7BEFF4FF48060FFF7DCFF4FF4006082
:1074C00007E0FFF7B5FF4FF48060FFF7D3FF4FF4FD
:1074D0000070FFF7CFFF4FF480700BE0FFF7A8FFBD
:1074E0004FF40070FFF7C6FF4FF40060FFF7C2FFD4
:1074F0004FF48060FFF7BEFF4FF48040FFF7BAFF04
:10750000014B1C6010BD00BFF4090020034B9B68B9
:1075100018420CBF00200120704700BFE402002089
:1075200010B504464FF48030FFF7F0FF012808D073
:10753000044B4FF480701C60FFF7A4FF024B002245
:107540001A6010BDF0090020100A002010B5044692
:107550004FF48030FFF7DAFF012808D0044B4FF4D6
:1075600000601C60FFF78EFF024B00221A6010BD06
:10757000D4090020100A002038B505464FF48030A9
:10758000FFF7C4FF01281FD0104B4FF480601C6828
:107590000F4B5D60FFF776FF4FF48040FFF76AFF07
:1075A000B4F5007F04D10B4B1A680B4B1A600BE04B
:1075B000B4F5807F02D0B4F5006F05D1074B186891
:1075C00008F040FC044B186038BD00BFF4090020EF
:1075D000E4020020100A002078090020E8090020B9
:1075E00008B5034B1B68C018FFF7C6FF08BD00BFF6
:1075F000D009002008B54FF40040FFF787FF0128AD
:1076000014BF0020012008BD034B93F89C2040EAE2
:10761000020283F89C2070474C000020034B93F833
:107620009C2022EA000283F89C2070474C00002036
:10763000034B93F89C3018420CBF00200120704788
:107640004C000020034B93F8CD2040EA020283F85F
:10765000CD2070474C000020034B93F8CD2022EA48
:10766000000283F8CD2070474C000020034B93F8B4
:10767000CD3018420CBF0020012070474C00002084
:1076800008B52F20FFF7F6FE08BD00BF034B10B56D
:107690009C68FFF7F5FF204610BD00BFE402002004
:1076A000034B10B59C68FFF7EBFF04F02F0010BDF3
:1076B000E402002038B505464FF48030FFF726FF7E
:1076C000012838D01C4B4FF400701C681B4B1D6008
:1076D000FFF7D8FEB4F5807F02D0B4F5006F05D176
:1076E000174B186808F0AEFB164B1860164CA368D1
:1076F00013F4005F05D1FFF7D3FF10B94FF4005327
:107700002361124B93F85630012B08D0022B09D17C
:107710000D4B4FF400525A61A2F5005200E00022D6
:10772000064B1A60094B93F85120012A03D1084BEC
:10773000197B01B91A7338BDF4090020200A002012
:10774000E8090020100A0020001001404C00002031
:10775000E4020020014B1868704700BFEC090020CC
:10776000014B1868704700BF240A0020014B58687D
:10777000704700BF240A0020014B1868704700BF03
:1077800080090020014B5868704700BF8009002025
:10779000014B1868704700BFA8090020014B5868CA
:1077A000704700BFA809002008B54FF48030FFF7EC
:1077B000ADFE01280DD04FF40030FFF7A7FE0128E1
:1077C00007D04FF40040FFF755FE4FF40040FFF79D
:1077D0002FFE08BD08B54FF40030FFF797FE0128D3
:1077E00006D00020FFF79CFE024B01225A739A73C9
:1077F00008BD00BFE4020020034B587B052814BFDE
:1078000000200120704700BFE40200200138052855
:1078100022D8DFE800F00717030F0B13012916D059
:10782000022912E0052912D003290EE004290ED006
:1078300001290AE006290AD0052906E0022906D016
:10784000042902E0032902D0062905D101E0012024
:1078500003E04FF0FF3000E000207047012808B53A
:1078600007D010F1050F04D0B0F1FF3F01D005287B
:1078700003D12020FFF7FEFD03E010B12020FFF729
:10788000D7FD08BD124B134A93F8513010781249B6
:10789000032B087005D8022B05D223B1012B16D17A
:1078A00010E0802B13D10D4B9968094B01F00701B3
:1078B00093F85420074B19704AB11A7882F00702E6
:1078C0001A7004E0064B9B68C3F382131370704771
:1078D0004C000020040A00201C0A0020000801407F
:1078E000000C0140704700BF08B50120FFF7BEFE45
:1078F00048B1054B002204201A60FFF7B7FE10B113
:107900000120FFF7A9FE08BDD009002008B5044BEF
:1079100093F8D8301BB94FF40030FFF7ABFD08BD2A
:107920004C00002008B54FF48030FFF7A3FD08BDE0
:1079300008B5042002F0D6FE10B1042002F0E0FEEB
:1079400008BD00BF10B50120FFF772FEF0B1104A6C
:1079500000230124D47313610E4A0F4819461360A3
:1079600004F068F90420FFF763FE10B12046FFF72A
:1079700055FE0A4B93F851300BB1052B06D1074B3E
:10798000D3F8983013B1024B05225A7310BD00BFD3
:10799000E4020020EC090020000400404C0000201C
:1079A00008B54FF4807002F09DFE38B14FF480703E
:1079B00002F0A6FEFFF7C6FFFFF796FF08BD00BF67
:1079C00070B5274B9C68274B04F0070493F854309C
:1079D0000BB184F00704244B21461D7D234E28461D
:1079E000FFF714FF1F4B3268B3F85830821819B2F2
:1079F0000029326003DD052D2FD1042C04E0002B7B
:107A00002BD0042D29D1052C27D1164D062295F80F
:107A100055305343154A1268002AB8BF52429A4261
:107A20001BDB134A002313600F4A194613611148E8
:107A300004F000F9B5F95830002B02DDB5F95C30DF
:107A400005E0D5F89430B5F95A20013B9B1A054A58
:107A5000C2F89830044B01225A75034B1C7570BD57
:107A6000000801404C000020E40200200C0A002025
:107A7000EC0900200004004037B5154B154993F878
:107A800051200120022A087021D093F85420124B73
:107A90009968124B01F0070119701AB11A7882F037
:107AA00007021A700E4B0D4C1A680E4B08481B78D3
:107AB0002578084C90F85610247890F869000095C5
:107AC000019406F033FE0848202103F073FE3EBD0A
:107AD0004C000020CC09002000080140040A0020CE
:107AE000D8090020E4090020002C014037B52C4CB7
:107AF000237B012B11D12B4B2B4D9A68A37DC2F315
:107B00008212A85CC01AFFF7A9FE2020FFF7FEFC36
:107B100018B9264B1B78EB5CA375214B2449DA7D01
:107B2000244B022A04D100220A70204A127801E074
:107B300001220A701A70204B1B7813B1012B19D146
:107B400007E01E4B184993F85400184A194B38B1F6
:107B50000AE01A4B144993F85400144A154B18B113
:107B60001B7859180B7C02E01B7859180B7A03F02C
:107B700007031370124B0D4C1A680F4B0F481B78FC
:107B800025780B4C90F85610247890F869000095F1
:107B9000019406F0CBFD0B48202103F00BFE3EBD07
:107BA000E4020020000C014054010020040A0020DF
:107BB000CC0900201C0A0020E40900204C00002011
:107BC000D8090020002C014037B50D4890F85130FD
:107BD000012B13D80B4B0C4C1A680C4B90F8561019
:107BE0001B7825780A4C90F8690024780095019458
:107BF00006F09CFD0748202103F0DCFD3EBD00BFE0
:107C00004C000020D8090020040A0020E4090020CC
:107C1000CC090020002C0140F7B51F4C1F4B2278E7
:107C20001F4D1A701B781F4E5B191B7C1E4803F0FA
:107C3000070323701D4B90F856101A681C4B90F8E0
:107C400069001B78277836780097019606F06EFD5C
:107C50002021184803F0AEFDEB7C227803F00703E7
:107C60009A4217D1144B00241C76204607F09AF94B
:107C70000146204607F09EF9012007F093F90146DE
:107C8000012007F097F9022007F08CF90146022045
:107C900007F090F9FEBD00BF040A00201C0A002076
:107CA00054010020CC0900204C000020D8090020FD
:107CB000E4090020002C0140E4020020F8B5354B17
:107CC00093F8514014B1012C61D10FE0324B334A8B
:107CD00019781878324B89188218127E087E997D9F
:107CE0009A75401AFFF7BAFD012451E02A4B1A7821
:107CF0002C4A10781978FFF789FD071E1BDD284DE7
:107D00000021EB69284A8B42116030DA03F094FBC2
:107D1000064606F083FA2B6A6C6AF31A041B48F6CF
:107D2000A04202FB0434214B68629C4294BF0024B1
:107D300001242E621CE01AD0194D1B4AEB69146015
:107D4000002B14DD03F078FB064606F067FAAB6AF9
:107D5000EC6AF31A041B48F6A04202FB0434134BEE
:107D6000E8629C4294BF00240124AE6200E001243A
:107D70000B4BDF6144B1084A0849127820208A5C25
:107D80009A75FFF777FB03E02020FFF751FB0024F3
:107D90002046F8BD4C000020040A002054010020B9
:107DA000E40200201C0A0020480A0020BFCF6A001D
:107DB000022138B51F4803F0A1FF01281AD1022182
:107DC0001C4803F0A1FFFFF75DFD1B4B93F85130FA
:107DD000032B0FD0FFF772FF012809D1174C184B66
:107DE00025681878174B1978FFF710FD40192060A7
:107DF000FFF7EAFE01210F4803F080FF012801464A
:107E000016D10C4803F080FF0F4B1B7E13B1FFF718
:107E100003FF0DE0084B93F85130042B01D1FFF71D
:107E200065FE054B93F85130022B01D8FFF724FE75
:107E300038BD00BF000800404C000020D0090020E1
:107E40001C0A0020040A0020E4020020022138B5A8
:107E50004FF0804003F052FF012826D102214FF05D
:107E6000804003F051FFFFF70DFD204B9B7B012B62
:107E700006D11F4B93F86630012B01D1FFF7A0FD0F
:107E80001B4B93F85130032B0FD0FFF717FF01283E
:107E900009D1184C184B25681878184B1978FFF73A
:107EA000B5FC40192060FFF78FFE01214FF08040A4
:107EB00003F024FF0128014617D14FF0804003F062
:107EC00023FF0A4B1B7E13B1FFF7A6FE0DE0084B04
:107ED00093F85130042B01D1FFF708FE044B93F8BF
:107EE0005130022B01D8FFF7C7FD38BDE402002056
:107EF0004C000020D00900201C0A0020040A0020A9
:107F000010B506F08BF9284B1B6BC31A002BB8BFBA
:107F10005B42FA2B47DD042007F044F804460820B2
:107F2000FFF7F4FAD0B940F6B3239C420BD90830DE
:107F3000FFF77EFA1D4B04221A614FF4005203F53D
:107F400080635A612BE0B4F5156F0BD80820FFF75A
:107F500091FA164B0422164C5A6111E040F60B239D
:107F60009C421CD80820FFF785FA104B9A6812F043
:107F7000040F02D004225A6101E004221A610C4C61
:107F8000A36813F4005F0AD1FFF78AFB38B900F544
:107F90000050FFF7BBFA10B94FF40053236106F00D
:107FA0003DF9014B186310BDE4020020000C0140B4
:107FB0000010014008B506F031F91D4B5B6BC31A88
:107FC000002BB8BF5B42B3F57A7F2FDD194B93F8D6
:107FD0006730012B0DD1032006F0E4FF40F6E1539A
:107FE000984206D9144B4FF4005204205A61FFF70F
:107FF0001FFA032006F0D6FF40F21633984203D949
:108000000B4B93F8383013B90220FFF711FA002018
:1080100006F0C8FF18B9064B93F8383013B10220A8
:10802000FFF728FA06F0FAF8014B586308BD00BFC5
:10803000E40200204C0000200010014010B506F0C2
:10804000EDF81D4CE36BC31A002BB8BF5B42B3F5D0
:108050007A7F30DD194B9A6812F4806F24D19B68C7
:1080600013F4005F09D00120FFF7E2F994F84030E3
:108070000A2B02D8013384F84030114A00210F4BFB
:10808000116010480022996802600F4811F4005FE7
:1080900002600CD0084A92F840200A2A07D84FF410
:1080A00000621A615A6102E0002384F8403006F051
:1080B000B5F8014BD86310BDE40200200010014068
:1080C000100A0020080A0020200A002010B5344BB6
:1080D00093F83820002A61D1013283F8382006F065
:1080E0009DF8044601E0FFF7A9FF2E4B9B6813F4AF
:1080F000806F08D106F092F8001B0028B8BF4042FC
:10810000B0F57A7FEFDB06F089F8041B002CB8BFCE
:108110006442B4F57A7F03DB214B002283F83820D8
:10812000214B93F85130032B02D8022B19D205E0D2
:10813000052B16D002D3802B21D112E006F06EF869
:10814000174B586406F06AF8154B5A6C821A002ACD
:10815000B8BF5242C72AF5DD01221A76134B1A70B6
:108160000DE006F05BF80E4B586406F057F80C4B28
:108170005B6CC31A002BB8BF5B42C72BF5DD002038
:108180004FF4006106F016FF01204FF4006106F085
:1081900011FF02204FF4006106F00CFF10BD00BF7C
:1081A000E4020020001001404C000020040A0020DE
:1081B00008B50248202103F0B7FD08BD002C01409E
:1081C00070B54F4B064693F85120032A48D006D38A
:1081D000052A7FD067D3802A40F090807AE006F0AD
:1081E0001DF8484B05469B6C984201DBC21A01E022
:1081F000DB43C218444B4549012E1C6808BF414B64
:10820000097808BFDC643F4B39B9DB6C9C4201DB69
:10821000E31A09E0DB431B1906E0DB6CA34201DB38
:108220001B1B01E0E143CB1842F210714B43344871
:10823000364990F855000978400800290CBF012103
:108240004FF0FF3159434243314E91FBF2F1306818
:10825000402205F0DDFA2B4B3060DC649D644DE07C
:10826000284A2C4B556D1C6802EB8500116D2A4B7A
:10827000866D0135611805EA0303891B002B8465AF
:10828000116505DA013B6FEA03736FEA137301337B
:10829000224841431A48D0F8940053651C4B91FB87
:1082A000F0F119602AE093F85520164B1C49D3F8D9
:1082B0009830520891FBF3F1154B91FBF2F11960E4
:1082C00019680029B8BF49424A43B2F5897F15DCD5
:1082D000002212E00B490E4BD1F89C206AB1D1F874
:1082E000982012214A4306494FF4806091F85510B6
:1082F00092FBF0F2490892FBF1F21A6070BD00BFE8
:108300004C000020E4020020D0090020E4090020F5
:10831000E8090020140A00200F000080F824010062
:1083200080A8120110B504464FF48040FFF7A2F870
:10833000034B01201C60034B5C60FFF741FF10BD45
:10834000D0090020E402002038B5484B5B7B013B9C
:10835000062B00F28A80DFE803F004884588881540
:108360007E000020FFF7DCF8414B002283F86920F3
:1083700083F8512005F052FF3C4B06225A73C3F894
:10838000A00072E005F04AFF384C394DD4F8A02027
:10839000B5F95E30821A002AB8BF52429A4217DD00
:1083A000344A0023B5F9580063751360FFF782F96A
:1083B000314BB5F958101A68022391FBF3F39A4236
:1083C00001DB032363734FF40040FFF753F84CE0E5
:1083D0000020FFF7A5F8294B002201201A60FFF7C3
:1083E000EFFE42E0214C657D012D1BD10020FFF7FF
:1083F00061F9214B1B68002BB8BF5B42042B34DCB6
:108400002846FFF7DDFE1A4B00220521A273617397
:1084100003214FF4004083F8511083F86920FFF7DF
:1084200007F822E04FF40040FFF724F8144B1A68D5
:108430000F4BD3F890309A4217DB05F0EFFED4F8DB
:10844000A030C31A002BB8BF5B42B3F5FA7F0CDD36
:108450000723637309E04FF40040FFF70BF8034A6A
:10846000002318469373FFF75BF838BDE402002041
:108470004C0000200C0A0020E8090020D009002050
:10848000F809002010B50446214803F02FFC214BC9
:1084900093F86830012B04D1C0F57E4000F5FF70E1
:1084A000013043F6FE711C4B88421B6807DC1B4AF7
:1084B0001269B2F5404F0FDBC2F580320AE0B0F529
:1084C000404F09DB154A12698A4205DCC2F17F423E
:1084D00002F57F02121802E0104A1269821A012C7A
:1084E00003D10F490C6814190C600A49D318D1F84C
:1084F00094100C4C8B42226001DB5B1A02E0002BD3
:10850000B8BF5B18054A1061034A136010BD00BF75
:10851000000400404C000020EC090020E402002090
:10852000D0090020140A00200121F8B5A84803F062
:10853000FBFBA84AA84BD2F8A41093F851300131A4
:10854000012BC2F8A41001D9042B32D105F082FE10
:10855000FF2837D006F09CFDE0B901219F4801F0CB
:1085600001FE05F077FE06F035FD9D4B9D4C186031
:108570001868994BB3F8641006F05EFD9A4B0146FB
:108580001B78012B08BF41422068802205F040F98A
:10859000206017E08F4BD3F8A8200132B2F57A7F24
:1085A000C3F8A8200ED30022C3F8A82006F076FD59
:1085B00008E006F06DFD08B106F070FD8748012166
:1085C00001F0D0FD834CA67B012E45D1824D95F85C
:1085D0006670002F40D13046FFF754FF834B394679
:1085E0001868FEF791FE637B0746032BC4F8AC00C6
:1085F00049D13046FFF71CF830B17D4B95F8550056
:108600001A68B2EB400F4CD3BB059B0D002B6CD10D
:10861000714B4FF00401B3F95820002A6D4A517391
:1086200074490EDB93F855C0D3F8942008684FEADC
:108630005C01B2FBF1F1091AB1FBF2F002FB10127E
:1086400004E0D3F894200968013A521AC3F898203C
:10865000604BC3F8B47048E05E4CA67B012E4DD150
:108660005D4D95F86630022B48D13046FFF70AFF82
:108670005E4B00211868FEF747FE637B0746032B1D
:10868000C4F8AC0002D0042B2FD12AE03046FEF70C
:10869000CFFFE8B1564B95F855001A68B2EB400F82
:1086A00016D25449D4F8B0600F68D5F89450C6EB90
:1086B000070CBCF1000FB5FBF0F0B8BFCCF1000C1B
:1086C000844512D309680132C4F8B0101A600CE076
:1086D000BB059B0D4BB93F4B0422C3F8B4705A73D2
:1086E00003E0D4F8B430C4F8AC303A4B3A4AB3F8AB
:1086F000B81092F85620D3F8AC0042E0364B93F80D
:108700005130052B00F2D380DFE813F0CE00D1000A
:108710003E002600D10006000120FFF7B3FE2D4BDE
:108720003149D3F89C200978C3F8BC2019B1D3F89B
:10873000C0108A1A02E0D3F8C0105218C3F8C02043
:10874000244B254AB3F9C24092F85620B3F8B8102A
:108750002046C3F8AC4014E00120FFF793FE1E4D05
:10876000244BD5F898101868FEF7CEFD194CC4F8C4
:10877000AC0007F09FF8B4F8B81095F85620D4F87C
:10878000AC0006F013F892E01748124B90F800C0C6
:10879000D3F8C020D3F8BC10BCF1000FD3F8C4400C
:1087A0001144007814BF6FF0FF024FF4807202EBA7
:1087B00021420134C3F8C010C3F8C440C3F8AC2050
:1087C0000549C8B1B1F95A105218524217E000BF1A
:1087D000002C0140E40200204C0000200024014055
:1087E000DC090020F8090020E40900207C090020B1
:1087F000000A0020EC090020B1F95C105218C3F8FF
:10880000AC202B4C2B4B94F85620B3F8B810D3F86F
:10881000AC0005F0CBFF284B284A19781170284A84
:10882000916894F8542001F0070119701AB11A7870
:1088300082F007021A70204B224A1B78127812B17C
:10884000012A0FD106E0013BDBB2052B0AD81E4AF4
:10885000D25C08E0013BDBB2052B03D81A4A9B1817
:108860001A7A00E00622134B93F8C81091421ED0EA
:10887000D3F8C400154C03EB8101B4FBF0F0C1F850
:10888000CC0003EB8201D1F8CC104FEA826C0620B9
:108890009CFBF0F00024C3F8C440C3F8C000C3F848
:1088A000BC1083F8C82002E00020FFF7EBFDF8BD04
:1088B0004C000020E4020020040A00201C0A0020D2
:1088C00000080140E4090020C4020108AAAAAA0085
:1088D000264B4FF4007210B5254C1A61012006F0AA
:1088E000E3FB94F8510006F039FA94F8510006F0D1
:1088F00075F994F8510006F0BDF84FF40040FEF70A
:1089000097FD1C4B93F82020012A06D1013A94F8D8
:10891000510083F8202006F011F8154C94F851000E
:1089200005F0A4FF94F8CC00104B4FF400425A61BC
:1089300000B101200D4C06F0BDFB4FF480532361C4
:1089400003F540532361A36813F4005F0AD1FEF7D7
:10895000A7FE38B900F50050FEF7D8FD10B94FF466
:1089600000532361FFF7B2FB10BD00BF00100140B0
:108970004C0000205401002010B5264B1A7B012A20
:108980001AD193F8E4100A46B1B993F8E510012919
:1089900012D1214991F8510001280DD01F4C1A73B2
:1089A00022601F4881F8692005F0A2F81D4805F0F3
:1089B0009FF81D4805F09CF8164A137B012B21D027
:1089C000154B92F8E51093F8513099421AD0527B2A
:1089D000052A03D0154A012182F82010042B09D161
:1089E0000C4B4FF6FF72C3F898204FF47A72C3F81D
:1089F000E82005E0052B03D1064B0022C3F89820A0
:108A0000FFF766FF044B93F85120024B83F8E520F3
:108A100010BD00BFE40200204C000020080A002026
:108A200080090020240A0020A80900205401002009
:108A30002DE9F04788B005F0F1FBA54C0546D4F8C8
:108A4000EC30C31A002BB8BF5B42B3F57A7F17DB5B
:108A5000D4F8F0301846C4F8F43006F001FFD4F82A
:108A6000FC10D4F804210023C4F8EC50C4F8F8102A
:108A7000C4F80021C4F80431C4F8F030C4F8FC3064
:108A8000944A934B1168944AD3F8F00092690029F4
:108A9000B8BF49420130002AB8BF52429142C3F8E0
:108AA000F00003DC1020FEF7C3FC02E01020FEF70C
:108AB000E1FC8A4B0021186807F0ACFBB0B1864B93
:108AC00093F85630012B06D14FF40050FEF7D2FC3C
:108AD0004FF4805007E0022B10D14FF48050FEF786
:108AE000C9FC4FF40050FEF7A3FC07E04FF48050A0
:108AF000FEF7C0FC4FF40050FEF7BCFC764B93F839
:108B0000CC0000B10120724D06F0D4FAFFF734FF1B
:108B1000FFF750FAFFF7F4F9FEF792FC2B7B002BDE
:108B200000F044816E4B1C6874B92046FEF7F8FCD7
:108B3000694B6FF07F0283F86920813283F85120FE
:108B4000FFF7C6FE85F8E440614C94F8E430072B4B
:108B500000F22C81DFE813F008001F002C00360023
:108B60002A0177002A0110015C4A00231360C4F82F
:108B700008310023E3755B4804F0BAFFD4F808011C
:108B800007F07AFBFEF7E2FC554B1B68002B00F068
:108B90000D81012212E0504B0025042283F8512060
:108BA00083F86950FFF794FEC4F80C51022347E0A4
:108BB000D4F80C31632B40F2F9800322444B83F844
:108BC000E420F3E0D4F80851414C284607F054FB68
:108BD000414B0028D3F89030B8BF4042984218DA91
:108BE0003F4B1B68002B08DB284606F0CDFF36A361
:108BF000D3E9002306F06AFE07E0284606F0C4FF2A
:108C000031A3D3E9002306F05FFE07F011F8C4F8A2
:108C100008012F4CD4F8080107F02EFBFEF796FC54
:108C2000D4F8080107F028FB2B4B0028D3F890302C
:108C3000B8BF40429842C0F2B9800223E3750333C3
:108C400084F8E430B2E0234B234C1B68D4F8DC10EA
:108C5000002BB8BF5B428B42C0F2A880224DD4F8F3
:108C600044E0D4F848C0E76CD4F8B860D4F8BC80CD
:108C7000D4F8C0A0D4F8C4902269236C2846CDF85B
:108C800000E0CDF804C002970396CDF81080CDF82F
:108C900014A0CDF8189004F031FF2B69A168AA69DF
:108CA00063B1B2F57A7FA8BF4FF47A724A434FF4AA
:108CB0007A71B2FBF1F2120492FBF3F3084A1268E4
:108CC000002A13DD032214E09A9999999999A93FF2
:108CD000E4020020E80900204C000020100A0020D7
:108CE000200A0020A80900208009002005D06FF08C
:108CF000020293FBF2F37A4A53607A48042102F0AD
:108D000081FF7848002102F005FE76484FF6FF719A
:108D100002F092FF7348012102F0FCFD714800212E
:108D200002F088FF704B71481A68714B714C1B78C8
:108D3000067871484FF0010C057884F851C06FF047
:108D40007F0C84F869C094F8561080200096019535
:108D500005F0ECFC2021694802F02CFD684B1868F6
:108D6000FEF7A8FC674B00221A6005F057FA664B25
:108D7000072283F8E42017E0624B1B68282B05DDEF
:108D8000624B00221A605E4B00221A6005F046FA20
:108D90005D4BD3F81021821A002AB8BF5242632AD1
:108DA00004DD584A00211160C3F81001564CA37B22
:108DB000002B76D04F4B93F86630012B25D002D391
:108DC000022B6ED124E0637B013B042B69D8DFE8E2
:108DD00003F0280368166200E37D022B02D14A4BA0
:108DE00003225A730120FEF70FFC0420FEF70CFC4F
:108DF0000120FEF727FC0420FEF724FC51E0D820D8
:108E00004349042206F0DAFA39E0FFF79DFA48E018
:108E1000637B013B042B44D8DFE803F003194331A3
:108E20003D00344B6FF07F02B3F9580083F85120B6
:108E3000FEF740FCE37D13B9334B0122DA75324A69
:108E400000230221D3735173324A136029E0E37D7A
:108E5000022B02D12C4B03225A730120FEF7D4FBC4
:108E60000420FEF7D1FB0120FEF7ECFB0420FEF707
:108E7000E9FBD8202649042206F07CFA11E01D4ABD
:108E800000230321184682F85110E375FEF712FC07
:108E90000523637305E000234FF40040A373FEF73E
:108EA000C7FA194AD2F81431002B3FD00023C2F878
:108EB0001431194A126812B10B4A126882BB0E4B68
:108EC00001221A70154B4FF480425A61002300BFF3
:108ED00001330A2BFBD1114B4FF480421A6125E07C
:108EE0008009002000080040D8090020040A002062
:108EF000E40900204C000020CC090020002C014097
:108F0000200A0020FC090020E4020020100A0020B2
:108F1000E4000020000A0020E809002000100140C1
:108F20009D4A4FF4804111619C4A13709C4C9D4DA9
:108F3000D4F818216B6B9A42C0F07982D4F80421DE
:108F4000002301321846C4F80421C4F81831FFF791
:108F500037F94FF40040FEF7D9FA012827D14FF432
:108F60008060FEF7D3FA012821D18F4F8F4E6268BF
:108F70003B68D6F800C08E492846CDF800C004F002
:108F800049FD62683B688B49D21A002A6B69B8BFF9
:108F900052429A4208600ADC3268EB68002AB8BF85
:108FA00052429A4203DC4FF48040FEF741FA4FF4FC
:108FB0000040FEF7ABFA012840F00C81794D95F89E
:108FC0005030012B40F006814FF48060FEF79EFA8E
:108FD000012840F08D8095F851302C6873B9764B9C
:108FE0001868014606F082FF744906F07FFF0646C6
:108FF00095F85500400806F025FF0DE0032B01D041
:1090000000231AE06C4B1868014606F06FFF064615
:10901000D5F8940006F012FF0146304606F066FFD0
:10902000EB6906467820584306F00CFF01463046AF
:1090300007F010F807F020F90346594A4FF4804032
:109040005168594A5C4D12689142554AB8BF644212
:109050005168554A12688A1A002AB8BF52429A4289
:10906000D8BF0024FEF752FA012804D1514B1868EA
:1090700006F0E8FE37E0204606F0E4FE2E680746DC
:109080003946304607F0D0F888B1464B44B95A6BA0
:109090000C214A43D869504306F0D0FE48491CE0F1
:1090A000586BDB69584306F0C9FE464915E039465E
:1090B000304607F0D7F8B8B13A4B44B95A6B0C2197
:1090C0004A43D869504306F0B9FE3F4905E0586B62
:1090D000DB69584306F0B2FE3C4906F0BBFF01468F
:1090E000304606F0FBFD2860334B1A68384B1A6097
:1090F0004FF40070FEF70AFA012871D1294DEE698C
:10910000002E67D095F85130802B63D0294B304C1E
:10911000186806F097FED4F80080074639464046A6
:1091200007F082F8B0B1686B2768704306F086FEDE
:10913000244906F08FFF0146384606F0CFFD206037
:10914000286806F07FFE266805462946304607F067
:109150006BF81CE02068394607F084F800283FD0FF
:10916000686B2768704306F069FE184906F072FFC5
:109170000146384606F0B2FD2B682060584206F0E2
:1091800061FE266805462946304607F06BF800B1B7
:1091900025680F4B1D6023E000100140CC09002022
:1091A000E40200204C000020D0090020E809002043
:1091B000240A0020200A0020780900200000C04076
:1091C00000401C4600007A4400401CC600007AC4DF
:1091D000100A00207E4B186806F034FE7D4B1860A4
:1091E0004FF40040FEF792F901280FD07A4B5A7BDA
:1091F000062A0BD05A7B032A08D0784A92F85120CD
:10920000012A3ED193F8E430072B3AD14FF4007095
:10921000FEF77CF9012805D04FF48060FEF776F95F
:1092200001282ED16D4C94F85130802B29D0042B7D
:1092300027D0684D6A4B28681E6807F01DF8334632
:1092400002466849204604F06FFB94F85130664AA4
:10925000012B106015D12868002107F003F818B120
:10926000624B1B68012B08D05A4B0021186806F08E
:10927000DBFF30B15D4B1B681BB95D4B1A680132D7
:109280001A604FF40070FEF741F9012821D1534ACA
:1092900092F85130802B1CD1564BB2F958101868F7
:1092A0000029ACBF01214FF0FF310918196019687E
:1092B000002904DAD2F8942019688A181A604D4BF4
:1092C000464A1968D2F89420B1FBF2F002FB101262
:1092D0001A604FF40060FEF719F9012805D03E4BE3
:1092E00093F8E430052B40F0A2803C4B93F85130CA
:1092F000042B40F09C80384BDA7D022A08D04FF6D0
:10930000FF72C3F898204FF47A72C3F8E8208EE019
:10931000DA7D022A40F08B802D4A1268002A08D19B
:109320004FF6FF72C3F898204FF47A72C3F8E82022
:1093300004E0314BCCBF002201221A70284A244B92
:1093400011681B6899421ADA244A234BD069556B7D
:10935000D3F8E84092F8551005FB0040274A490829
:1093600092FBF1F191FBF0F10A2251434FF6FF72AB
:109370009142C3F8E800C3F898101EDD1BE01268A4
:109380009A421ADD154A144BD469506BD3F8E85051
:1093900092F8551000FB1450184A490892FBF1F15D
:1093A00091FBF0F10A225143154AC3F8E8009142BB
:1093B000C3F8981001DAC3F89820094B1A68002AFC
:1093C00020DD094B1A68002AB8BF524222E000BFD4
:1093D000200A0020100A0020E40200204C00002097
:1093E000E809002080090020D4090020480A002054
:1093F000FC0900207C090020E409002000D2496B10
:109400000100FFFF1B68002B05DA7A4B1A68002A5F
:10941000C8BF52421A60784C206806F013FD2368DA
:10942000764A1060184606F00DFD754B1860754CB5
:10943000754BD4F8A4209B6B9A42C0F09081D4F86D
:10944000FC30002201334FF40040C4F8A420C4F8DB
:10945000FC30FEF75BF8012805D0637B072B1BD19E
:109460006A4B1B68C3B94FF48070FEF74FF80128B0
:1094700012D1664B66491C681A68002CB8BF64425A
:10948000002A0C6003DD634B00221A7004E01B68A5
:10949000002BBCBF5F4B18705B4B93F85130052B12
:1094A00006D003D8023B012B18D801E0802B15D140
:1094B00005F01EFE584B594C18601868524BB3F813
:1094C000641005F0B9FD534B01461B78012B08BF12
:1094D00041422068402204F09BF920604A4B93F8F7
:1094E0005120012A01D9042A07D1474B4B4A996BD5
:1094F00010684900D3F8D42004E04849D3F8D420B8
:109500000868996B04F0EAFD04F020FE3E4DD5F8A2
:10951000D030984227D904F081FE3A4CD4F81C315F
:10952000C31A002BB8BF5B42B3F57A7F1BDB04F094
:10953000CDFD4FF40030FDF77BFF95F8D8305BB9D7
:109540002946012201F8D82F4FF48C7005F036FF20
:1095500004F064FEC4F8200104F00AFE04F05EFE8C
:10956000284BC3F81C0104F059FE264B2649D3F8BA
:109570002021D1F8D430821A002AB8BF52429A4230
:109580000AD391F8D820012A06D1002301F8D83F48
:109590004FF48C7005F012FF1B4B93F8D830012B61
:1095A00003D14FF40030FDF743FF174B93F85130D0
:1095B000802B01D0052B52D1124BDB7D012B4ED1DC
:1095C000174B1B681BB1104BD3F890301BB9104BD5
:1095D00000221A6043E0114A124D1468002CB8BFF3
:1095E00064421C1B002C1FDD28684FF0745106F0EC
:1095F00075FB1EE0D4090020E8090020780900204E
:10960000100A0020E40200204C000020F009002095
:10961000080A0020E4090020DC090020F8090020E5
:10962000200A0020180A002028684FF0745106F024
:1096300053FB914B2860914D00215A68286804F033
:10964000CFF8286006F018FE0028B8BF40428C4BC7
:109650001334262C186002D88A4B0222DA754FF494
:109660000040FDF753FF012806D0864B5A7B062A9F
:1096700002D05B7B032B46D14FF48060FDF746FFA1
:1096800001280BD04FF40070FDF740FF012805D0F2
:109690004FF40060FDF73AFF012834D1764C94F87E
:1096A0005130802B2FD0042B2DD8774B77491A6857
:1096B000774B20461B680D687649009504F0C8F882
:1096C00094F851306E4A012B106001D0042B10D158
:1096D000714B1B68002B03DD674B00215A6804E0C7
:1096E00007D0654B00225968494204F071F8644B79
:1096F0001860634B1B68002B01DD002201E002D0E3
:109700000122664B1A70664B186805F06FFC4FF427
:109710000030FDF7FBFE01280BD1594B00226148B8
:109720001A6004F0E5F9604804F0E2F9594804F0E1
:10973000DFF9574B1A68504B002A9B68B8BF52425A
:109740009A4206DD0120FDF773FE584B20221A6174
:1097500005E00120FDF78EFE544B20225A61464B56
:1097600093F85120032A33D005D8012A10D0504C49
:10977000434A39D806E0052A6CD046D3802A40F007
:10978000B6809BE010685A680028B8BF40420BE0E2
:109790005B6809225A433A4B454C18680A23002853
:1097A00092FBF3F2B8BF4042002104F011F82060B0
:1097B0002168404889B202F041FA21683D4889B2E7
:1097C00002F03EFA21683B4889B202F03BFA8EE093
:1097D0005A682B4B002118680028B8BF404203F09C
:1097E000F7FF334B18600AE012685B68002AB8BFC5
:1097F0005242226022689A42C8BF23602C4B1A68EA
:10980000022392FBF3F21F4B6FE05A681C4B284C6B
:1098100018680028B8BF4042002103F0D9FF20603B
:109820002168244889B202F009FA2168214889B2E6
:1098300002F006FA21681F4889B202F003FA114BC0
:109840001D48D3F898100029B8BF494289B202F0E8
:10985000F3F94CE00A49164A09685B680029B8BF69
:109860004942116011689942C8BF1360054B104A04
:10987000D3F89810106830E04C000020180A00203F
:10988000080A0020E4020020D4090020E809002092
:10989000F8090020A8090020200A0020E40900207F
:1098A000DC09002080090020240A0020000C01406F
:1098B000D8090020002C0140000800405A68444BA1
:1098C000002118680028B8BF404203F081FF414AD8
:1098D000414B10601068D3F8981002220029B8BFDD
:1098E000494290FBF2F2C3F89C10C3F8B8203B4BFE
:1098F00093F8522012F0010F22D0394A1268002A40
:109900001EDA93F8533013F0010F03D0002005F056
:109910001DFD40B9314B93F8530010F001000FD1F9
:1099200005F014FD60B90220FDF7A0FE10B12D4B2B
:1099300000221A602C4B00221A602C4B00221A6065
:10994000264B93F8522012F0020F23D0244A1268BB
:10995000002A1FDD93F8533013F0020F03D00120CB
:1099600005F0F4FC48B91D4B93F8533013F0020F87
:1099700010D1012005F0EAFC60B90220FDF776FE67
:1099800010B1184B00221A60174B00221A60174BB7
:1099900000221A60164EF369BBB1164D2C78A4B99B
:1099A00004F03CFC144AF3691268821A002AB8BF1A
:1099B00052429A4209D901232B701020FDF738FD3D
:1099C000094B00221A60094B1C6008B0BDE8F08703
:1099D000080A0020D8090020E40200204C000020E2
:1099E000E8090020D0090020100A0020200A0020E9
:1099F00008000020700900206C090020AFF30080EF
:109A0000014B03221A60704708040020044A054BEA
:109A1000927A0AB1052200E001221A60704700BF65
:109A2000580A002008040020704700BF014B0022A4
:109A30005A6070470804002008B5074B1A6892B2B4
:109A400042F008021A601A6892B242F004021A60E8
:109A5000FFF7D6FF08BD00BF405C004010B5064CC4
:109A60004FF6FB73226802EA03032360FFF7CEFF81
:109A70004FF40643236010BD405C0040072818BF28
:109A80001F4B10B51E4C18BF18702378052B33D808
:109A9000DFE803F003060A0E1621FFF7DFFF2BE0D5
:109AA000FFF7DCFF042328E002236370013324E086
:109AB0006378013BDBB263706378FBB9042218E082
:109AC000104B1A6892B242F010021A6005232370FC
:109AD000DB18637012E06378013BDBB2637063787C
:109AE00063B9084A4FF6EF73116801EA0303136084
:109AF0000622034B1A7001E00623237010BD00BF3D
:109B0000BC0A0020405C0040034B9B7A13B1034B1E
:109B100005221A60704700BF580A00200804002080
:109B2000014B04221A60704708040020034B1A7A84
:109B3000202A01D100221A72704700BF08040020B9
:109B4000704700BF212808B508D1124B1B681B784D
:109B500003F07F03212B1AD10F4B0EE0202816D1E2
:109B60000C4B0E4A1B681B7810720D4A03F07F03E2
:109B7000212B0CBF134600234BB1064A4FF00001C6
:109B800012680020518293619847002000E0022073
:109B900008BD00BFB80A0020D99B000808040020B7
:109BA000F59B0008074B1B681B7803F07F03212BF4
:109BB00005D1022801D0222801D1002000E0022096
:109BC000704700BFB80A002019B9012801D808461B
:109BD00000E00220704700BF28B9044B4FF0080294
:109BE0001B681A8200E00248704700BFB80A0020D4
:109BF0007801002028B9044B4FF008021B681A8234
:109C000000E00248704700BFB80A00207801002039
:109C10000B4B10B5DA6882B11B68052B01D000220E
:109C20000BE0002303E00749595CC15401330449A8
:109C3000CC68A342F7D30023CB60104610BD00BF11
:109C400008040020C00A0020084BDB68082B01D85C
:109C500000200AE00023064A9A5CC2540133092B13
:109C6000F9D1024B0022DA6001207047080400207D
:109C7000C00A002010B5074C0B468AB2C0216360B1
:109C800003F00CF90120A18803F016FB012003F07A
:109C9000E1F910BD0804002008B5064B1B68DB780D
:109CA000042B01D9002004E0034901EBC30102F0B9
:109CB0009DFC08BDB80A00208001002008B50249BB
:109CC00002F094FC08BD00BFA001002008B50249C5
:109CD00002F08CFC08BD00BFA8010020334B10B57A
:109CE0001B686FF03F0200245A72DC729C7220469F
:109CF00003F028F920464FF4007103F041F91021D8
:109D0000204603F053F94021204603F0A9FA8021B0
:109D1000204603F095FA204603F0D2F9244B204662
:109D200093F8641003F0EAFA204603F0A1F9012049
:109D3000214603F025F90120C02103F081FA01201A
:109D4000202103F033F90120214603F047F90220D6
:109D50004FF4C06103F014F902204FF4807103F056
:109D60006FFA0220214603F039F90220202103F086
:109D70001DF90320214603F003F903204FF48871F5
:109D800003F06EFA0320402103F0B8FA03204FF4E9
:109D9000405103F023F92146032003F007F9204640
:109DA00002F032FC034B01221A6010BDB80A0020F9
:109DB000780100200804002008B5174B174A1968DD
:109DC00089B2118016491288098801EA020212F448
:109DD000806F05D04FF6FF321A60124BDB6B98474D
:109DE0000E4B1A880E4B1B8803EA020212F4007F06
:109DF00008D009490C4A4FF6FF500860117C013128
:109E0000C9B21174054A1288134013F4004F01D0EF
:109E100002F080FF08BD00BF445C00404E0A0020F5
:109E2000000B0020780100200804002010B503205A
:109E300003F094FA064C034602464FF48871054835
:109E4000E36003F043F8032003F012F910BD00BFF4
:109E500008040020C00A002008B520B104480421ED
:109E600000F0E0FC03E00248042100F0D9FC08BD4A
:109E70000014014038B5064D01232B60054B00242A
:109E800020461C60FFF7E8FF03232B60204638BD07
:109E9000405C0040445C004008B5FFF7EBFF08BDA4
:109EA00008B50120FFF7D8FF064B012119600649CC
:109EB0004FF4E0520A8005490020186008601A60DB
:109EC00008BD00BF405C0040000B0020445C004027
:109ED000084B10B51B6800249C72FFF7E1FF064A8F
:109EE0004FF406431460043A1360044A1460044AB1
:109EF000138010BDB80A0020445C00400804002014
:109F0000000B002007B5142200238DF8042001A8BF
:109F100001228DF806308DF807208DF8053000F00D
:109F200089FD0EBD002008B500F092FF4FF400003F
:109F3000012101F025F808BD07B5FFF7F3FFFFF792
:109F4000E1FF02F089FE2020012101F00BF803233C
:109F50008DF806300D338DF8073004484FF00403B8
:109F600001A9ADF8043000F0F5FB0EBD001401406E
:109F7000704700BFFEE700BFFEE700BFFEE700BF7F
:109F8000FEE700BF704700BF704700BF704700BFCB
:109F9000704700BF704700BF704700BF704700BFE9
:109FA000704700BF704700BF704700BF704700BFD9
:109FB000704700BF704700BF704700BF704700BFC9
:109FC000704700BF704700BF704700BF704700BFB9
:109FD000704700BF704700BF08B5024B1B68984729
:109FE00008BD00BF5409002008B5024B1B68984704
:109FF00008BD00BF74090020684620F00701044B2B
:10A000008D4601B51B689847BDE8014085467047FD
:10A010005C09002008B5024B1B68984708BD00BFCB
:10A0200060090020704700BF704700BF704700BF45
:10A03000704700BF704700BF704700BF704700BF48
:10A04000704700BF704700BF704700BF704700BF38
:10A05000704700BF704700BF704700BF704700BF28
:10A06000704700BF704700BF704700BF704700BF18
:10A07000704700BF704700BF704700BF704700BF08
:10A08000704700BF704700BF704700BF704700BFF8
:10A09000704700BF704700BF08B503F0E5FD08BD7D
:10A0A000436830B523F470230C680A7923F4807375
:10A0B000234343EA0223436082688D68CC680A4BDD
:10A0C00045EA040C02EA03034A794CEA030343EA33
:10A0D000420383600B7CC26A013B22F47002DBB254
:10A0E00042EA0353C36230BDFDF7F1FF00230122B2
:10A0F0000274C3600360037143718360704700BFE3
:10A1000019B1836843F0010302E0836823F001037F
:10A110008360704719B1836843F4807302E08368F9
:10A1200023F4807383607047C9B212B14368194346
:10A1300002E0436823EA010141607047836843F00D
:10A1400008038360704700BF8068C0F3C000704799
:10A15000836843F004038360704700BF8068C0F3E6
:10A160008000704719B1836843F4A00302E083685C
:10A1700023F4A003836070478068C0F38050704769
:10A180004368013923F4604343EA41334360704735
:10A1900019B1436843F4006302E0436823F40063A9
:10A1A00043607047092930B511D94FF0030C0CFBFF
:10A1B00001FC0725ACF11E0C05FA0CF503FA0CFCAA
:10A1C000C46824EA050343EA0C03C3600EE04FF0C1
:10A1D000030C0CFB01FC072505FA0CF503FA0CFC3B
:10A1E000046924EA050343EA0C030361062A0DD837
:10A1F0000523013A5A434FF01F0C0CFA02FC914020
:10A20000436B23EA0C020A4342631CE00C2A0DD87C
:10A2100005235A434FF01F0C233A0CFA02FC9140DD
:10A22000036B23EA0C020A4302630CE005235A4342
:10A230004FF01F0C413A0CFA02FC9140C36A23EA2A
:10A240000C020A43C26230BD19B1836843F4801323
:10A2500002E0836823F4801383607047C06C80B28F
:10A26000704700BF014B1868704700BF4C24014085
:10A2700019B1436843F4806302E0436823F48063C8
:10A280004360704719B1436843F4805302E0436868
:10A2900023F4805343607047836823F4E04341EA2A
:10A2A00003038360704700BF19B1836843F4004320
:10A2B00002E0836823F400438360704719B1836828
:10A2C00043F4021302E0836823F4021383607047AF
:10A2D0008068C0F340507047092930B511D94FF05C
:10A2E000030C0CFB01FC0725ACF11E0C05FA0CF568
:10A2F00003FA0CFCC46824EA050343EA0C03C360B8
:10A300000EE04FF0030C0CFB01FC072505FA0CF5E1
:10A3100003FA0CFC046924EA050343EA0C03036115
:10A32000836BC3F3015CCCEB020202324FF0050CED
:10A33000D2B20CFB02F20CF11A0C0CFA02FC9140A6
:10A3400023EA0C030B43836330BD00BF836B0139E9
:10A3500023F4401343EA0153836370470A50704764
:10A360002830405880B27047436823F4400323F4F8
:10A37000007341EA03034360704700BF4162826299
:10A38000704700BF436823F01F0341EA03034360A3
:10A39000704700BF20B1054B9A6842F4000203E009
:10A3A000024B9A6822F400029A6070470024014030
:10A3B000036819420CBF002001207047C9430160A7
:10A3C000704700BF4368006810EA112004D0C9B28A
:10A3D00019420CBF00200120704700BF6FEA112115
:10A3E0000160704708B5134B98420FD003F5A05396
:10A3F000984213D0A3F5C053984219D14FF400707E
:10A40000012100F0CBFD4FF400700EE04FF48060AE
:10A41000012100F0C3FD4FF4806006E04FF40040DE
:10A42000012100F0BBFD4FF40040002100F0B6FD1B
:10A4300008BD00BF002801400268002322F001028D
:10A440000260036043608360C3602D4B984233D049
:10A4500011D83C3B984229D006D8283B984221D0BD
:10A46000143398424BD11FE0264B984220D014332E
:10A47000984244D11EE0244B98422CD008D8A3F532
:10A48000677398421DD003F56273984237D11DE07F
:10A490001E4B984229D0143398422BD0283B984227
:10A4A0002DD11DE01A4B12E0194B15E0184B18E0A6
:10A4B000174B1BE0164B1EE0154B5A6842F4700216
:10A4C0001CE0134B5A6842F0706217E0114B5A6857
:10A4D00042F00F0212E00F4B5A6842F0F0020DE01A
:10A4E0000C4B5A6842F4706208E00A4B5A6842F416
:10A4F000704203E0074B5A6842F470225A6070477A
:10A500006C000240440002401C040240440402402B
:10A5100000000240000402408A6870B50C6A0B69B2
:10A5200044EA02024C691A438B692243CC690568EC
:10A530004E6A42EA030323438C6A334325F4FE4CFC
:10A5400023432CF0F00C43EA0C030360CB68436018
:10A550000B6883604B68C36070BD00BF00238362DB
:10A56000036043608360C360036143618361C361CF
:10A5700003624362704700BF19B1036843F00103EF
:10A5800002E0036823F001030360704712B103681F
:10A59000194302E0036823EA01010160704700BF2C
:10A5A000406880B2704700BF10F0805F14BF044B5A
:10A5B000044B1B6803420CBF00200120704700BF02
:10A5C000000402400000024010F0805F14BF024B04
:10A5D000024B5860704700BF000402400000024078
:10A5E00010F0805F14BF044B044B1B6803420CBF88
:10A5F00000200120704700BF00040240000002401C
:10A6000010F0805F14BF024B024B5860704700BFD0
:10A610000004024000000240044B00221A605A600D
:10A620009A60DA60024A5A61704700BF0004014034
:10A63000FFFF0700837930B5016802794BB3184BEF
:10A64000CC431D6890F805C004EA05051D605D68EF
:10A650002C405C60D45844EA0101D15002689868EB
:10A66000D14301EA00009860D8680140BCF1100FA6
:10A67000D96007D1996811439960D96841EA02020B
:10A68000DA600BE05CF8031041EA02024CF80320A8
:10A6900004E0034BD05820EA0101D15030BD00BF87
:10A6A0000004014000230C22837142710360037196
:10A6B000704700BF024B1A6940EA02021A617047F4
:10A6C00000040140034B5B6918420CBF00200120CD
:10A6D000704700BF00040140014B5861704700BF44
:10A6E00000040140054B1A685B69034001D118461C
:10A6F00003E010420CBF002001207047000401401D
:10A70000014B5861704700BF00040140044B1A68B8
:10A7100002F038021A601A6840EA02021A607047B2
:10A7200000200240044B1A6822F008021A601A68DE
:10A7300040EA02021A60704700200240044B1A6887
:10A7400022F010021A601A6840EA02021A6070478A
:10A7500000200240CB78F0B513F0100F18BF8A78B4
:10A76000098803F00F0C18BF4CEA020C11F0FF0F20
:10A770001AD0046800220126964006EA0105B54277
:10A780000ED196000F27B7400CFA06F624EA07040C
:10A790003443282B01D1456102E0482B08BF0561F5
:10A7A0000132082AE7D10460FF291CD9446800223D
:10A7B00002F108050126AE4006EA0105B5420ED1B8
:10A7C00096000F27B7400CFA06F624EA0704344334
:10A7D000282B01D1456102E0482B08BF05610132F9
:10A7E000082AE5D14460F0BD0423C37002238370BE
:10A7F0004FF0FF3303807047836819420CBF00207D
:10A8000001207047806880B2704700BFC36819425A
:10A810000CBF002001207047C06880B2704700BFA5
:10A8200001617047416170470AB1016100E0416117
:10A83000704700BFC160704741F48033836181611C
:10A840008361836983697047064A10B514684FF6BF
:10A85000807341EA001104EA030341EA0303136031
:10A8600010BD00BF00000140014B1860704700BFE1
:10A870001C0020420304154A00F4401C1B0CBCF5CC
:10A88000401F30B5546806D1556824F0706425F037
:10A890007065556011E010F4801F06D0C0F30342CC
:10A8A0004FF0030C0CFA02F203E0420D120113FA0E
:10A8B00002F224EA020444F0706419B1400D000170
:10A8C00083401C43014B5C6030BD00BF0000014071
:10A8D00001F003039B000F229A4010FA03F310B516
:10A8E0008908074C023154F8210020EA020244F89A
:10A8F000212054F82120134344F8213010BD00BF1B
:10A90000000001400120014608B500F047FB01208E
:10A91000002100F043FB08BD08B5264B98422BD020
:10A920000CD8A3F5006398421AD003F580639842CF
:10A930001CD0A3F5006398423AD10BE01E4B98421D
:10A9400026D003F58063984228D0A3F5006398428F
:10A950002ED117E00420012100F020FB042024E088
:10A960000820012100F01AFB08201EE01020012120
:10A9700000F014FB102018E02020012100F00EFB55
:10A98000202012E04020012100F008FB40200CE0D4
:10A990008020012100F002FB802006E04FF480704F
:10A9A000012100F0FBFA4FF48070002100F0F6FA6C
:10A9B00008BD00BF00140140001C01400B4B4FF0CC
:10A9C000FF316FF07042C3F88010C3F88420C3F8E1
:10A9D0008011C3F88421002303F1C001034A01332D
:10A9E00000200F2B42F82100F6D1704700E100E073
:10A9F000094B4FF020605860084800224FF0FF31AB
:10AA00009A60D8601A615A619A61DA611A625A6270
:10AA10009962D9621963704700ED00E00000FA0501
:10AA200040F0BE60024B40F42020D860704700BF69
:10AA300000ED00E030B5C27803787AB31C4A417863
:10AA4000D2684FF00F0CD243C2F302222CFA02FC60
:10AA5000C2F104029140807803F003020CEA000C7A
:10AA60004CEA010CD2004FEA0C1CFF2090400CFA7B
:10AA700002FC012403F01F02944099080D4AC031E2
:10AA800052F821500CEA000C25EA00004CEA0000C4
:10AA90005B0942F8210042F8234008E003F01F025E
:10AAA000012191405B09034A203342F8231030BD55
:10AAB00000ED00E000E100E00023C370037043708C
:10AAC00083707047024B5868C0F30930704700BF6D
:10AAD00000ED00E0012200F01F0312FA03F3400929
:10AAE000044A403052F820001840984214BF002019
:10AAF0000120704700E100E0014B1860704700BF83
:10AB000000EF00E000F01F0301229A404009024BD1
:10AB1000603043F82020704700E100E0024B5868A5
:10AB20008005800D704700BF00ED00E0012200F0BD
:10AB30001F0312FA03F34009044A803052F8200040
:10AB40001840984214BF00200120704700E100E047
:10AB5000014B1868704700BF00ED00E021F0604134
:10AB600021F07F01014B01439960704700ED00E047
:10AB7000014A024BDA6070470400FA0500ED00E07C
:10AB8000014A024BDA6070470100FA0500ED00E06F
:10AB900019B1054B1A69104303E0034B1A6922EA05
:10ABA00000001861704700BF00ED00E000F01F00DA
:10ABB000012313FA00F019B1044B5A6A104303E061
:10ABC000024B5A6A22EA00005862704700ED00E02A
:10ABD000144B70B5DC684FF0FF0CE443C4F302245F
:10ABE0002CFA04F5C4F1040411FA04F4C0F30126AC
:10ABF000F6000CFA06FC02EA050545EA0404240105
:10AC000014FA06F6C0F38110063053F8202022EA29
:10AC10000C0243F8202053F82020164343F820600C
:10AC200070BD00BF00ED00E0C0F38320012383402E
:10AC3000044A506A03EA0000984214BF0020012031
:10AC4000704700BF00ED00E000F01F0001228240CD
:10AC5000024B59680A435A60704700BF00ED00E09C
:10AC600000F01F020123013A13FA02F2024B596865
:10AC70000A435A60704700BF00ED00E0C0F3833024
:10AC800001238340044A506A03EA0000984214BF3B
:10AC900000200120704700BF00ED00E0C0F38143B9
:10ACA00013B90A4BD86A10E0012B0CD1074AC0F344
:10ACB0000153906ADA00D040022B14BF00F00F005D
:10ACC00000F0FF0001E0014B186B704700ED00E061
:10ACD00010F4800F0BBF024B014B586B986B704701
:10ACE00000ED00E008B5F9F743FA08BD08B500012A
:10ACF000F9F73BFA08BD00BF08B5F9F734FA08BD0B
:10AD000008B5F9F72EFA08BD08B5F9F728FA08BD15
:10AD100008B5F9F722FA08BD0D4B0E4A196841F043
:10AD200001011960596801EA02025A601A6822F0AA
:10AD3000847222F480321A601A6822F480221A6027
:10AD40005A6822F4FE025A6000229A60704700BFDF
:10AD5000001002400000FFF80C4BB0F5803F1A686D
:10AD600022F480321A601A6822F480221A6003D01A
:10AD7000B0F5802F08D103E01A6842F4803202E077
:10AD80001A6842F4A0221A60704700BF0010024007
:10AD9000034B1A6822F0F80242EAC0021A607047B8
:10ADA00000100240014B1860704700BF0000424293
:10ADB000044B5A6822F47C1240EA02020A435A60A9
:10ADC000704700BF00100240014B1860704700BF81
:10ADD00060004242034B5A6822F0030240EA02023A
:10ADE0005A60704700100240024B586800F00C0097
:10ADF000704700BF00100240034B5A6822F0F00277
:10AE000040EA02025A60704700100240034B5A6841
:10AE100022F4E06240EA02025A60704700100240E9
:10AE2000034B5A6822F4605242EAC0025A607047EB
:10AE30000010024019B1054B1A78104303E0034B90
:10AE40001A7822EA00001870704700BF091002400B
:10AE5000014B1860704700BFD8004242034B5A684C
:10AE600022F4404240EA02025A6070470010024059
:10AE7000064B002201281A701A7002D0042804D14F
:10AE800001E0187001E005221A707047201002409E
:10AE9000014B1860704700BF80044242024B1A6A9F
:10AEA00040EA02021A62704700100240014B18602B
:10AEB000704700BF3C0442421F4B10B55A6802F075
:10AEC0000C02042A13D0082A11D15A685968C2F317
:10AED0008342023211F4803F03D05B6813F4003FD9
:10AEE00001D0164B00E0164B5A43026001E0144BB0
:10AEF0000360114A134B51680468C1F30311595C94
:10AF000034FA01F141605468C4F3022C13F80C4088
:10AF100031FA04F484605468C4F3C22C13F80CC0F2
:10AF200021FA0CF1C1605268C2F381329B181B7C7C
:10AF3000B1FBF3F1016110BD0010024000093D00BA
:10AF400000127A008C03010819B1054B5A691043AD
:10AF500003E0034B5A6922EA00005861704700BFC2
:10AF60000010024019B1054B9A69104303E0034BEE
:10AF70009A6922EA00009861704700BF0010024001
:10AF800019B1054BDA69104303E0034BDA6922EA91
:10AF90000000D861704700BF0010024019B1054B96
:10AFA000DA68104303E0034BDA6822EA0000D86055
:10AFB000704700BF0010024019B1054B1A691043D9
:10AFC00003E0034B1A6922EA00001861704700BFD2
:10AFD00000100240014B1860704700BF400442421D
:10AFE000014B1860704700BF4C004242014B187083
:10AFF000704700BF071002404309012B02D1084BE4
:10B000001B6805E0022B0BBF054B054B1B6A5B6AF7
:10B0100000F01F0033FA00F000F00100704700BF9D
:10B020000010024008B53120FFF7E6FF094B187009
:10B030005A6801325A601A7822B95A6840F2FF13EE
:10B040009A42F0D13120FFF7D7FF003818BF012016
:10B0500008BD00BF1C040020024B5A6A42F08072F7
:10B060005A62704700100240034B9B6818420CBFA5
:10B0700000200120704700BF00100240014B1870F3
:10B08000704700BF0A1002400B884A88B1F804C01C
:10B090001A43CB8842EA0C02B1F808C01A434B8924
:10B0A00030B542EA0C028D89B0F800C0CC891A4351
:10B0B0002A4322430CF4415313439BB20380838BF6
:10B0C00023F400631B041B0C83830B8A038230BDB3
:10B0D00000234FF00702C3810282038043808380F4
:10B0E000C380038143818381704700BF0023438174
:10B0F000038043808380C3804FF002030381704745
:10B1000021B103889BB243F0400304E0038823F09D
:10B1100040031B041B0C0380704700BF21B1838BCD
:10B120009BB243F4806304E0838B23F480631B04AD
:10B130001B0C8383704700BF0909012313FA01F137
:10B1400089B21AB183889BB2194303E083889BB20A
:10B1500023EA0101818070471AB183889BB21943A9
:10B1600003E083889BB223EA01018180704700BF1E
:10B1700081817047808980B2704700BF4FF6FF63BE
:10B18000994205D003889BB243F48073038002E0A8
:10B19000038819400180704721B183889BB243F036
:10B1A000040304E0838823F004031B041B0C838046
:10B1B000704700BF038823F400631B041B0C03804B
:10B1C00003889BB241EA03030380704703889BB264
:10B1D00043F480530380704721B103889BB243F44A
:10B1E000005304E0038823F400531B041B0C03806A
:10B1F000704700BF012914BF008B808A80B270475E
:10B20000008A80B2704700BFB1F5804F04D1038837
:10B210009BB243F4804304E0038823F480431B047F
:10B220001B0C0380704700BF038919420CBF00202C
:10B2300001207047202906D1038903889BB243F07F
:10B240004003038008E0402901D0082901D1038987
:10B2500002E0C94389B20181704700BF012301F0B8
:10B260000F0213FA02F2B0F804C000891FFA8CFC36
:10B2700080B2104006D009098B401CEA030F0CBFB6
:10B2800000200120704700BF552906D1038903889B
:10B290009BB243F0400303800DE0562901D05329AF
:10B2A00001D1038907E001F00F01012313FA01F135
:10B2B000C94389B201817047838BF0B523F47A6367
:10B2C00023F01F031B041B0C83834FF00203038432
:10B2D0000B89868B022B87B004460D46B6B201D18E
:10B2E000002225E001A88F88FFF7E6FDEB88002FFC
:10B2F0000CBF01270227B3F5007F2989019A06D1E7
:10B30000A3F5FB7353430902B3FBF1F305E00A23F2
:10B3100049015A434F43B2FBF7F305330A229BB26C
:10B32000B3FBF2F303F001021202C3F34F0392B234
:10B33000991E89B2FE2928BF002228BF0223E9886E
:10B3400042EA03030B439BB223842B886A8846EAB4
:10B350000303A98843F4006313436A890B4313432F
:10B360009BB2A38307B0F0BD08B5154B98421BD024
:10B3700003F57443984204D0A3F5784398421DD155
:10B380000AE001214FF48050FFF708FE4FF480508F
:10B390000021FFF703FE11E04FF480400121FFF789
:10B3A0000BFE4FF4804006E04FF400400121FFF710
:10B3B00003FE4FF400400021FFF7FEFD08BD00BF73
:10B3C000003C0040042804D1054B1A6842F00402F6
:10B3D00003E0034B1A6822F004021A60704700BFB2
:10B3E00010E000E0014B5860704700BF10E000E043
:10B3F000012804D1084B1A6842F0010206E010F15E
:10B40000020F05D1044B1A6822F001021A6002E013
:10B41000014B00229A60704710E000E020B1054B1C
:10B420001A6842F0020203E0024B1A6822F002029C
:10B430001A60704710E000E0014B9868704700BF49
:10B4400010E000E0C308022B0BBF044B034B1B684A
:10B45000DB6833FA00F000F00100704710E000E014
:10B46000038803F08F0303800388B1F806C04A887D
:10B470009BB243EA0C0313439BB203808B88838502
:10B480000B880385064B984203D003F5006398426E
:10B4900001D10B7A03864FF001038382704700BF0E
:10B4A000002C0140038C2DE9F04123F001031B0423
:10B4B0001B0C0384038C0A894C8823F002031C4E66
:10B4C00014431B048288B1F806C0058B1B0CA4B280
:10B4D000B04244EA030392B20C88ADB2A0F834C083
:10B4E00003D006F50066B04218D18E894F89B1F8B5
:10B4F0000E804FF6F77C03EA0C0C4CEA070748EA8B
:10B5000006064FF6FB73898847F6FF4C02EA0C0CDF
:10B5100007EA0303B2B20B4342EA0C024FF68F7103
:10B5200005EA01012143828001830384BDE8F081A3
:10B53000002C0140038C2DE9F04123F010031B0483
:10B540001B0C0384028CB1F808C022F02002120404
:10B550008488120C4B8842EA0C1242EA0313A2B20E
:10B560001B4C068BB1F806C0A0420D88B6B29BB248
:10B57000A0F838C003D004F50064A0421BD1B1F894
:10B580000A804FF67F748F8903EA040447F2FF3C78
:10B5900002EA0C0C44EA0814CA894FF6BF73898882
:10B5A00004EA03034CEA870C43EA01134CEA8202E3
:10B5B0003C469BB292B248F6FF7106EA010141EAAD
:10B5C000052189B2828001830384BDE8F08100BF38
:10B5D000002C0140038C2DE9F04123F480731B04FF
:10B5E0001B0C0384028CB1F808C022F40072120410
:10B5F0008488120C4B8842EA0C2242EA0323A2B24E
:10B600001A4C868BB1F806C0A0420D88B6B29BB228
:10B61000A0F83CC003D004F50064A0421BD1B1F8EF
:10B620000A804FF2FF748F8903EA040444F6FF7C1A
:10B6300002EA0C0C44EA0824CA894FF6FF338988D1
:10B6400004EA03034CEA071C43EA01234CEA021212
:10B650003C469BB292B24FF68F7106EA0101294334
:10B66000828081830384BDE8F08100BF002C01400B
:10B67000038CF0B523F480531B041B0C0384B1F836
:10B6800006C0078C0C8882880D89868B4B88A0F8B1
:10B6900040C0DFF848C0BFB2604592B2B6B203D036
:10B6A0000CF5006C604505D192048989920C42EA40
:10B6B000811292B24DF6FF7C07EA0C0C48F6FF713E
:10B6C00006EA01014CEA053C41EA04214CEA033355
:10B6D00089B29BB2828081830384F0BD002C01403B
:10B6E000B1F802C00B888A884CEA0303B1F806C09F
:10B6F00013430A8943EA0C03B1F80AC013438A8949
:10B7000043EA0C0313439BB2A0F84430704700BFD8
:10B7100000234FF0FF320372438082800380C38096
:10B72000704700BF0023C381038043808380C380B0
:10B73000038143818381704700234FF0010203811D
:10B74000038043808280C380704700BF00238381D1
:10B75000038043808380C38003814381704700BF9F
:10B7600021B103889BB243F0010304E0038823F076
:10B7700001039B059B0D0380704700BF39B1B0F8F2
:10B7800044306FEA43436FEA53439BB203E0B0F89F
:10B7900044305B045B0CA0F8443070471AB18389D5
:10B7A0009BB2194303E083899BB223EA01018181A3
:10B7B000704700BF818270470A43A0F84820704755
:10B7C0001AB183899BB2194303E083899BB223EAB0
:10B7D00001018181704700BF038923F007031B0427
:10B7E0001B0C0381704700BFB0F808C05FFA8CFCE7
:10B7F00041EA0C0C42EA0C0C4CEA032C1FFA8CFCBC
:10B80000A0F808C0704700BF10B50446FFF7ECFF72
:10B8100023899BB243F48043238110BD10B50446B5
:10B82000FFF7E2FF238923F077031B041B0C43F08F
:10B830007703238110BD00BF01858282704700BF5E
:10B84000038823F070039B059B0D41EA03030380EB
:10B85000704700BF038923F070031B041B0C41EAEF
:10B8600003030381704700BF10B50446FFF7F2FFE2
:10B8700023899BB243F00703238110BD30B50489AF
:10B88000B0F818C0058C2CF4407CADB22CF0030C41
:10B8900024F007044FEA0C4C25F0220542EA050586
:10B8A00024044FEA1C4C45EA0315240C4CF4807C1C
:10B8B00021434CF0010CADB20181A0F818C0058401
:10B8C00030BD00BF038B23F070031B041B0C41EA47
:10B8D00003030383704700BF038B23F4E0431B047F
:10B8E0001B0C43EA01239BB203837047838B23F035
:10B8F00070031B041B0C41EA03038383704700BFE2
:10B90000838B23F4E0431B041B0C43EA01239BB20B
:10B910008383704721B103889BB243F0800304E026
:10B92000038823F080039B059B0D0380704700BFB5
:10B9300021B183889BB243F0040304E0838823F0A1
:10B9400004031B041B0C8380704700BF21B1838854
:10B950009BB243F0080304E0838823F008031B0430
:10B960001B0C8380704700BF21B183889BB243F0DA
:10B97000010304E0838823F001031B041B0C838074
:10B98000704700BF038B23F008031B041B0C41EA24
:10B9900003030383704700BF038B23F400631B047E
:10B9A0001B0C43EA01239BB203837047838B23F074
:10B9B00008031B041B0C41EA03038383704700BF89
:10B9C000838B23F400631B041B0C43EA01239BB20B
:10B9D00083837047038B23F004031B041B0C41EA91
:10B9E00003030383704700BF038B23F480631B04AE
:10B9F0001B0C43EA01239BB203837047838B23F024
:10BA000004031B041B0C41EA03038383704700BF3C
:10BA1000838B23F480631B041B0C43EA01239BB23A
:10BA200083837047038B23F080031B041B0C41EAC4
:10BA300003030383704700BF038B5B045B0C43EA83
:10BA400001239BB203837047838B23F080031B0485
:10BA50001B0C41EA03038383704700BF838B5B04A5
:10BA60005B0C43EA01239BB283837047038C23F072
:10BA700002031B041B0C41EA03030384704700BF4D
:10BA8000038C23F008031B041B0C41EA030303840B
:10BA9000704700BF038C23F020031B041B0C43EAF8
:10BAA00001139BB203847047038C23F080031B04B3
:10BAB0001B0C43EA01139BB203847047038C23F4ED
:10BAC00000731B041B0C43EA01239BB203847047E1
:10BAD000038C23F400631B041B0C43EA01239BB279
:10BAE00003847047038C23F400531B041B0C43EAAC
:10BAF00001339BB20384704701238B408A40018C41
:10BB000089B221EA03030384018C0A4392B20284BE
:10BB1000704700BF04238B408A40018C89B221EA20
:10BB200003030384018C0A4392B20284704700BF6E
:10BB300001238B40B0F820C010B51FFA8CFC2CEA12
:10BB40000303038409B1082909D11830490844586E
:10BB50004FF68F7304EA0303435043580CE0043953
:10BB60001830C1F34E01445848F6FF7304EA03034A
:10BB700043501202435892B243EA0202425010BDAF
:10BB800021B103889BB243F0020304E0038823F051
:10BB900002039B059B0D0380704700BF21B1038802
:10BBA0009BB243F0040304E0038823F004039B05E5
:10BBB0009B0D0380704700BF21B183889BB243F087
:10BBC000800304E0838823F080031B041B0C838024
:10BBD000704700BF038823F008039B059B0D03807B
:10BBE00003889BB241EA030303807047838823F0F4
:10BBF00070031B041B0C838083889BB241EA030300
:10BC000083807047038923F007031B041B0C038107
:10BC100003899BB241EA030303817047038923F040
:10BC200080031B041B0C038103899BB241EA0303BD
:10BC30000381704781847047818570478186704792
:10BC40000187704781877047A0F84010704700BF98
:10BC5000038B23F00C031B041B0C0383038B9BB28D
:10BC600041EA030303837047038B23F440631B04FF
:10BC70001B0C0383038B9BB243EA01239BB2038318
:10BC8000704700BF838B23F00C031B041B0C8383C2
:10BC9000838B9BB241EA030383837047838B23F436
:10BCA00040631B041B0C8383838B9BB243EA0123F9
:10BCB0009BB28383704700BF0388DBB20380038895
:10BCC0009BB241EA03030380704700BF808E80B2BD
:10BCD000704700BF008F80B2704700BF808F80B276
:10BCE000704700BFB0F8400080B27047808C80B2CF
:10BCF000704700BF008D80B2704700BF038A1942B1
:10BD00000CBF002001207047C94389B201827047EF
:10BD1000038A828911EA030092B203D011420CBF58
:10BD200000200120704700BFC94389B201827047DB
:10BD3000B0F820C010B52CF0010C4FEA0C4C4FEAC3
:10BD40001C4CA0F820C0048BB0F820C0A4B21FFA8D
:10BD50008CFC24F0F30442EA04042CF0020C44EAC4
:10BD600003144CF0010C4CEA010CA4B20483A0F8BB
:10BD700020C010BDB0F820C010B52CF0100C4FEA58
:10BD80000C4C4FEA1C4CA0F820C0B0F818C0048C32
:10BD90002CF4407CA4B24FEA0C5C4FEA1C5C24F00B
:10BDA00020044CEA022C44F010044CEA033C44EA20
:10BDB00001141FFA8CFCA4B2A0F818C0048410BDB2
:10BDC00038B50D46602D1146044603D10122FFF718
:10BDD000D1FF02E00122FFF7ABFF29462046FFF723
:10BDE00039FD23899BB243F00703238138BD00BF8F
:10BDF000F8B50C46A2884988B4F800C00546002969
:10BE00000CBF02270027012A0CBF02260126238926
:10BE1000BCF1000F10D1FFF78BFF2846E188FFF738
:10BE200017FF2846394632462389FFF7A3FF2846E5
:10BE3000E188FFF719FF0FE0FFF79CFF2846E18834
:10BE4000FFF712FF2846394632462389FFF770FF75
:10BE50002846E188FFF7FCFEF8BD00BF38B50B8827
:10BE60000C4605464BB94988A2882389FFF760FF35
:10BE70002846E188FFF7ECFE53E0042B09D14988FE
:10BE8000A2882389FFF776FF2846E188FFF7ECFEBA
:10BE900047E0082BB1F802C0B1F804E0098920D1CD
:10BEA000028C22F480721204120C0284838B028CA6
:10BEB0009BB292B223F0F30322F4007243EA011121
:10BEC00042EA0C2C89B21FFA8CFC41EA0E0E4CF4AB
:10BED000807CA0F81CE0A0F820C0E188FFF7D2FE2B
:10BEE0001FE0028C22F480521204120C0284838B15
:10BEF000028C23F4407392B21B051B0D22F40052F6
:10BF000043EA0E2342EA0C3C43EA01331FFA8CFC5D
:10BF10009BB24CF4805C8383A0F820C0E188FFF7DB
:10BF2000BDFE38BD08B52D4B984237D00BD8A3F5D0
:10BF30000063984226D003F58063984228D0B0F180
:10BF4000804F4AD118E0264B984233D004D8A3F54D
:10BF50008063984241D127E0224B984204D003F5F8
:10BF60000063984239D12EE04FF400600121FFF7C1
:10BF700015F84FF400602DE001200146FFF71CF892
:10BF800001201CE002200121FFF716F8022016E034
:10BF900004200121FFF710F8042010E008200121FF
:10BFA000FFF70AF808200AE010200121FFF704F843
:10BFB000102004E020200121FEF7FEFF20200021B8
:10BFC000FEF7FAFF09E04FF400500121FEF7E6FF0B
:10BFD0004FF400500021FEF7E1FF08BD000C0040C7
:10BFE00000140040002C0140002383814FF41652BE
:10BFF0008380C38003814FF00C030260438170474C
:10C000000A8810B54C88B1F804C0038AC98844EA8C
:10C01000020242EA0C0223F470630A431B041B0C65
:10C0200092B242EA0303038210BD00BF0023C38023
:10C03000038043808380704721B183899BB243F49E
:10C04000005304E0838923F400531B041B0C8381F9
:10C05000704700BF01F01F034FF0010CC1F3421104
:10C0600061450CFA03F301D10C3004E0022901D13F
:10C07000103000E014301AB1026842EA030302E013
:10C08000026822EA03030360704700BF1AB1838A83
:10C090009BB2194303E0838A9BB223EA01018182A8
:10C0A000704700BF038A23F00F031B041B0C03829D
:10C0B000038A9BB241EA030303827047838923F416
:10C0C00000631B041B0C838183899BB241EA030339
:10C0D0008381704721B183899BB243F0020304E05E
:10C0E000838923F002031B041B0C8381704700BF6C
:10C0F000038A23F020031B041B0C0382038A9BB2D8
:10C1000041EA03030382704721B1038A9BB243F4DF
:10C11000804304E0038A23F480431B041B0C038246
:10C12000704700BFC905C90D818070478088C00570
:10C13000C00D704783899BB243F001038381704730
:10C14000038BDBB20383038B9BB243EA012303839C
:10C15000704700BF038B03F47F430383038B9BB2C1
:10C1600041EA03030383704721B1838A9BB243F002
:10C17000200304E0838A23F020031B041B0C83822A
:10C18000704700BF21B1838A9BB243F0100304E0E3
:10C19000838A23F010031B041B0C8382704700BFAB
:10C1A00021B1838A9BB243F0080304E0838A23F021
:10C1B00008031B041B0C8382704700BF838A23F093
:10C1C00004031B041B0C8382838A9BB241EA030392
:10C1D0008382704721B1838A9BB243F0020304E05B
:10C1E000838A23F002031B041B0C8382704700BF69
:10C1F000038819420CBF002001207047C94389B24F
:10C20000018070474FF0010CC1F3421201F01F038F
:10C2100062450CFA03F301D1828903E0022A0CBFC4
:10C22000028A828A92B21340028892B20BB91846EF
:10C2300007E0090A012313FA01F111420CBF0020A3
:10C2400001207047090A01238B40DB439BB2038026
:10C25000704700BF038ACA8823F440531B041B0C99
:10C260001343038283898A8830B5044608890D46C2
:10C2700023F4B053498940EA020223F00C030A4335
:10C280001B041B0C92B242EA0303A381A38AAA896E
:10C2900023F440731B041B0C134387B0A38201A833
:10C2A000FEF70AFE0E4B2A689C420CBF049B039BC0
:10C2B0001921594392006423B1FBF2F1B1FBF3F26F
:10C2C0001201100903FB101109013231B1FBF3F324
:10C2D00003F00F0343EA020292B2228107B030BD9D
:10C2E0000038014008B5214B98422BD008D8A3F55F
:10C2F0000063984216D003F58063984234D119E068
:10C300001B4B984226D003F5684398422CD101215B
:10C310004FF48040FEF742FE4FF480400021FEF7CC
:10C320003DFE21E04FF400300121FEF745FE4FF4C1
:10C33000003016E04FF480200121FEF73DFE4FF45F
:10C3400080200EE04FF400200121FEF735FE4FF46F
:10C35000002006E04FF480100121FEF72DFE4FF47F
:10C3600080100021FEF728FE08BD00BF004C0040F1
:10C3700000500040684620F007018D4601B50023BB
:10C3800003E00B495958995004330A4A0A4998184E
:10C390008842F6D3094B02E0002243F8042B084AF6
:10C3A0009342F9D3F7F7ECFEBDE8014085467047AC
:10C3B000AC09010800000020640200206402002093
:10C3C000E40C002010B5074C20B922684FF001039F
:10C3D000138205E0044B1B681B68984720680A30ED
:10C3E00010BD00BFB80A0020740A002010B50A4B27
:10C3F0000A4A1B685178DA7891420AD3997841B990
:10C400009C8834B99A72064B1B685B689847204633
:10C4100000E0022010BD00BFB80A00203402002056
:10C42000740A002010B5074C20B922684FF00103B0
:10C43000138205E0044B1B689B68984720680C300A
:10C4400010BD00BFB80A0020740A002038B50E4C99
:10C450000E4B22681B68D1789B69507998472368F6
:10C460009A7A7AB170B91A7962B99D7855B9084B40
:10C470001B68DB689847236828465979DA78D972AF
:10C480001A7300E0022038BDB80A0020500A0020CC
:10C49000740A002008B50246244B20B91B684FF0EF
:10C4A0000201198240E0224A4FF000011B6811800E
:10C4B000197811F07F0113D15B7A13F0200F03D0AC
:10C4C000117841F00201117013F0400F184B15BFA5
:10C4D0001A781A7822F0010242F001021A701EE066
:10C4E000012921D0022901D000221DE0597911F043
:10C4F000800F01F00F0306D00E4951F8233003F0EE
:10C500003003102B06E00B4951F8233003F440535D
:10C51000B3F5805F03D1137843F001031370064B2A
:10C520001B681B699847024A104608BDB80A0020DC
:10C53000040B0020005C0040740A002010B51E4B64
:10C5400019684A7912F0800F22F0800305D01B4849
:10C5500050F8230000F0300004E0184850F82300A1
:10C5600000F44050164C94F800C0634522D24C8829
:10C5700004BBF8B1897AE9B112F0800F09D00F49F4
:10C5800048F6BF7251F8230000EA020282F010025E
:10C5900008E00A494BF68F7251F8230000EA0202C4
:10C5A00082F4805241F82320064B1B689B69984710
:10C5B000002000E0022010BDB80A0020005C00400E
:10C5C00034020020740A002008B5064B1B685A7A12
:10C5D00042F020025A72044B1B68DB699847002026
:10C5E00008BD00BFB80A0020740A0020054B1A6875
:10C5F000538A18B98988CB1A138201E00868181881
:10C60000704700BFB80A002030B50E4B1C780023DD
:10C6100010E05FFA83FC4FEA8C0202F1804202F5DF
:10C62000B842156848F68F7105EA010141EA0C012C
:10C6300011600133A342ECD3034B40F0800018603B
:10C6400030BD00BF340200204C5C0040704700BF8A
:10C6500008B50C4B002093F82C1000F04FFE0A4B4D
:10C660001B68187A082807D1084B4FF480521A80AB
:10C67000074B4FF010021A80092814BF0020012038
:10C6800008BD00BFB0010020B80A0020060B002042
:10C69000080B002070B52D4B1C68237A032B01D0AA
:10C6A000052B46D1A369228AABB1A2B1A58A9542D6
:10C6B00028BF154628469847228A638A521BEB18E2
:10C6C000064622826382002000F0E8FD2A460146E9
:10C6D000304600F0FBFB238A5BB11D4B4FF4405208
:10C6E00000201A80014600F0E7FD1A4B4FF030029F
:10C6F0001A80A28A238A9A4203D8144B03221B6809
:10C7000003E0124A1BB1136805221A720DE0126889
:10C7100006211172104A1168104A89B28A18520013
:10C7200013600C4B4FF030021A80084B1B681B7AC9
:10C7300006E0072B03D10A4B1B68DB6898470823E8
:10C74000024A12681372FFF783FF70BDB80A002017
:10C75000060B0020080B0020505C00400230002037
:10C76000500A0020F8B5244B1C68238A267ABBB9EE
:10C77000042E15D1214822490278012A0BD1214CDF
:10C78000214A24680370A0B28218520013604FF04F
:10C7900030020A802BE04FF010030B80072626E0C2
:10C7A000A68AA2699E4234BF35461D462846B3423A
:10C7B00094BF0426022690470746002000F060FD43
:10C7C0002A460146384600F069FB2946002000F061
:10C7D00073FD638A228AEB186382094B551B4FF065
:10C7E000300225821A80094B4FF440521A80024BC6
:10C7F0001B681E72F8BD00BFB80A00202404002088
:10C80000080B0020505C004002300020060B002086
:10C8100008B5144B1B681A7A022A01D0042A05D1E4
:10C82000FFF7A0FF0F4B1B681B7A14E0062A11D1FB
:10C830005A78052A0AD11A7812F07F0F06D1D878D3
:10C84000FFF7E2FE084B1B681B6A9847074B1B6803
:10C850009B6898470823034A12681372FFF7F8FE93
:10C8600008BD00BFB80A0020740A0020500A00204A
:10C8700038B5324B1B68187810F07F0004D15A7A13
:10C8800022F020025A7258E0022855D15A88002A14
:10C8900052D11A79002A4FD15A7912F0800F22F022
:10C8A000800405D0264951F8241001F0300104E03D
:10C8B000234951F8241001F4405122480078844261
:10C8C0003AD2002938D09B7A002B35D012F0800F55
:10C8D0000FD01B4B53F8243003F03003102B25D11D
:10C8E000E4B2204600F082FC2046302100F05EFBDE
:10C8F0001CE0134D55F8243003F44053B3F5805F2A
:10C9000014D134B9104B204693F82C1000F0F6FCEB
:10C9100002E0204600F056FC55F824204BF68F73B9
:10C9200002EA030383F4405345F82430074B1B68A5
:10C930005B699847002000E0022038BDB80A00205B
:10C94000005C004034020020B0010020740A002086
:10C95000F7B58D4B8D4E1A6835688D4B92B2D31852
:10C960002A7A5B00092A1B681BD09BB203F1005393
:10C9700003F540535B001C4614F8012B03F10A0732
:10C980002A705B786B70B4F8030000F063FE688077
:10C99000B4F80700346800F05DFEA08033687F883B
:10C9A000DF807A4C01212368DA8819725D78002AC9
:10C9B00062D11A7812F07F022ED1092D02D1FFF731
:10C9C00015FD3BE0052D0DD193F90320002A4EDB28
:10C9D0009A78002A4BD19A88002A48D19B7A002B5A
:10C9E00037D044E0032D0BD1DA78012A27D19A8879
:10C9F0002ABB5B7A13F0200F21D0FFF7E5FD1DE085
:10CA0000012D1CD1DA78012A19D19A88BAB95B7A3A
:10CA100013F0200F13D00AE0012A04D10B2D0ED100
:10CA2000FFF714FD0AE0022A09D1012D02D1FFF718
:10CA30001FFF03E0032D02D1FFF780FD48B1554BE6
:10CA400028461B685B699847032801D109230FE03A
:10CA500068B94D4A504B12684FF0300192B2D3186A
:10CA60005B0000221A604D4B1980062300E008236A
:10CA7000464A12681372E3E0062D18D11A7812F0B4
:10CA80007F0F40F097809B78012B03D1414B1B68AF
:10CA9000DB696EE0022B03D13E4B1B681B6A68E02A
:10CAA000032B40F087803B4B1B685B6A61E0002DE5
:10CAB0003CD1598800297DD15A6822F47F42B2F5D1
:10CAC000003F77D11A7812F07F0203D19B88002BA8
:10CAD00070D129E0012A0BD158792E4B1B689B6934
:10CAE0009847002866D123689B7A002B62D01BE010
:10CAF000022A5FD15B7913F0800F03F00F0205D09B
:10CB0000274951F8221001F0300104E0244951F87E
:10CB1000221001F440512348007882424AD213F097
:10CB2000700F47D1002945D01F4B23E0082D05D1B8
:10CB30001B7813F07F0F3DD11C4B1BE00A2D39D120
:10CB40001A7802F07F02012A34D19A7A002A31D071
:10CB5000598800292ED15A6822F47F42B2F5803FCD
:10CB600028D158790B4B1B689B69984710BB104B19
:10CB700000E0FBB1054A4FF000011268002093610C
:10CB800051829847002020E0505C0040B80A002005
:10CB900004300020500A002002300020080B002042
:10CBA000005C00403402002095C40008C5C30008A2
:10CBB00025C40008244C254B22681B6850781B694B
:10CBC0009847032801D1236806E01F4B4FF6FF71F9
:10CBD0001B681A8A8A4201D1092203E0022800D088
:10CBE00012B908221A722BE093F90010002921DAF9
:10CBF000D98801910198824202D9019A1A8211E0E2
:10CC00008A420FD21149096891F82C108A4201D248
:10CC1000002105E092FBF1F001FB102212B9012185
:10CC20000B4A1170094A126892F82C209A82FFF779
:10CC300099FD05E003221A72064B4FF440521A8008
:10CC4000FFF706FDFEBD00BFB80A0020500A002015
:10CC500024040020060B0020074A022108B50748DB
:10CC600011720749074B086007490A60074A1360B9
:10CC70001B68984708BD00BF580A002038020020F2
:10CC8000740A0020B0010020B80A0020500A0020D9
:10CC900008B529E047F6FF700860198801F00F0118
:10CCA0008B0003F18043117003F5B843196889B212
:10CCB00011F4004F09D0186840F68F7100EA0101A5
:10CCC000196012780E4B013A0BE011F0800F0BD077
:10CCD000186848F60F7100EA010119601278094BD3
:10CCE000013A53F8223098470749084B0868084A28
:10CCF00080B21880188800B20028CBDB08BD00BFC6
:10CD000018020020FC010020445C00404E0A002074
:10CD1000540A0020F8B59AE047F6FF761E601688A0
:10CD2000564F06F00F06B30003F1804303F5B843F6
:10CD30003E70002E64D127682668236807F4405CA3
:10CD400003EA000080F400502060236806F0300001
:10CD500003EA010181F0200121601388484A13F0A1
:10CD6000100F1080A5F800C004D023689BB213F008
:10CD7000800F08D0226848F60F7302EA030323608D
:10CD8000FFF746FD16E013F4006F08D0226840F666
:10CD90008F7302EA03032360FFF7DAFD0AE013F45E
:10CDA000004F54D0226840F68F7302EA03032360D9
:10CDB000FFF770FC21682A884BF68F7301EA0303A2
:10CDC00012F4805F18BF83F4805312F4005F2D4A81
:10CDD00018BF83F400531360294B11681A8848F672
:10CDE000BF7301EA030312F0100F18BF83F01003A2
:10CDF00012F0200F234A18BF83F0200313603BE09A
:10CE00001C68A4B214F4004F0BD0196840F68F725E
:10CE100001EA02021A603A781B4B013A53F82230B9
:10CE2000984714F0800F12D0144948F60F720B780F
:10CE30009B0003F1804303F5B843186800EA02023F
:10CE40001A600A78114B013A53F822309847104B78
:10CE5000104A1D680B4C1FFA85FCA2F800C0B2F8FE
:10CE600000C04BF68F700FFA8CFCBCF1000F48F637
:10CE7000BF71094DFFF650AFF8BD00BF540A002046
:10CE8000080B0020005C004018020020FC0100207C
:10CE9000445C00404E0A0020060B002001F10051C6
:10CEA000013201F5405110B549005208002308E055
:10CEB00010F803C06478013A4CEA042C21F813C03E
:10CEC0000233C418002AF3D110BD00BF01F1005194
:10CED000013201F5405110B549005208002304E029
:10CEE00031F81340013AC4520233002AF8D110BD80
:10CEF000014B1860704700BF405C0040014B186850
:10CF000080B27047405C0040014B1860704700BF22
:10CF1000445C0040014B186880B27047445C00409C
:10CF2000014B186880B27047485C0040014B1860A4
:10CF3000704700BF4C5C0040014B186880B27047DE
:10CF40004C5C00404FF6F873024A00EA030313609A
:10CF5000704700BF505C0040014B186880B27047BA
:10CF6000505C0040014B43F820107047005C0040CB
:10CF7000024B53F8200080B2704700BF005C0040B5
:10CF8000054B10B553F8204048F68F1204EA020210
:10CF90000A4343F8202010BD005C0040024B53F8C8
:10CFA000200000F4C0607047005C00400A4B10B5E0
:10CFB00053F8202048F6BF7402EA040411F0100F61
:10CFC00018BF84F0100411F0200F18BF84F0200463
:10CFD00043F8204010BD00BF005C00400A4B10B574
:10CFE00053F820204BF68F7402EA040411F4805F9A
:10CFF00018BF84F4805411F4005F18BF84F4005407
:10D0000043F8204010BD00BF005C004038B50D461D
:10D010000446FFF7ADFF012D02D120F4805003E05C
:10D02000022D04D120F01000014B43F8240038BD3C
:10D03000005C0040024B53F8200000F030007047C5
:10D04000005C0040024B53F8200000F44050704751
:10D05000005C0040054B48F6BF7253F8201001EA0F
:10D06000020282F0300243F820207047005C00404A
:10D07000054B4BF68F7253F8201001EA020282F43E
:10D08000405243F820207047005C0040054B48F6B2
:10D090008F6253F8201001EA020242F4807243F8D2
:10D0A00020207047005C0040044B48F68F6253F824
:10D0B000201001EA020243F820207047005C004083
:10D0C000044B48F68F6253F8201001EA020243F83D
:10D0D00020207047005C0040054B48F68F6253F8F3
:10D0E000201001EA020242F4807243F820207047C7
:10D0F000005C0040054B48F68F6253F8201001EAAF
:10D10000020242F4807243F820207047005C004025
:10D11000044B48F68F6253F8201001EA020243F8EC
:10D1200020207047005C0040044B53F8200000F0C2
:10D130003000102814BF002001207047005C004020
:10D14000054B53F8200000F44050B0F5805F14BF49
:10D1500000200120704700BF005C0040044B40F6F7
:10D160008F7253F8201001EA020243F82020704722
:10D17000005C0040044B48F60F7253F8201001EA9F
:10D18000020243F820207047005C0040054B48F63F
:10D190008F7253F8201001EA020242F4804243F8F1
:10D1A00020207047005C0040054B48F68F7253F812
:10D1B000201001EA020242F0400243F820207047AA
:10D1C000005C0040084B53F8202012F4804F09D037
:10D1D00053F8201048F68F7201EA020242F48042AE
:10D1E00043F82020704700BF005C0040084B53F814
:10D1F000202012F0400F09D053F8201048F68F720B
:10D2000001EA020242F0400243F82020704700BFCA
:10D21000005C0040054B10B553F8204048F68F7273
:10D2200004EA02020A4343F8202010BD005C0040DB
:10D23000024B53F8200000F00F007047005C0040E4
:10D24000064B49081B6849009BB203EBC00303F17E
:10D25000005303F540535B0019607047505C004079
:10D26000054A064B1268490892B202EBC002D31875
:10D270005B00490019607047505C0040043000209A
:10D28000054B1B689BB203EBC00303F1005303F58E
:10D2900040535B0018887047505C0040044A054BBF
:10D2A000126892B202EBC002D3185B001888704774
:10D2B000505C004004300020044A054B126892B2D2
:10D2C00002EBC002D3185B0019607047505C00404D
:10D2D000023000203E2909D94B0911F01F0F01D15E
:10D2E000013B9BB29B0243F4004305E04B0811F065
:10D2F000010F18BF01339B02036070470D4A0E4BAC
:10D30000126892B2D31803EBC0035B003E2909D91F
:10D310004A0911F01F0F01D1013A92B2920242F470
:10D32000004205E04A0811F0010F18BF01329202D5
:10D330001A607047505C004006300020054A064BDA
:10D34000126892B202EBC002D3185B001868800525
:10D35000800D7047505C004002300020054A064BAB
:10D36000126892B202EBC002D3185B001868800505
:10D37000800D7047505C0040063000200C4B30B5EB
:10D380001D681C68C0001FFA85FC8444A4B2094BC8
:10D3900000190CF1005CC3180CF5405C49085208F8
:10D3A0004FEA4C0049005B00520001601A6030BD3A
:10D3B000505C004004300020064B49081B684900BF
:10D3C0009BB203EBC00303F1005303F540535B0032
:10D3D00019607047505C0040054A064B12684908C6
:10D3E00092B202EBC002D3185B004900196070478B
:10D3F000505C004004300020054B1B689BB203EBDF
:10D40000C00303F1005303F540535B0018887047D5
:10D41000505C0040044A054B126892B202EBC00215
:10D42000D3185B0018887047505C0040043000201F
:10D43000012910B524D1254B25491B68C0009BB29A
:10D44000591809184B003E2A09D9510912F01F0F2B
:10D4500001D1013989B2890241F4004105E0510846
:10D4600012F0010F18BF0131890219601749194BD9
:10D47000096889B2CB18181840003E2A1ED913E05B
:10D48000022922D1114BC0001C681B68A4B21FFAEC
:10D4900083FC0F490F4B8444001941186344490031
:10D4A0005B000A601A6010E0530912F01F0F01D1EF
:10D4B000013B9BB29B0243F4004305E0530812F08A
:10D4C000010F18BF01339B02036010BD505C004088
:10D4D000023000200630002001291BD11349144BD3
:10D4E000096889B2CB1803EBC00040003E2A09D975
:10D4F000530912F01F0F01D1013B9BB29B0243F471
:10D50000004305E0530812F0010F18BF01339B02DE
:10D5100003600AE0022908D10449054B096889B271
:10D5200001EBC000C3185B001A607047505C0040FC
:10D530000230002001291BD11349144B096889B21C
:10D54000CB1803EBC00040003E2A09D9530912F062
:10D550001F0F01D1013B9BB29B0243F4004305E046
:10D56000530812F0010F18BF01339B0203600AE059
:10D57000022908D10449054B096889B201EBC000B2
:10D58000C3185B001A607047505C004006300020F2
:10D59000054A064B126892B202EBC002D3185B0038
:10D5A00018688005800D7047505C004002300020F4
:10D5B000054A064B126892B202EBC002D3185B0018
:10D5C00018688005800D7047505C004006300020D0
:10D5D0000D4BC00019680D4A89B241188A185200D3
:10D5E000128812F47C4F01D001200CE01A68084B1D
:10D5F00092B28018C3185B0018888005800D00283F
:10D6000014BF022000207047505C0040063000200C
:10D6100002300020012909D10B4A48F68F7352F8D5
:10D62000201001EA030343F040030AE002290AD173
:10D63000054A48F68F7352F8201001EA030343F4B9
:10D64000804342F820307047005C004041EA0020EF
:10D65000704700BF030AC0B243EA0020704700BF12
:10D6600003464FF6FF7083424EDDB3F1807F27DB28
:10D67000B3F1805F11DBB3F1804F08DB3A4A93428C
:10D6800070DC3A4A191652F82120120212E0374A89
:10D69000991552F82120D2010CE0B3F1806F334A82
:10D6A00004DB191552F82120920103E0991452F875
:10D6B0002120520193FBF2F10132521852101DE069
:10D6C000B3F5801F0DDBB3F5800F284A04DB191476
:10D6D00052F82120120111E0991352F82120D200B2
:10D6E0000CE0B3F5802F214A04DB191352F82120F6
:10D6F000920003E0991252F82120520093FBF2F1BC
:10D70000501C401840101FE0FF2B23DDB3F5805F55
:10D710000CDBB3F5804F154A03DB191252F82100D8
:10D7200011E0991152F8210040100CE0B3F5806F20
:10D730000E4A04DB191152F82100801003E0991001
:10D7400052F82100C010013000FB00F29A4209DDBE
:10D75000013807E0002BA9BF044A4FF0FF3052F810
:10D7600023000011704700BF0080FE7FA003010866
:10D77000B0F5806F01D3002025E0FF2805D9B0F572
:10D78000007F08D2C0F5FE700330104B03EB400061
:10D79000B0F800340FE0B0F5407F0C4A02D232F806
:10D7A000103006E0C0F57E70073002EB4000B0F8A4
:10D7B00000345B429BB21BB201FB03F04FF6FE72DA
:10D7C00090FBF2F080B200B2704700BFA0030108E6
:10D7D000904203DC8142ACBF0A46024610467047C5
:10D7E00070B5044610460E4602F02CFB054629464D
:10D7F000204602F037FD40B9304602F023FB0546D3
:10D800002946204602F010FD00B12C46204670BD8E
:10D8100070B514460E4602F015FB0546204602F090
:10D820000DFB04462146284602F014FC014628461A
:10D8300002F052FA0546304602F004FB214602F09F
:10D8400009FC0146284602F049FA02F015FD70BDB8
:10D850002DE9F04F05460C46D0F880108BB02E6FA6
:10D860000991D0F874E0D0F878C0C76FD0F8848000
:10D87000D0F888A091469B46D5F88C20EB6E009698
:10D88000099E20461499CDF804E0CDF808C004960E
:10D890000397CDF81480CDF818A000F02FF9A968EF
:10D8A00048460A464942FFF793FF002106464FF4D7
:10D8B0007A72A069FFF78CFF21696B6839B1434325
:10D8C0004FF47A7293FBF2F39B0493FBF1F16068DF
:10D8D000CBEB060630180A46266049426060FFF727
:10D8E00077FF23680246A068E1686769181A26690D
:10D8F00001FB03FE784306FB02FC4FF4807190FBB2
:10D90000F1F09EFBF1F14FF4802E40189CFBFEFCE1
:10D9100060446260A360206269680A464942FFF77A
:10D9200057FF0BB0BDE8F08F2DE9F04F05461E46BE
:10D93000D0F8B8308BB06F6C0993D0F848E0036C26
:10D94000D0F84CC0D0F8BC80D0F8C0A0D0F8C490BB
:10D9500093462A690097099F0C4608463146CDF840
:10D9600004E0CDF808C00397CDF81080CDF814A0DE
:10D97000CDF8189000F0C2F8296858460A46494286
:10D98000FFF726FF002180464FF47A72A069FFF767
:10D990001FFF2769AB683FB143434FF47A72B3FB73
:10D9A000F2F31B0493FBF7F7C6EB0800206018495D
:10D9B0004FF6FF72FFF70CFF0346606879421818B4
:10D9C0003A4623606060FFF703FF23680246A068C1
:10D9D000E1686769181A266901FB03FE784306FBB4
:10D9E00002FC4FF4807190FBF1F09EFBF1F14FF4DB
:10D9F000803E40189CFBFEFC60446260A360206295
:10DA0000A9680A464942FFF7E3FE0BB0BDE8F08F74
:10DA10000100FFFF2DE9F04F05460C46D0F8AC1091
:10DA20008BB0AE6A0991D0F82CE0D0F830C0D0F8B5
:10DA3000A870D0F8B080D0F8B4A091469B462A6A6E
:10DA40006B6A0096099E20461499CDF804E0CDF843
:10DA500008C004960397CDF81480CDF818A000F004
:10DA60004DF8A06900214FF47A72FFF7B1FE2669E4
:10DA70002B683EB143434FF47A7293FBF2F31B04DD
:10DA800093FBF6F6CBEB0900206018494FF6FF72C6
:10DA9000FFF79EFE03466068714218183246236005
:10DAA0006060FFF795FE23680246A068E168676939
:10DAB000181A266901FB03FE784306FB02FC4FF4AB
:10DAC000807190FBF1F09EFBF1F14FF4803E401825
:10DAD0009CFBFEFC60446260A360206229680A46E9
:10DAE0004942FFF775FE0BB0BDE8F08F0100FFFF64
:10DAF0000023036203604360836070472DE9F74FA2
:10DB0000164681EAE17582EAE272A5EBE175A2EBC5
:10DB1000E67295429B460446DDF830800F9BDDF8A7
:10DB200040A007DB1299C3608161C0F810A0119A70
:10DB3000426149E03046019302F084F907465846B5
:10DB400002F080F9019B8146CBEB030B05FB0BF048
:10DB500002F078F9394602F07DFA0146484602F0B3
:10DB6000BDF802F089FBE060404602F06BF9C8EBBB
:10DB70000A08814605FB08F002F064F9394602F014
:10DB800069FA0146484602F0A9F802F075FB2061E7
:10DB90000D9802F057F9119B0D998046581A684369
:10DBA00002F050F9394602F055FA0146404602F0BB
:10DBB00095F802F061FB0E99129A6061531A5D4369
:10DBC00095FBF6F67618A661BDE8FE8F094B19683D
:10DBD0005A68914201D100200BE01A68D118097AE5
:10DBE000013201701A601A68202A01D100221A60DD
:10DBF0000120704728040020014B9862704700BF45
:10DC000028040020034B1A78104612B100221A7023
:10DC1000012070470C0B002038B50B4B8446DC6AA2
:10DC20001A6B0134202C08BF002494420AD0DD6A0C
:10DC30000648ED1885F834C040F227710122DC62F5
:10DC4000FEF708FA38BD00BF280400200048004055
:10DC500038B50546002401E0FFF7DEFF2B5D0134F7
:10DC60001846002BF8D138BD234910B50B8813F0A6
:10DC7000200F15D0214B5A6818680132202A08BF9E
:10DC80000022824205D05C688888E118C0B2087220
:10DC90005A601B4B0A221A60184B9A6A194B1A6079
:10DCA0001548038813F0800F18D0164B1A68AAB9CC
:10DCB000124BDC6A196B8C420CD0196BCC1894F89F
:10DCC00034C00131A0F804C01963196B202905D1B3
:10DCD0001A6303E040F22771FEF7BCF90648038897
:10DCE00013F0400F06D040F22661FEF7ABFA034B6B
:10DCF0001A6BDB6A10BD00BF0048004028040020FA
:10DD0000100B0020140B002030B5054687B0544896
:10DD1000FEF7E8FA4FF480200121FDF731F90820E1
:10DD20000121FDF71FF908200021FDF737F94D48C3
:10DD30000021FCF79FFD06AC4FF4806324F8043DFE
:10DD40000323494821468DF8163015338DF81730D6
:10DD5000FCF700FD042344488DF8173021464FF4AA
:10DD60000063ADF81430FCF7F5FC6846FEF73CF9AB
:10DD70000B2D25D8DFE805F02406090C0F12151825
:10DD80001B1E20224FF461531CE04FF4964319E010
:10DD90004FF4E14316E04FF4164313E04FF46143B0
:10DDA00010E04FF496330DE04FF4E1330AE04FF406
:10DDB000613307E02D4B05E02D4B03E02D4B01E0D7
:10DDC0004FF41653694626480093FEF743FA27237B
:10DDD0000024012504A88DF8103005238DF811309A
:10DDE0008DF812408DF81350FCF724FE1C4840F2C9
:10DDF000FF31FEF703FA282122461948FEF72AF9D7
:10DE00002A46174840F22771FEF724F92A4614489B
:10DE100040F22661FEF71EF92A46114840F22551CC
:10DE2000FEF718F922460E4840F22441FEF712F997
:10DE300022460B4840F64601FEF70CF922460848F8
:10DE400040F66A11FEF706F9602122460448FEF703
:10DE500001F929460248FEF7EFF807B030BD00BFD0
:10DE60000048004010001400000C014090D0030056
:10DE700020A1070040420F00704700BF704700BF5D
:10DE800018B1012806D0002008E0054B986800F082
:10DE9000010003E0024B9868C0F34000704700BFE8
:10DEA000000C014000207047704700BF08B508B162
:10DEB000002002E0052001F075F808BD2DE9F341CE
:10DEC0004E4F01AD042001210324FDF74BF810262D
:10DED0004FF0180338462946ADF804308DF8064057
:10DEE0008DF80760FCF736FC082001213E61FDF744
:10DEF00039F841F23C43424829464FF00408ADF856
:10DF000004308DF806408DF80760FCF723FC4FF4D1
:10DF100000733B482946ADF804308DF806408DF873
:10DF20000780FCF717FC4823294635488DF8073051
:10DF300040F6030307F50067ADF804308DF806409E
:10DF4000FCF708FC30460121FDF70CF838464FF687
:10DF500000232946ADF804308DF806408DF807609F
:10DF6000FCF7F8FB4FF4A04338463B6129464FF4D9
:10DF70008063ADF804308DF806408DF80780FCF71B
:10DF8000E9FB4FF03F03384629460027ADF804303F
:10DF90008DF806408DF80770FCF7DCFB202001218E
:10DFA000FCF7E0FF17482946ADF804808DF80640DD
:10DFB0008DF80760FCF7CEFB38463B4610494FF41E
:10DFC00080644C610A468968013711F4006F4FF490
:10DFD00080611161926808BF013312F4006F18BFAD
:10DFE00001300A2FEAD10A2B01D0002003E00A28D1
:10DFF00014BF00200120BDE8FC8100BF00080140E3
:10E00000000C01400014014007B500238DF80730D3
:10E0100004484FF03F0301A9ADF80430FCF79AFB28
:10E020000EBD00BF00100140014B1868704700BFD3
:10E03000200B0020014B1860704700BF200B002010
:10E0400008B5054B05491868042201F0B7F900F03E
:10E05000E5F8034B186008BD1C0B0020200B0020C6
:10E06000180B002038B500F0D9F80C4C4EF65F22A2
:10E070002368C31A002BB8BF5B4293420CDD084BE8
:10E08000084A1D6810680135194604221D6001F018
:10E0900095F900F0C3F8206038BD00BF180B0020D0
:10E0A000200B00201C0B002008B5054B054918600B
:10E0B000042201F05FF900F0B1F8034B186008BDCD
:10E0C0001C0B0020200B0020180B0020024B1A68AC
:10E0D00001321A60704700BF280B00200028B8BF2B
:10E0E0004042404314235343484370B5154C44F613
:10E0F000206C2268656890FBFCF0B3FBF1F14FF0F7
:10E10000640C0132B1FBFCF140198A42226060606C
:10E1100016DBA3680C495A1C92FBFCF50CFB152579
:10E12000E66851F823200CF5617CB0FBFCF0B61AD0
:10E1300036180022626041F82300E660A560226084
:10E1400070BD00BF7C0400202C0B0020014BD86860
:10E15000704700BF7C040020014B1868704700BF67
:10E16000280B0020014B1860704700BF280B0020CF
:10E1700008B5034B03491868042201F01FF908BDD4
:10E18000240B0020280B002008B5034B0349042270
:10E19000186001F0EFF808BD240B0020280B0020C8
:10E1A000164B1A78DAB15A68154901325A600B6871
:10E1B000144A01330B601168134B01311160196867
:10E1C000124A013119601168114B013111601A684E
:10E1D00012B11A68013A1A600022084B00E00122CD
:10E1E0001A700C4B1A683AB11A68013A1A601B6827
:10E1F00013B9094B01221A70704700BF8C0400202C
:10E2000040090020FC030020F8030020F003002058
:10E21000140B0020100B00200C0B0020014B586841
:10E22000704700BF8C04002008B50420FDF7CAF831
:10E2300048F6A040FDF7D6F80120FDF7D9F80448CC
:10E2400003210022FCF7C4FC0120FDF7E7F808BD1C
:10E250009AC30200014B1878704700BFBC0C002025
:10E26000042807D0082808D008B1002007E0044B94
:10E27000186804E0024B586801E0014B9868704749
:10E2800094040020042807D0082808D008B10020F2
:10E2900007E0044BD86804E0024B186901E0014B29
:10E2A000586970479404002038B5064D0446002292
:10E2B00028462146FDF720FC284621460022FDF78E
:10E2C00029FC38BD002C014008B50020FFF7ECFF09
:10E2D0000420FFF7E9FF0820FFF7E6FF08BD00BFB5
:10E2E00038B5094D0446602228462146FDF720FC3A
:10E2F000284621460022FDF7FFFB2846214604223E
:10E30000FDF708FC38BD00BF002C014038B5094DB1
:10E310000446602228462146FDF70AFC284621468D
:10E320000122FDF7E9FB284621460022FDF7F2FB1A
:10E3300038BD00BF002C0140013938B504461546F0
:10E3400005294FD8DFE801F0311926033E0E0020E1
:10E35000FFF7AAFF0420FFF7C3FF0820FFF7D6FF4F
:10E36000D4B33CE00020FFF7BBFF0420FFF79CFF85
:10E370000820FFF7CBFF54B90AE00020FFF7B0FFF9
:10E380000420FFF7C3FF0820FFF78EFF04B925B371
:10E39000002325E00020FFF787FF0420FFF7B6FFEA
:10E3A0000820FFF79DFF54B90AE00020FFF7AEFFF9
:10E3B0000420FFF779FF0820FFF792FF04B965B149
:10E3C00002230DE00020FFF7A1FF0420FFF788FFE4
:10E3D0000820FFF769FF14B10DB9FF2300E0012306
:10E3E000014A136038BD00BFBC0C0020013938B5AC
:10E3F0000446154605294FD8DFE801F00E3E0326F6
:10E400001B330020FFF750FF0420FFF77FFF082099
:10E41000FFF766FF54B90AE00020FFF777FF0420FA
:10E42000FFF742FF0820FFF75BFF04B97DB302232B
:10E4300030E00020FFF76AFF0420FFF751FF0820BB
:10E44000FFF732FF54B90AE00020FFF72DFF042048
:10E45000FFF746FF0820FFF759FF04B9BDB10123BC
:10E4600018E00020FFF73CFF0420FFF71DFF082005
:10E47000FFF74CFF54B90CE00020FFF731FF0420F8
:10E48000FFF744FF0820FFF70FFF14B90DB9FF2372
:10E4900000E00023014A136038BD00BFBC0C00201F
:10E4A00038B5094D0446402228462146FDF740FB79
:10E4B000284621460122FDF71FFB2846214604225B
:10E4C000FDF728FB38BD00BF002C014008B5002037
:10E4D000FFF7E6FF0420FFF7E3FF0820FFF7E0FF68
:10E4E00008BD00BF013938B50446154605294FD887
:10E4F000DFE801F00E3E03261B330020FFF7D4FEB9
:10E500000420FFF7D1FE0820FFF7CAFF54B90AE044
:10E510000020FFF7C9FE0420FFF7C6FE0820FFF722
:10E52000BFFF04B97DB3022330E00020FFF7BCFE3B
:10E530000420FFF7B5FF0820FFF7B6FE54B90AE044
:10E540000020FFF7B1FE0420FFF7AAFF0820FFF725
:10E55000ABFE04B9BDB1012318E00020FFF7A0FF16
:10E560000420FFF7A1FE0820FFF79EFE54B90CE03F
:10E570000020FFF795FF0420FFF796FE0820FFF725
:10E5800093FE14B90DB9FF2300E00023014A136084
:10E5900038BD00BFBC0C0020013938B50446154613
:10E5A00005294FD8DFE801F00E3E03261B3300207B
:10E5B000FFF77AFE0420FFF7A9FE0820FFF770FF9F
:10E5C00054B90AE00020FFF7A1FE0420FFF76CFE1B
:10E5D0000820FFF765FF04B97DB3022330E0002077
:10E5E000FFF794FE0420FFF75BFF0820FFF75CFEB7
:10E5F00054B90AE00020FFF757FE0420FFF750FF50
:10E600000820FFF783FE04B9BDB1012318E0002004
:10E61000FFF746FF0420FFF747FE0820FFF776FECE
:10E6200054B90CE00020FFF73BFF0420FFF76EFE1B
:10E630000820FFF739FE14B90DB9FF2300E00023CD
:10E64000014A136038BD00BFBC0C002038B5094D2D
:10E650000446502228462146FDF76AFA28462146FC
:10E660000122FDF749FA284621460422FDF752FA15
:10E6700038BD00BF002C0140013938B504461546AD
:10E6800005294FD8DFE801F00E3E03261B3300209A
:10E69000FFF70AFE0420FFF7D9FF0820FFF720FE4E
:10E6A00054B90AE00020FFF7D1FF0420FFF7FCFD7A
:10E6B0000820FFF715FE04B97DB3022330E00020E7
:10E6C000FFF7C4FF0420FFF70BFE0820FFF7ECFD67
:10E6D00054B90AE00020FFF7E7FD0420FFF700FE31
:10E6E0000820FFF7B3FF04B9BDB1012318E00020F3
:10E6F000FFF7F6FD0420FFF7D7FD0820FFF7A6FF80
:10E7000054B90CE00020FFF7EBFD0420FFF79EFF5B
:10E710000820FFF7C9FD14B90DB9FF2300E000235D
:10E72000014A136038BD00BFBC0C002038B58446D8
:10E730000C4615469DF810109DF8142018460BB194
:10E7400081F00701BCF1800F21D007D8BCF1010F87
:10E7500010D00BD3BCF1020F27D10FE0BCF1820F18
:10E760001ED01AD3BCF1830F1FD11CE03DB1FFF7BF
:10E7700013FF1AE01DB1FFF77FFF16E025B9022C49
:10E7800011D0012C09D10BE0FFF730FE0DE008B1EC
:10E7900081F00701FFF7D0FD07E0FFF7A3FE04E0DB
:10E7A000FFF794FE01E0FFF78FFD38BDF8B5A0F547
:10E7B000AA73013B9B059B0D2A4E0C4605464FF460
:10E7C000E1611846F3601746FEF7D2FF01B26143DC
:10E7D0004FF4E16391FBF3F101F5617131601CB914
:10E7E000012F08BF4FF4617189B21F48FDF726FA67
:10E7F000AB059B0D1B4E18464FF4E1613361FEF7EC
:10E80000B7FF01B261434FF4E16391FBF3F101F50E
:10E81000617171601CB9012F08BF4FF4617105F57A
:10E82000AA750135AD0589B20F48AD0D0D4EFDF746
:10E8300007FA4FF4E16128467561FEF799FF01B2CE
:10E8400061434FF4E16391FBF3F101F56171B16054
:10E850001CB9012F08BF4FF4617189B20248FDF75E
:10E86000F1F9F8BD94040020002C014010B50128F6
:10E8700088B001D0042854D101200146FCF780FB68
:10E8800004200121FCF76EFB18238DF81F300323B1
:10E8900007A98DF81E3028484FF00803ADF81C304A
:10E8A000FBF758FF4FF08040FDF73CFB4FF00004B2
:10E8B00004A94FF01C034FF08040ADF81430ADF8C0
:10E8C0001040ADF81640ADF812408DF81840FCF736
:10E8D000C7FD4FF030036946ADF800304FF080407F
:10E8E0004FF00103ADF80230ADF80C40ADF8064032
:10E8F000ADF80840FCF7BCFE0E214FF08040FDF75C
:10E90000A3F901214FF08040FDF704F801214FF0F9
:10E910008040FCF725FF4FF080400121FCF72EFFDF
:10E9200008E038B1022805D0032803D04FF080401A
:10E93000FDF7F8FA08B010BD00080140F0B5032853
:10E940008BB007D001D828B188E0052802D08028F4
:10E9500040F0848002200121FCF712FB09AC012168
:10E960001020FCF7FFFA2046FBF73EFF4823214624
:10E970008DF827303C484FF4E073ADF82430FBF7B6
:10E98000E9FE01213948FBF775FF03AC3848FDF774
:10E99000C9FA2046FCF7BCFE21464FF0FF334FF08A
:10E9A00000043348ADF81030ADF80C40ADF812401B
:10E9B000ADF80E40FCF754FD0022134603212C480D
:10E9C000FCF75CFF6846FCF7B7FE4FF002076946AC
:10E9D000274808AEADF80870FDF740FA69464FF0D9
:10E9E000040323480125ADF80030FDF737FA1D2355
:10E9F00030468DF820308DF821708DF822408DF84A
:10EA00002350FCF717F81A4841F65F61FDF77CF9CF
:10EA100017480021FDF70EF929461548FCF7A0FE1E
:10EA200008210220FBF754FF4FF4807306A80693D9
:10EA300008238DF81D308DF81C408DF81E50FBF713
:10EA4000F9FD172330468DF820308DF822408DF8DF
:10EA500023508DF82140FBF7EDFF02E00448FDF75D
:10EA600061FA0BB0F0BD00BF00100140000C1A00AD
:10EA70000004004070B501288CB0044602D0042880
:10EA800040F0A28004200121FCF77AFA0AAD0121AE
:10EA90000820FCF767FA2846FBF7A6FE482329461C
:10EAA0004C488DF82B304FF4E073ADF8283007ADAB
:10EAB000FBF750FE4848FDF735FA2846FCF728FEDC
:10EAC0004FF0FF332946444804ADADF820304FF0F5
:10EAD0000003ADF82230FCF7C3FC2846FCF72CFEFF
:10EAE0004FF00003ADF81030ADF812304FF00B03CB
:10EAF00029463948ADF818304FF00303ADF814300B
:10EB0000FDF7ACF9012228213348FCF795FE324885
:10EB1000FCF762FE01213048FDF74EF840212E48F7
:10EB2000FCF798FE012C02D12B48042101E02A4871
:10EB30000021FDF767F801212748FDF72FF84FF076
:10EB400070034FF001054FF000066946ADF8003044
:10EB500021484FF4C873ADF80630ADF80250ADF857
:10EB60000860FCF7E7FC08211B48FCF715FF0121B2
:10EB70001948FCF7CFFE02241E230BA88DF82C3079
:10EB80008DF82E608DF82F508DF82D40FBF752FF39
:10EB9000114841F65F61FDF7B7F8214601220E48A2
:10EBA000FCF7FCFD01210A460B48FCF7F7FD50215C
:10EBB0000948FDF71BF800210748FDF73BF8064818
:10EBC0000121FCF7CDFD02E00348FDF7ABF90CB0E5
:10EBD00070BD00BF000C01400008004070B5032864
:10EBE0008CB003D8022804D218B1ADE0802840F0E0
:10EBF000AB8001200146FCF7C3F90AAC01210420D7
:10EC0000FCF7B0F92046FBF7EFFD042521464FF055
:10EC100007035148ADF8283007AC8DF82B50FBF7AF
:10EC200099FD4FF08040FDF77DF92046FCF770FD1F
:10EC300004AE21464FF0FF334FF000044FF0804008
:10EC4000ADF82030ADF82240FCF70AFC3046FCF766
:10EC500073FD4FF00B033146ADF818304FF0804094
:10EC60004FF00303ADF81430ADF81040ADF812408A
:10EC7000FDF7F4F8012228214FF08040FCF7DCFD7D
:10EC80004FF08040FCF7A8FD01214FF08040FCF7D9
:10EC900093FF40214FF08040FCF7DCFD29464FF008
:10ECA0008040FCF7AFFF01214FF08040FCF776FF7A
:10ECB0004FF070034FF001066946ADF800304FF099
:10ECC00080404FF4C873ADF80630ADF80260ADF87F
:10ECD0000840FCF72FFC08214FF08040FCF75CFE59
:10ECE00001214FF08040FCF715FE02251C230BA8E4
:10ECF0008DF82C308DF82E408DF82F608DF82D502A
:10ED0000FBF798FE4FF0804041F65F61FCF7FCFF97
:10ED1000012229464FF08040FCF740FD01210A46C0
:10ED20004FF08040FCF73AFD50214FF08040FCF757
:10ED30005DFF00214FF08040FCF77CFF4FF08040EA
:10ED40000121FCF70DFD05E0012803D04FF08040C4
:10ED5000FDF7E8F80CB070BD0008014070B5012166
:10ED60008EB0044640F60C00FCF7FCF801250026A6
:10ED70001A230DA88DF834308DF836508DF83750A1
:10ED80008DF83560FBF756FE1923022C13BF8DF862
:10ED900036508DF836608DF835408DF835608DF839
:10EDA00034300DA801238DF83730FBF743FE1823CC
:10EDB0000CAD8DF833300323774829468DF8323077
:10EDC0004FF4E063ADF83030FBF7C4FC4EF20003C3
:10EDD00029467248ADF83030FBF7BCFC7048FDF7AF
:10EDE000A1F8032C02D8022C65D206E0052C62D0D3
:10EDF00003D3802C40F0C2805DE04FF46163ADF836
:10EE000028304FF00003012409A9ADF82430ADF8F3
:10EE10002A3063484FF04003ADF826308DF82C407F
:10EE2000FCF71EFB4FF00003ADF804304FF0040375
:10EE3000ADF808304FF0000301ADADF80A30ADF881
:10EE40000C30ADF80E304FF480732946ADF8103019
:10EE500053484FF40073ADF81230ADF80640FCF79C
:10EE600021FB29464E48FCF765FB29464C48FCF738
:10EE7000B1FB4FF40063ADF814304FF48063ADF88C
:10EE800016304FF00003ADF81830ADF81C304FF4D9
:10EE9000005305A9ADF81E3041484FF48043ADF84A
:10EEA0001A40ADF82030FCF71BFC22463C482021DC
:10EEB000FCF774FC5DE04FF4E163ADF828304FF0EF
:10EEC00000030124364809A9ADF82430ADF82A30F2
:10EED0004FF06003ADF826308DF82C40FCF7C0FAF7
:10EEE0004FF06003ADF804304FF00403ADF8083084
:10EEF0004FF00003ADF80A304FF0020301ADADF85A
:10EF00000C304FF0080326482946ADF80E304FF07C
:10EF10000003ADF81030ADF81230ADF80640FCF744
:10EF2000C1FA1F482946FCF705FB29461C48FCF797
:10EF300051FB4FF40063ADF814304FF48063ADF82B
:10EF400016304FF00003ADF81830ADF81C304FF418
:10EF50000053134805A9ADF81E304FF48043ADF8B7
:10EF60001A40ADF82030FCF7BBFB0D482146FCF7FA
:10EF700015FE21460A482246FCF710FC01210848EC
:10EF8000FCF7F2FC01210648FCF7EAFB04480121EA
:10EF9000FCF7F4FB0EB070BD00080140000C01400E
:10EFA000002C0140024B33F8100080B2704700BFC4
:10EFB000AC040020024B03EB40031982704700BFF2
:10EFC000AC040020024B03EB4003188A704700BFDB
:10EFD000AC040020044B03EB400233F81030108ADD
:10EFE0009BB2C01A704700BFAC0400200F4B1A78C8
:10EFF0007AB1012A19D10028B8BF4042B0F5E16FBB
:10F0000013DD0B494FF40070486100211970094B62
:10F010000AE0C730B0F5C77F07D805494FF4007044
:10F020000861044901220A701A707047C20C00205E
:10F0300000100140C10C00200D4B1B780BB1642166
:10F0400002E0002908BF3E214FF47A735843414340
:10F05000F13391FBF3F16420064B48431B78002BFE
:10F0600014BF4FF402634FF4F17390FBF3F0704759
:10F07000C00C0020C20C0020044B44F2740202FBBE
:10F0800000304FF4805190FBF1F070470060FCFDC0
:10F09000014B1878704700BFC10C0020014B0022C3
:10F0A0001A707047C10C0020014B1870704700BFE8
:10F0B000C20C0020014B1870704700BFC00C00202C
:10F0C00038B50A4D288880B2FFF7D6FF0446688815
:10F0D00080B2FFF7D1FF04FB04F300FB00330019FB
:10F0E00000FB0030FEF7BCFA38BD00BFAC040020C6
:10F0F000F8B52648FCF7EAFD40F20153984202D9E0
:10F100000724002705E0224B06241F881E8ABFB271
:10F11000F71B1E48FCF7DEFD40F20153984201D96F
:10F12000002606E01A4B24F002045E885B8AB6B221
:10F130009E1B1648FCF7D2FD40F20153984201D9BC
:10F14000002506E0124B24F004049D889B8AADB292
:10F150005D1B022C05D0042C05D0012C04D1AF1965
:10F1600002E0EE1900E0F51938467F4300F084FB19
:10F17000304606FB067600F085FB284600F088FB4B
:10F1800005FB0560FEF76CFAF8BD00BF002C0140DE
:10F19000AC04002070B590B0FEF736FF01200146A8
:10F1A000FBF7D2FE01214FF40070FBF7DBFE3E4877
:10F1B000FBF742F93D4B002400933D4B072601939A
:10F1C00080230593DB18069303F540730793A3F59B
:10F1D000787335486946089303F5FF530993029401
:10F1E000039604940A94FBF797F901212E48FBF744
:10F1F000C3F901254FF460232E480BA90D930B94FE
:10F200008DF830508DF831400E948DF83C60FAF74F
:10F2100047FF0B21032327482A46FAF7C3FF0C2197
:10F22000022203232348FAF7BDFF032213460D21D0
:10F230002048FAF7B7FF0A21042203231D48FAF7F2
:10F24000B1FF052203231B480E21FAF7ABFF0F2164
:10F25000184806220323FAF7A5FF03233246154870
:10F260000921FAF79FFF224612484FF4FC61FAF792
:10F270005BFF10482946FAF74DFF0E482946FAF77A
:10F280003FFF0C48FAF75AFF0A48FAF75DFF0028DB
:10F29000FAD10848FAF75CFF0648FAF75FFF002842
:10F2A000FAD110B070BD00BF080002404C240140EC
:10F2B000AC04002000240140114B82B01B78E3B164
:10F2C000104B04221A611C325A61002301E0019B99
:10F2D00001330193019A0C4B9A42F8D9094B04224D
:10F2E0005A611C321A61002301E0019B0133019332
:10F2F000019A054B9A42E3D8F7E702B0704700BF86
:10F3000058090020000C01403F0D030062B6704711
:10F3100072B67047024B4FF400521A61704700BF3B
:10F3200000100140024B4FF400525A61704700BF79
:10F330000010014008B510B1FBF71AFC01E0FBF723
:10F340001FFC08BD08B5FEF7ADFD08BD08B5FEF70A
:10F3500097FD08BD08B5FEF791FD08BD08B5FEF79D
:10F360008BFD08BD08B5FEF7A9FD014B187008BD5F
:10F370005809002070B5044600200E4615460321AA
:10F380000246F4F799FF0020C4F307210246F4F780
:10F3900093FF0020E1B20246F4F78EFF002407E05D
:10F3A000944214BF00220122F4F786FF3055013445
:10F3B00000206A1EAC420146F2D370BD2DE9F04137
:10F3C00004460F461646002006210122F4F774FF7A
:10F3D000002005210246F4F76FFF002001220146BC
:10F3E000F4F76AFF10F0020FF2D00020022102466B
:10F3F000F4F762FF0020C4F307210246F4F75CFF34
:10F400000020E1B20246F4F757FF002543E0013443
:10F4100014F03F08795D01D1012204E0721E95428B
:10F4200014BF002201220020F4F746FFB8F1000FBC
:10F4300030D1731E9D422DD2002005210246F4F7E3
:10F440003BFF002001220146F4F736FF10F00100D7
:10F45000F2D106210122F4F72FFF002005210246F8
:10F46000F4F72AFF002001220146F4F725FF10F0EF
:10F47000020FF2D0002002210246F4F71DFF002007
:10F48000C4F307210246F4F717FF0020E1B2024659
:10F49000F4F712FF0135B542B9D300200521024629
:10F4A000F4F70AFF002001220146F4F705FF10F0EF
:10F4B000010FF2D1BDE8F08110B504460020032110
:10F4C0000246F4F7F9FE0020C4F307210246F4F7E0
:10F4D000F3FE0020E1B20246F4F7EEFE0020014602
:10F4E0000122F4F7E9FE10BD38B5012204460D46AD
:10F4F00000200621F4F7E0FE002005210246F4F783
:10F50000DBFE002001220146F4F7D6FE10F0020FC8
:10F51000F2D0002002210246F4F7CEFE0020C4F310
:10F5200007210246F4F7C8FE0020E1B20246F4F7D4
:10F53000C3FE294600200122F4F7BEFE002005216B
:10F540000246F4F7B9FE002001220146F4F7B4FEAA
:10F5500010F0010FF2D138BD38B50725454305F548
:10F5600000650C46284609780135FFF7BDFF28469F
:10F5700061780135FFF7B8FF2846A1780135FFF71C
:10F58000B3FF284621790135FFF7AEFF28466179A0
:10F590000135FFF7A9FF2846A179FFF7A5FF681CF1
:10F5A000E179FFF7A1FF38BD37B5072545430020B6
:10F5B0000C4602460321F4F77FFE05F500650020A6
:10F5C000C5F307210246F4F777FE0020E9B20246B0
:10F5D000F4F772FE002001460246F4F76DFE8DF846
:10F5E0000000002001460246F4F766FE8DF8010097
:10F5F000002001460246F4F75FFE8DF8020000206D
:10F6000001460246F4F758FE8DF80400002001463A
:10F610000246F4F751FE8DF805000020014602462F
:10F62000F4F74AFE8DF80600002001220146F4F7A7
:10F6300043FE2368009A23F07F4322F07F429A42E0
:10F640008DF8070001D0002005E06368019898421A
:10F6500014BF002001203EBD38B54FF400640020E7
:10F6600006210122F4F728FE002005210246F4F7C6
:10F6700023FE002001220146F4F71EFE10F0020FC7
:10F68000F2D0002002210246F4F716FE0020C4F357
:10F6900007210246F4F710FE0020E1B20246F4F71B
:10F6A0000BFE002500203F2D14BF00220122014641
:10F6B0000135F4F701FE402DF4D10020052102466A
:10F6C000F4F7FAFD002001220146F4F7F5FD10F0F1
:10F6D000010FF2D14034B4F5804FC0D138BD00BF26
:10F6E00008B540F2FF70FFF7E7FE392802D1164B4C
:10F6F0001B78EBB140F2FF700021FFF7F5FEFFF73A
:10F70000ABFF002011494022FFF758FE402010496E
:10F710004FF48072FFF752FE4FF4A0700C494FF483
:10F720008072FFF74BFE40F2FF703921FFF7DCFEDD
:10F73000002040220549FFF71DFE402004494FF4F8
:10F740008072FFF717FE08BD58090020080000204E
:10F750004C00002038B50725454300200C460246E2
:10F760000321F4F7A9FD05F500650020C5F3072185
:10F770000246F4F7A1FD0020E9B20246F4F79CFD31
:10F78000002001460246F4F797FD20700020014654
:10F790000246F4F791FD6070002001460246F4F73E
:10F7A0008BFDA070002001460246F4F785FD207114
:10F7B000002001460246F4F77FFD607100200146FB
:10F7C0000246F4F779FDA071002001460122F4F70A
:10F7D00073FDE07138BD00BF704700BF704700BFC8
:10F7E000704700BF704700BF704700BF704700BF41
:10F7F000704700BF704700BF704700BF704700BF31
:10F80000014B1868704700BFE00C0020014B1868DE
:10F81000704700BFD80C0020014B1868704700BF2C
:10F82000D40C0020014B1868704700BFD00C00209A
:10F83000014B1868704700BFDC0C0020014B1868B2
:10F84000704700BFC40C0020014B1868704700BF10
:10F85000CC0C0020014B1868704700BFC80C00207A
:10F86000014B1860704700BFE00C0020014B18608E
:10F87000704700BFD80C0020014B1860704700BFD4
:10F88000D40C0020014B1860704700BFD00C002042
:10F89000014B1860704700BFDC0C0020014B186062
:10F8A000704700BFC40C0020014B1860704700BFB8
:10F8B000CC0C0020014B1860704700BFC80C002022
:10F8C00081F0004102E000BF83F0004330B54FEA11
:10F8D00041044FEA430594EA050F08BF90EA020F7E
:10F8E0001FBF54EA000C55EA020C7FEA645C7FEA11
:10F8F000655C00F0E2804FEA5454D4EB5555B8BF34
:10F900006D420CDD2C4480EA020281EA030382EAA4
:10F91000000083EA010180EA020281EA0303362D36
:10F9200088BF30BD11F0004F4FEA01314FF4801C09
:10F930004CEA113102D0404261EB410113F0004F1B
:10F940004FEA03334CEA133302D0524263EB4303D2
:10F9500094EA050F00F0A780A4F10104D5F1200E70
:10F960000DDB02FA0EFC22FA05F2801841F10001CB
:10F9700003FA0EF2801843FA05F359410EE0A5F19F
:10F9800020050EF1200E012A03FA0EFC28BF4CF0D0
:10F99000020C43FA05F3C01851EBE37101F0004586
:10F9A00007D54FF0000EDCF1000C7EEB00006EEB93
:10F9B0000101B1F5801F1BD3B1F5001F0CD349081D
:10F9C0005FEA30004FEA3C0C04F101044FEA445274
:10F9D00012F5800F80F09A80BCF1004F08BF5FEAFB
:10F9E000500C50F1000041EB045141EA050130BDDB
:10F9F0005FEA4C0C404141EB010111F4801FA4F17E
:10FA00000104E9D191F0000F04BF01460020B1FAD2
:10FA100081F308BF2033A3F10B03B3F120020CDA0A
:10FA20000C3208DD02F1140CC2F10C0201FA0CF0E8
:10FA300021FA02F10CE002F11402D8BFC2F1200C4D
:10FA400001FA02F120FA0CFCDCBF41EA0C01904003
:10FA5000E41AA2BF01EB0451294330BD6FEA04044C
:10FA60001F3C1CDA0C340EDC04F11404C4F1200237
:10FA700020FA04F001FA02F340EA030021FA04F349
:10FA800045EA030130BDC4F10C04C4F1200220FAA0
:10FA900002F001FA04F340EA0300294630BD21FADE
:10FAA00004F0294630BD94F0000F83F4801306BFA4
:10FAB00081F480110134013D4EE77FEA645C18BF98
:10FAC0007FEA655C29D094EA050F08BF90EA020F2F
:10FAD00005D054EA000C04BF1946104630BD91EA27
:10FAE000030F1EBF0021002030BD5FEA545C05D12A
:10FAF0004000494128BF41F0004130BD14F5800469
:10FB00003CBF01F5801130BD01F0004545F0FE41DC
:10FB100041F470014FF0000030BD7FEA645C1ABF11
:10FB2000194610467FEA655C1CBF0B46024650EA48
:10FB3000013406BF52EA033591EA030F41F4002174
:10FB400030BD00BF90F0000F04BF0021704730B5FA
:10FB50004FF4806404F132044FF000054FF00001CF
:10FB600050E700BF90F0000F04BF0021704730B590
:10FB70004FF4806404F1320410F0004548BF404265
:10FB80004FF000013EE700BF42004FEAE2014FEABA
:10FB900031014FEA02701FBF12F07F4393F07F4F95
:10FBA00081F06051704792F0000F14BF93F07F4FC7
:10FBB000704730B54FF4607401F0004521F000410A
:10FBC00020E700BF50EA010208BF704730B54FF090
:10FBD00000050AE050EA010208BF704730B511F095
:10FBE000004502D5404261EB41014FF4806404F1CD
:10FBF00032045FEA915C3FF4DCAE4FF003025FEA4F
:10FC0000DC0C18BF03325FEADC0C18BF033202EBD6
:10FC1000DC02C2F1200300FA03FC20FA02F001FA30
:10FC200003FE40EA0E0021FA02F11444C1E600BFCF
:10FC30004FEA4102B2F1E04324BFB3F5001CDCF10E
:10FC4000FE5C0DD901F0004C4FEAC0024CEA507046
:10FC5000B2F1004F40EB830008BF20F00100704775
:10FC600011F0804F21D113F13872BCBF01F0004078
:10FC7000704741F480114FEA5252C2F11802C2F1AA
:10FC8000200C10FA0CF320FA02F018BF40F001002B
:10FC90004FEAC1234FEAD32303FA0CFC40EA0C00DD
:10FCA00023FA02F34FEA4303CCE77FEA625307D11A
:10FCB00050EA01331EBF4FF0FE4040F44000704751
:10FCC00001F0004040F0FE4040F40000704700BFEB
:10FCD00080F0004002E000BF81F0004142001FBF01
:10FCE0005FEA410392EA030F7FEA226C7FEA236C0A
:10FCF0006AD04FEA1262D2EB1363C1BFD2184140FF
:10FD000048404140B8BF5B42192B88BF704710F094
:10FD1000004F40F4000020F07F4018BF404211F037
:10FD2000004F41F4000121F07F4118BF494292EA9F
:10FD3000030F3FD0A2F1010241FA03FC10EB0C00CB
:10FD4000C3F1200301FA03F100F0004302D5494258
:10FD500060EB4000B0F5000F13D3B0F1807F06D305
:10FD600040084FEA310102F10102FE2A51D2B1F1FD
:10FD7000004F40EBC25008BF20F0010040EA0300F2
:10FD80007047490040EB000010F4000FA2F101029F
:10FD9000EDD1B0FA80FCACF1080CB2EB0C0200FA29
:10FDA0000CF0AABF00EBC25052421843BCBFD04077
:10FDB0001843704792F0000F81F4000106BF80F4F1
:10FDC00000000132013BB5E74FEA41037FEA226CB4
:10FDD00018BF7FEA236C21D092EA030F04D092F07F
:10FDE000000F08BF0846704790EA010F1CBF0020B3
:10FDF000704712F07F4F04D1400028BF40F0004010
:10FE0000704712F100723CBF00F50000704700F02F
:10FE1000004343F0FE4040F4000070477FEA226256
:10FE200016BF08467FEA23630146420206BF5FEA27
:10FE3000412390EA010F40F4800070474FF0000327
:10FE400004E000BF10F0004348BF40425FEA000CEE
:10FE500008BF704743F0964301464FF000001CE096
:10FE600050EA010208BF70474FF000030AE000BFEC
:10FE700050EA010208BF704711F0004302D540422A
:10FE800061EB41015FEA010C02BF8446014600209C
:10FE900043F0B64308BFA3F18053A3F50003BCFAB7
:10FEA0008CF2083AA3EBC25310DB01FA02FC634464
:10FEB00000FA02FCC2F12002BCF1004F20FA02F26B
:10FEC00043EB020008BF20F00100704702F120025E
:10FED00001FA02FCC2F1200250EA4C0021FA02F2BF
:10FEE00043EB020008BF20EADC7070474FF0FF0CC4
:10FEF0001CEAD0521EBF1CEAD15392EA0C0F93EABF
:10FF00000C0F6FD01A4480EA010C400218BF5FEA60
:10FF100041211ED04FF0006343EA501043EA5111D3
:10FF2000A0FB01310CF00040B1F5000F3EBF4900CD
:10FF300041EAD3715B0040EA010062F17F02FD2AD1
:10FF40001DD8B3F1004F40EBC25008BF20F00100B4
:10FF5000704790F0000F0CF0004C08BF49024CEACB
:10FF6000502040EA51207F3AC2BFD2F1FF0340EA5D
:10FF7000C250704740F400004FF00003013A5DDCCE
:10FF800012F1190FDCBF00F000407047C2F100020F
:10FF9000410021FA02F1C2F1200200FA02FC5FEAFC
:10FFA000310040F1000053EA4C0308BF20EADC7046
:10FFB000704792F0000F00F0004C02BF400010F4B8
:10FFC000000F013AF9D040EA0C0093F0000F01F065
:10FFD000004C02BF490011F4000F013BF9D041EA87
:10FFE0000C018FE70CEAD15392EA0C0F18BF93EA89
:10FFF0000C0F0AD030F0004C18BF31F0004CD8D1B3
:020000040801F1
:1000000080EA010000F00040704790F0000F17BF39
:1000100090F0004F084691F0000F91F0004F14D07F
:1000200092EA0C0F01D142020FD193EA0C0F03D1D7
:100030004B0218BF084608D180EA010000F00040DA
:1000400040F0FE4040F40000704740F0FE4040F4B5
:10005000400070474FF0FF0C1CEAD0521EBF1CEA54
:10006000D15392EA0C0F93EA0C0F69D0A2EB030272
:1000700080EA010C49024FEA402037D04FF080530C
:1000800043EA111143EA10130CF000408B4238BFD1
:100090005B0042F17D024FF4000C8B4224BF5B1ADF
:1000A00040EA0C00B3EB510F24BFA3EB510340EA2D
:1000B0005C00B3EB910F24BFA3EB910340EA9C00DB
:1000C000B3EBD10F24BFA3EBD10340EADC001B014B
:1000D00018BF5FEA1C1CE0D1FD2A3FF650AF8B42EF
:1000E00040EBC25008BF20F0010070470CF0004CFC
:1000F0004CEA50207F32C2BFD2F1FF0340EAC25027
:10010000704740F400004FF00003013A37E792F0E7
:10011000000F00F0004C02BF400010F4000F013A45
:10012000F9D040EA0C0093F0000F01F0004C02BF40
:10013000490011F4000F013BF9D041EA0C0195E7A9
:100140000CEAD15392EA0C0F08D142027FF47DAF42
:1001500093EA0C0F7FF470AF084676E793EA0C0F32
:1001600004D14B023FF44CAF08466EE730F0004C30
:1001700018BF31F0004CCAD130F000427FF45CAFC0
:1001800031F000437FF43CAF5FE700BF4FF0FF3C2E
:1001900006E000BF4FF0010C02E000BF4FF0010C81
:1001A0004DF804CD4FEA40024FEA41037FEA226C4A
:1001B00018BF7FEA236C11D001B052EA530C18BF6C
:1001C00090EA010F58BFB2EB030088BFC81738BFD1
:1001D0006FEAE17018BF40F0010070477FEA226CBF
:1001E00002D15FEA402C05D17FEA236CE4D15FEABB
:1001F000412CE1D05DF8040B704700BF84460846EF
:100200006146FFE70FB5FFF7C9FF002848BF10F1AF
:10021000000F0FBD4DF808EDFFF7F4FF0CBF0120F4
:1002200000205DF808FB00BF4DF808EDFFF7EAFF7E
:1002300034BF012000205DF808FB00BF4DF808ED39
:10024000FFF7E0FF94BF012000205DF808FB00BF2E
:100250004DF808EDFFF7D2FF94BF012000205DF8B4
:1002600008FB00BF4DF808EDFFF7C8FF34BF0120C1
:1002700000205DF808FB00BF4FEA4002B2F1FE4FDC
:100280000FD34FF09E03B3EB12620DD94FEA002358
:1002900043F0004310F0004F23FA02F018BF404231
:1002A00070474FF00000704712F1610F01D1420218
:1002B00005D110F0004008BF6FF0004070474FF0CC
:1002C000000070470105000302040000010302055D
:1002D000000400001201100102000040D0161B05AE
:1002E000100101020301000009024300020100C0E5
:1002F000320904000001020201000524001001057A
:1003000024010001042402020524060001070582DD
:10031000030800FF09040100020A000000070503AA
:1003200002400000070581024000000004030904A8
:1003300026035400720069006E0061006D006900C0
:1003400063004D006F00740069006F006E002000B4
:10035000430074006C000000320345007600610029
:100360006C002D003600300033002000280076009D
:10037000690072007400750061006C002000430089
:100380004F004D0029002000200000000000000068
:100390000102030401020304060708090204060817
:1003A0000000000010000000160000001B0000000C
:1003B0002000000023000000270000002A000000A9
:1003C0002D00000030000000320000003500000069
:1003D00037000000390000003B0000003D00000035
:1003E0004000000041000000430000004500000004
:1003F00047000000490000004B0000004C000000D6
:100400004E000000500000005100000053000000AA
:100410005400000056000000570000005900000082
:100420005A0000005B0000005D0000005E0000005C
:100430006000000061000000620000006300000036
:100440006500000066000000670000006800000012
:100450006A0000006B0000006C0000006D000000EE
:100460006E000000700000007100000072000000CB
:1004700073000000740000007500000076000000AA
:100480007700000078000000790000007A0000008A
:100490007B0000007C0000007D0000007E0000006A
:1004A0008000000080000000810000008200000049
:1004B000830000008400000085000000860000002A
:1004C0008700000088000000890000008A0000000A
:1004D0008B0000008C0000008D0000008E000000EA
:1004E0008F000000900000009000000091000000CC
:1004F00092000000930000009400000095000000AE
:100500009600000096000000970000009800000090
:10051000990000009A0000009B0000009B00000072
:100520009C0000009D0000009E0000009F00000055
:10053000A0000000A0000000A1000000A200000038
:10054000A3000000A3000000A4000000A50000001C
:10055000A6000000A7000000A7000000A8000000FF
:10056000A9000000AA000000AA000000AB000000E3
:10057000AC000000AD000000AD000000AE000000C7
:10058000AF000000B0000000B0000000B1000000AB
:10059000B2000000B2000000B3000000B400000090
:1005A000B5000000B5000000B6000000B700000074
:1005B000B7000000B8000000B9000000B90000005A
:1005C000BA000000BB000000BB000000BC0000003F
:1005D000BD000000BD000000BE000000BF00000024
:1005E000C0000000C0000000C1000000C100000009
:1005F000C2000000C3000000C3000000C4000000EF
:10060000C5000000C5000000C6000000C7000000D3
:10061000C7000000C8000000C9000000C9000000B9
:10062000CA000000CB000000CB000000CC0000009E
:10063000CC000000CD000000CE000000CE00000085
:10064000CF000000D0000000D0000000D10000006A
:10065000D1000000D2000000D3000000D300000051
:10066000D4000000D4000000D5000000D600000037
:10067000D6000000D7000000D7000000D80000001E
:10068000D9000000D9000000DA000000DA00000004
:10069000DB000000DB000000DC000000DD000000EB
:1006A000DD000000DE000000DE000000DF000000D2
:1006B000E0000000E0000000E1000000E1000000B8
:1006C000E2000000E2000000E3000000E3000000A0
:1006D000E4000000E5000000E5000000E600000086
:1006E000E6000000E7000000E7000000E80000006E
:1006F000E8000000E9000000EA000000EA00000055
:10070000EB000000EB000000EC000000EC0000003B
:10071000ED000000ED000000EE000000EE00000023
:10072000EF000000F0000000F0000000F100000009
:10073000F1000000F2000000F2000000F3000000F1
:10074000F3000000F4000000F4000000F5000000D9
:10075000F5000000F6000000F6000000F7000000C1
:10076000F7000000F8000000F8000000F9000000A9
:10077000F9000000FA000000FA000000FB00000091
:10078000FB000000FC000000FC000000FD00000079
:10079000FD000000FE000000FE000000FF00000061
:1007A0000000C90092015B022403ED03B6047F053B
:1007B00047061007D907A2086A09330AFB0AC30BC8
:1007C0008B0C530D1B0EE30EAB0F7210391101127F
:1007D000C8128E1355141B15E215A8166D17331881
:1007E000F818BD19821A471B0B1CCF1C931D561EEF
:1007F000191FDC1F9F2061212322E522A6236724E5
:100800002825E825A82667272628E528A329612A80
:100810001F2BDC2B982C552D112ECC2E872F4130E1
:10082000FB30B5316E322633DE3396344D35043627
:10083000BA366F372438D8388C39403AF23AA53B6B
:10084000563C073DB83D683E173FC53F73402141C8
:10085000CE417A422543D0437A442445CD4575465E
:100860001C47C34769480F49B449584AFB4A9E4B45
:100870003F4CE14C814D214EBF4E5E4FFB4F975098
:100880003351CE51695202539B533354CA5460556D
:10089000F5558A561D57B0574258D4586459F359E4
:1008A000825A105B9D5B295CB45C3E5DC75D505E07
:1008B000D75E5E5FE35F6860EC606F61F1617162FB
:1008C000F2627163EF636C64E8646365DD655766CB
:1008D000CF664667BD673268A66819698C69FD698D
:1008E0006D6ADC6A4A6BB86B246C8F6CF96C626D54
:1008F000CA6D306E966EFB6E5F6FC16F2370837032
:10090000E27041719E71FA715572AF7207735F7335
:10091000B5730B745F74B27404755575A575F47571
:1009200041768E76D97623776C77B477FA774078EC
:100930008478C77809794A798A79C879057A427AB8
:100940007D7AB67AEF7A267B5D7B927BC57BF87BDE
:10095000297C5A7C897CB77CE37C0F7D397D627D64
:100960008A7DB07DD67DFA7D1D7E3F7E5F7E7F7E57
:100970009D7EBA7ED57EF07E097F217F387F4D7FB8
:10098000627F757F877F977FA77FB57FC27FCE7F8E
:10099000D87FE17FE97FF07FF67FFA7FFD7FFF7FE1
:0C09A00036303356312E34370000000092
:1009AC0001000000EB646E01000102000008000071
:1009BC000100000002000000000000000000000028
:1009CC00000000000000000000000000F401000026
:1009DC00000000000000000000000000000000000B
:1009EC00000000000000000000000000A00F00004C
:1009FC000F0E0000A00F0000F4010000000000002A
:100A0C000500000005000000D007000000000000F9
:100A1C00F40100000000000000000000F4010000E0
:100A2C00010000000100000000000000C8000000F0
:100A3C00C800000000000000F401000001000000EC
:100A4C0000080000640000000000E8030000000043
:100A5C000000010100000000320000003200000024
:100A6C0000000000F40100003C00000050000000F9
:100A7C0000000000E803000000000000DC0500009E
:100A8C00A00F0000000000000000000000000000AB
:100A9C00D0020000A00F00000000000000000000C9
:100AAC00E803000020030000200300000000000009
:100ABC00E803000001000000010000000039030001
:100ACC009033000000000000D00700000000000080
:100ADC00000000000000000000000000000000000A
:100AEC0000000000000000000000000000000000FA
:100AFC00000000000014101512131100000B161A40
:100B0C0025293400000D1319262C32000011131264
:100B1C00151014000100000000C2010000000800C4
:100B2C002C0301080400000030030108260000001B
:100B3C005803010832000000E00100201A000000F8
:100B4C00E802010843000000D40201081200000072
:100B5C00D19E0008DD9C00082D9B0008419B0008DD
:100B6C00459B0008A59B0008C99B0008CD9C00086C
:100B7C00BD9C0008999C000800000000400000008B
:100B8C001A034500760061006C003600300033001B
:100B9C000000000000000000000000002D9A00087A
:100BAC004DC600084DC600084DC600084DC60008CD
:100BBC004DC600084DC600084DC600084DC60008BD
:100BCC002D9E00084DC600084DC600084DC60008F5
:100BDC004DC60008040100004DC60008099B000822
:100BEC004DC600084DC600084DC600084DC600088D
:100BFC004DC600084DC60008219B000801000000EE
:040C0C00A009010832
:04000005080041109E
:00000001FF
